:1000000080720120B554000073390700A15400002C
:10001000A1540000A1540000A1540000A15400000C
:10002000000000000000000000000000ED5400008F
:10003000A15400000000000039570000A154000046
:10004000F9570000F9570000F9570000F957000070
:10005000F9570000F9570000F9570000F957000060
:10006000F9570000F9570000F9570000F957000050
:10007000F9570000F9570000F9570000F957000040
:10026000F9570000F9570000A1670200F957000094
:10027000F9570000F9570000F9570000F95700003E
:10028000F9570000F9570000F9570000F95700002E
:10029000F9570000F9570000F9570000F95700001E
:1002A000F9570000F9570000F9570000F95700000E
:1004C80081F0004102E000BF83F0004330B54FEAFD
:1004D80041044FEA430594EA050F08BF90EA020F6A
:1004E8001FBF54EA000C55EA020C7FEA645C7FEAFD
:1004F800655C00F0E2804FEA5454D4EB5555B8BF20
:100508006D420CDD2C4480EA020281EA030382EA90
:10051800000083EA010180EA020281EA0303362D22
:1005280088BF30BD11F0004F4FEA01314FF4801CF5
:100538004CEA113102D0404261EB410113F0004F07
:100548004FEA03334CEA133302D0524263EB4303BE
:1005580094EA050F00F0A780A4F10104D5F1200E5C
:100568000DDB02FA0EFC22FA05F2801841F10001B7
:1005780003FA0EF2801843FA05F359410EE0A5F18B
:1005880020050EF1200E012A03FA0EFC28BF4CF0BC
:10059800020C43FA05F3C01851EBE37101F0004572
:1005A80007D54FF0000EDCF1000C7EEB00006EEB7F
:1005B8000101B1F5801F1BD3B1F5001F0CD3490809
:1005C8005FEA30004FEA3C0C04F101044FEA445260
:1005D80012F5800F80F09A80BCF1004F08BF5FEAE7
:1005E800500C50F1000041EB045141EA050130BDC7
:1005F8005FEA4C0C404141EB0101013C28BFB1F5D9
:10060800801FE9D291F0000F04BF01460020B1FA23
:1006180081F308BF2033A3F10B03B3F120020CDAF6
:100628000C3208DD02F1140CC2F10C0201FA0CF0D4
:1006380021FA02F10CE002F11402D8BFC2F1200C39
:1006480001FA02F120FA0CFCDCBF41EA0C019040EF
:10065800E41AA2BF01EB0451294330BD6FEA040438
:100668001F3C1CDA0C340EDC04F11404C4F1200223
:1006780020FA04F001FA02F340EA030021FA04F335
:1006880045EA030130BDC4F10C04C4F1200220FA8C
:1006980002F001FA04F340EA0300294630BD21FACA
:1006A80004F0294630BD94F0000F83F4801306BF90
:1006B80081F480110134013D4EE77FEA645C18BF84
:1006C8007FEA655C29D094EA050F08BF90EA020F1B
:1006D80005D054EA000C04BF1946104630BD91EA13
:1006E800030F1EBF0021002030BD5FEA545C05D116
:1006F8004000494128BF41F0004130BD14F5800455
:100708003CBF01F5801130BD01F0004545F0FE41C8
:1007180041F470014FF0000030BD7FEA645C1ABFFD
:10072800194610467FEA655C1CBF0B46024650EA34
:10073800013406BF52EA033591EA030F41F4002160
:1007480030BD00BF90F0000F04BF0021704730B5E6
:100758004FF4806404F132044FF000054FF00001BB
:1007680050E700BF90F0000F04BF0021704730B57C
:100778004FF4806404F1320410F0004548BF404251
:100788004FF000013EE700BF42004FEAE2014FEAA6
:1007980031014FEA02701FBF12F07F4393F07F4F81
:1007A80081F06051704732F07F4208BF704793F084
:1007B8007F4F04BF41F40021704730B54FF4607497
:1007C80001F0004521F000411CE700BF50EA01029A
:1007D80008BF704730B54FF000050AE050EA010243
:1007E80008BF704730B511F0004502D5404261EBB3
:1007F80041014FF4806404F132045FEA915C3FF4F4
:10080800D8AE4FF003025FEADC0C18BF03325FEA90
:10081800DC0C18BF033202EBDC02C2F1200300FA41
:1008280003FC20FA02F001FA03FE40EA0E0021FA66
:1008380002F11444BDE600BF70B54FF0FF0C4CF454
:10084800E06C1CEA11541DBF1CEA135594EA0C0F06
:1008580095EA0C0F00F0DEF82C4481EA030621EA41
:100868004C5123EA4C5350EA013518BF52EA03357C
:1008780041F4801143F4801338D0A0FB02CE4FF02E
:100888000005E1FB02E506F00042E0FB03E54FF05E
:100898000006E1FB03569CF0000F18BF4EF0010E56
:1008A800A4F1FF04B6F5007F64F5407404D25FEA52
:1008B8004E0E6D4146EB060642EAC62141EA555105
:1008C8004FEAC52040EA5E504FEACE2EB4F1FD0C47
:1008D80088BFBCF5E06F1ED8BEF1004F08BF5FEAC5
:1008E800500E50F1000041EB045170BD06F0004677
:1008F80046EA010140EA020081EA0301B4EB5C0424
:10090800C2BFD4EB0C0541EA045170BD41F480111B
:100918004FF0000E013C00F3AB8014F1360FDEBF40
:10092800002001F0004170BDC4F10004203C35DA1C
:100938000C341BDC04F11404C4F1200500FA05F39F
:1009480020FA04F001FA05F240EA020001F0004240
:1009580021F0004110EBD37021FA04F642EB0601B6
:100968005EEA430E08BF20EAD37070BDC4F10C04E0
:10097800C4F1200500FA04F320FA05F001FA04F2A4
:1009880040EA020001F0004110EBD37041F1000190
:100998005EEA430E08BF20EAD37070BDC4F120059B
:1009A80000FA05F24EEA020E20FA04F301FA05F203
:1009B80043EA020321FA04F001F0004121FA04F2AB
:1009C80020EA020000EBD3705EEA430E08BF20EA7B
:1009D800D37070BD94F0000F0FD101F000464000B5
:1009E80041EB010111F4801F08BF013CF7D041EA37
:1009F800060195F0000F18BF704703F0004652003B
:100A080043EB030313F4801F08BF013DF7D043EA0B
:100A18000603704794EA0C0F0CEA135518BF95EAC1
:100A28000C0F0CD050EA410618BF52EA4306D1D148
:100A380081EA030101F000414FF0000070BD50EA67
:100A4800410606BF1046194652EA430619D094EAF1
:100A58000C0F02D150EA013613D195EA0C0F05D1DB
:100A680052EA03361CBF104619460AD181EA03012F
:100A780001F0004141F0FE4141F470014FF00000E7
:100A880070BD41F0FE4141F4780170BD70B54FF082
:100A9800FF0C4CF4E06C1CEA11541DBF1CEA135502
:100AA80094EA0C0F95EA0C0F00F0A7F8A4EB0504E4
:100AB80081EA030E52EA03354FEA013100F08880DB
:100AC8004FEA03334FF0805545EA131343EA1263A4
:100AD8004FEA022245EA111545EA10654FEA002659
:100AE8000EF000419D4208BF964244F1FD0404F512
:100AF800407402D25B084FEA3202B61A65EB03056E
:100B08005B084FEA32024FF480104FF4002CB6EB2A
:100B1800020E75EB030E22BFB61A754640EA0C00AA
:100B28005B084FEA3202B6EB020E75EB030E22BFEA
:100B3800B61A754640EA5C005B084FEA3202B6EB2B
:100B4800020E75EB030E22BFB61A754640EA9C00EA
:100B58005B084FEA3202B6EB020E75EB030E22BFBA
:100B6800B61A754640EADC0055EA060E18D04FEA78
:100B7800051545EA16754FEA06164FEAC30343EA18
:100B880052734FEAC2025FEA1C1CC0D111F4801FE5
:100B98000BD141EA00014FF000004FF0004CB6E7DE
:100BA80011F4801F04BF01430020B4F1FD0C88BF7D
:100BB800BCF5E06F3FF6AFAEB5EB030C04BFB6EB88
:100BC800020C5FEA500C50F1000041EB045170BD7B
:100BD8000EF0004E4EEA113114EB5C04C2BFD4EBA8
:100BE8000C0541EA045170BD41F480114FF0000E2C
:100BF800013C90E645EA060E8DE60CEA135594EAA8
:100C08000C0F08BF95EA0C0F3FF43BAF94EA0C0FAA
:100C18000AD150EA01347FF434AF95EA0C0F7FF41F
:100C280025AF104619462CE795EA0C0F06D152EA73
:100C380003353FF4FDAE1046194622E750EA410657
:100C480018BF52EA43067FF4C5AE50EA41047FF468
:100C58000DAF52EA43057FF4EBAE12E74FF0FF3CCD
:100C680006E000BF4FF0010C02E000BF4FF0010C9E
:100C78004DF804CD4FEA410C7FEA6C5C4FEA430C17
:100C880018BF7FEA6C5C1BD001B050EA410C0CBF66
:100C980052EA430C91EA030F02BF90EA020F0020C8
:100CA800704710F1000F91EA030F58BF994208BF2F
:100CB80090422CBFD8176FEAE37040F001007047EC
:100CC8004FEA410C7FEA6C5C02D150EA013C07D143
:100CD8004FEA430C7FEA6C5CD6D152EA033CD3D08E
:100CE8005DF8040B704700BF8446104662468C4688
:100CF8001946634600E000BF01B5FFF7B7FF0028BB
:100D080048BF10F1000F01BD4DF808EDFFF7F4FFE3
:100D18000CBF012000205DF808FB00BF4DF808ED6E
:100D2800FFF7EAFF34BF012000205DF808FB00BF91
:100D38004DF808EDFFF7E0FF94BF012000205DF8B3
:100D480008FB00BF4DF808EDFFF7CEFF94BF012068
:100D580000205DF808FB00BF4DF808EDFFF7C4FF61
:100D680034BF012000205DF808FB00BF4FEA4102B4
:100D780012F5001215D211D56FF47873B3EB6252E5
:100D880012D94FEAC12343F0004343EA505311F00C
:100D9800004F23FA02F018BF404270474FF000009E
:100DA800704750EA013005D111F0004008BF6FF0DC
:100DB800004070474FF00000704700BF4FEA410203
:100DC800B2F1E04324BFB3F5001CDCF1FE5C0DD9A1
:100DD80001F0004C4FEAC0024CEA5070B2F1004FEB
:100DE80040EB830008BF20F00100704711F0804FEE
:100DF80021D113F13872BCBF01F00040704741F4B3
:100E080080114FEA5252C2F11802C2F1200C10FAB6
:100E18000CF320FA02F018BF40F001004FEAC1239A
:100E28004FEAD32303FA0CFC40EA0C0023FA02F33E
:100E38004FEA4303CCE77FEA625307D150EA013314
:100E48001EBF4FF0FE4040F44000704701F00040E4
:100E580040F0FE4040F40000704700BF80F00040C2
:100E680002E000BF81F0004142001FBF5FEA41037A
:100E780092EA030F7FEA226C7FEA236C6AD04FEA7A
:100E88001262D2EB1363C1BFD218414048404140BF
:100E9800B8BF5B42192B88BF704710F0004F40F471
:100EA800000020F07F4018BF404211F0004F41F48D
:100EB800000121F07F4118BF494292EA030F3FD059
:100EC800A2F1010241FA03FC10EB0C00C3F120036C
:100ED80001FA03F100F0004302D5494260EB4000FB
:100EE800B0F5000F13D3B0F1807F06D340084FEA66
:100EF800310102F10102FE2A51D2B1F1004F40EB5B
:100F0800C25008BF20F0010040EA030070474900C2
:100F180040EB0000013A28BFB0F5000FEDD2B0FA5F
:100F280080FCACF1080CB2EB0C0200FA0CF0AABF82
:100F380000EBC25052421843BCBFD0401843704720
:100F480092F0000F81F4000106BF80F40000013226
:100F5800013BB5E74FEA41037FEA226C18BF7FEAFD
:100F6800236C21D092EA030F04D092F0000F08BF3F
:100F78000846704790EA010F1CBF0020704712F026
:100F88007F4F04D1400028BF40F00040704712F165
:100F980000723CBF00F50000704700F0004343F0CA
:100FA800FE4040F4000070477FEA226216BF084600
:100FB8007FEA23630146420206BF5FEA412390EAC3
:100FC800010F40F4800070474FF0000304E000BFB9
:100FD80010F0004348BF40425FEA000C08BF70476A
:100FE80043F0964301464FF000001CE050EA01022E
:100FF80008BF70474FF000030AE000BF50EA010243
:1010080008BF704711F0004302D5404261EB41012F
:101018005FEA010C02BF84460146002043F0B64354
:1010280008BFA3F18053A3F50003BCFA8CF2083A79
:10103800A3EBC25310DB01FA02FC634400FA02FC82
:10104800C2F12002BCF1004F20FA02F243EB020089
:1010580008BF20F00100704702F1200201FA02FCEB
:10106800C2F1200250EA4C0021FA02F243EB0200DE
:1010780008BF20EADC7070477BB972B90029BEBF8F
:1010880000204FF0004106E008BF00281CBF6FF0A9
:1010980000414FF0FF3000F077B8ADF1080C6DE972
:1010A80004CE002909DB002B1ADB00F0A9F8DDF8D3
:1010B80004E0DDE9022304B07047404261EB4101DE
:1010C800002B1BDB00F09CF8DDF804E0DDE90223CF
:1010D80004B0404261EB4101524263EB4303704765
:1010E800524263EB430300F08BF8DDF804E0DDE9DE
:1010F800022304B0404261EB41017047524263EB66
:10110800430300F07DF8DDF804E0DDE9022304B0D4
:10111800524263EB4303704753B94AB9002908BFE9
:1011280000281CBF4FF0FF314FF0FF3000F02CB803
:10113800ADF1080C6DE904CE00F062F8DDF804E0CA
:10114800DDE9022304B07047D0B5FFF71DFB00228C
:101158000B4B06460F46FFF76FFB00F017F80446E7
:10116800FFF7F0FA0022074BFFF766FB02460B4633
:1011780030463946FFF7A8F900F008F82146D0BDF7
:101188000000F03D0000F041704700BF4A0011D256
:1011980012F5001211D20DD56FF47873B3EB6252C9
:1011A8000ED44FEAC12343F0004343EA505323FAD5
:1011B80002F070474FF00000704750EA013002D14A
:1011C8004FF0FF3070474FF00000704710F8012BC8
:1011D80011F8013B012A28BF9A42F7D0D01A70476C
:1011E800034611F8012B03F8012B002AF9D17047A7
:1011F800034613F8012B002AFBD1181A013870474F
:101208002DE9F0478C468E46089E15460446194639
:10121800002B40F0D080724547D9B2FA82F74FB11F
:10122800C7F120030EFA07FCBD40BC4020FA03F3C7
:1012380043EA0C0C4FEA154EA8B2230CBCFBFEF88F
:101248000EFB18CC08FB00F943EA0C43994528D952
:10125800EB1808F1FF3204D2994502D9A8F102022D
:101268002B44A3EB0903A4B2B3FBFEFC0EFB1C3317
:101278000CFB00F044EA0344A04214D92C190CF1E9
:10128800FF3304D2A04202D9ACF102032C44241A41
:1012980043EA02401EB1FC40002334607360BDE89D
:1012A800F0874246DDE76346F1E7002A79D0B2FAD3
:1012B80082F3002B3FD01946C1F1200302FA01F551
:1012C80000FA01F42EFA03F20EFA01FE20FA03F3F3
:1012D800AFB243EA0E034FEA154EB2FBFEFC0EFB1B
:1012E8001C201A0C0CFB07F842EA004290455AD918
:1012F800AA180CF1FF3004D2904502D9ACF10200D3
:101308002A44A2EB08029BB2B2FBFEFC0EFB1C2295
:101318000CFB07F743EA02439F4246D9EB180CF14E
:10132800FF3204D29F4202D9ACF102022B44DB1BEC
:1013380042EA004202E0AEEB020301224FEA154EF8
:10134800AFB2200CB3FBFEFC0EFB1C330CFB07F802
:1013580040EA034398452AD9EB180CF1FF3004D230
:10136800984502D9ACF102002B44A3EB0803A4B2C0
:10137800B3FBFEFC0EFB1C330CFB07F744EA0344EB
:10138800A74216D92C190CF1FF3304D2A74202D96F
:10139800ACF102032C44E41B43EA00400F4611461B
:1013A80078E71F2188E76046ABE76246BFE76046FB
:1013B800DBE76346EFE7734506D916B9002108460F
:1013C8006DE7C6E9000EF9E7B3FA83F787B9734505
:1013D80001D3824207D8841A6EEB030301209C468E
:1013E8001EB900215BE73846FAE7C6E9004CF8E782
:1013F800C7F1200CBB4000FA07F422FA0CF520FADA
:101408000CF1BA401D432EFA0CF30EFA07FE4FEA10
:10141800154941EA0E011FFA85FEB3FBF9F809FBED
:1014280018300B0C08FB0EFA43EA00439A4540D9E2
:10143800EB1808F1FF3004D29A4502D9A8F102004E
:101448002B44A3EB0A0389B2B3FBF9F809FB183361
:1014580008FB0EFE41EA03418E452CD9691808F1B4
:10146800FF3304D28E4502D9A8F10203294443EA86
:101478000040A1EB0E01A0FB02984145CE46434631
:1014880002D306D14C4504D20138B9EB020E68EB01
:101498000503002EA5D0B4EB0E0261EB030101FA9F
:1014A8000CFC22FA07F3F9404CEA0303C6E90031C1
:1014B80097E74046C5E74346D9E70000000000002B
:1014C8000022F0B5114640F6034085B008F004FF4D
:1014D8000446002856D108F077F9214641F2030066
:1014E80003AA08F0F9FE044600284BD1039A274DB9
:1014F800D16805F12C03D1F80100D1F8051003C318
:10150800104604F03DFD214641F2010003AA08F00F
:10151800E3FE0446002835D10398C3685A7885F855
:1015280023205A88EA841A7985F82420B3F80720FA
:101538002A85B3F805306B8504F022FD214641F277
:10154800020003AA08F0C8FE0446D8B9039F05F1B3
:101558003406FA68531C413234461868596808330F
:1015680003C493422646F7D1384604F009FD95F89E
:101578003030580610D40121054A064873F048FE59
:101588006FF01204204605B0F0BD00BF80010020B6
:10159800AB600A00786B0900002142F2030003AA3D
:1015A80008F09AFE04460028ECD1039AC04BD16893
:1015B800D1F80100D1F8051003C3104604F0E0FC8F
:1015C800214642F2020003AA08F086FE04460028DB
:1015D800D8D1039EF468B4F801309AB292B1E27897
:1015E80082B1A5F8BC30E378032B06D00322022190
:1015F8000092B048B04A71F0B7FEE278AF481146A1
:1016080079F025F9304604F0BBFC002142F23A009B
:1016180003AA08F061FE0446002840F020810398E0
:10162800C368B3F80130A5F8D83004F0A9FC95F8E0
:10163800306016F0200619D14FF0FF304FF0FF311F
:1016480008F078FC0446002800F0768102210C306E
:1016580072F098FA0123214603704670324640F62C
:101668006D4008F039FE044600288BD195F85030BB
:101678001A0713D5002142F21C0003AA08F02CFE19
:10168800044600287FF47EAF0398C368D3F801208E
:10169800D3F80530C5E9262304F072FC95F890309C
:1016A8009B0626D50DF10A0102A808F0BFFE0446E4
:1016B80000287FF467AF4FF0FF304FF0FF3108F09C
:1016C80039FC0646002800F0378104210C3072F0FE
:1016D80059FABDF8083022460380BDF80A30314671
:1016E800438042F2240008F0F7FD044600287FF406
:1016F80049AF95F890305F0610D5002142F22A00D4
:1017080003AA08F0E9FD044600287FF43BAF0398DC
:10171800C3685B7885F8DA3004F032FC4FF0FF30AC
:101728004FF0FF3108F006FC0446002800F0048161
:1017380008210C3072F026FA95F89010024660489D
:1017480011F0020F5F4B08BF034695F891008E0613
:1017580048BF43F0400310F0090F18BF43F400637B
:1017680001F0010143EA0110002173F075FD2146E3
:10177800002242F2010008F0AFFD044600287FF481
:1017880001AF95F83030B5F8BC10980673D4C9B9D4
:1017980041F2050003AA08F09FFD044600287FF4E3
:1017A800F1AEB5F8BC30039C4BB9E368B3F801203F
:1017B800A5F8BC209A884148114679F048F8204697
:1017C80004F0DEFB4FF0FF304FF0FF3108F0B2FBC2
:1017D8000446002800F0B08008210C3072F0D2F9DD
:1017E80095F890300246D90747BF2FA1D1E90001EB
:1017F8004FF00051344873F02FFD2146002240F687
:10180800014008F069FD044600287FF4BBAE01469C
:1018180003AA4FF6014008F05FFD0446002834D0C3
:101828002A4A0221234873F0F3FCEB79002B74D188
:1018380073F0ABFF044600287FF4A4AE0CF072FCF2
:10184800044600287FF49EAEEB79002B3FF49AAE55
:1018580008211F4873F0E5FC08F070FC92E6411D72
:101868007FF490AE02211B4A124873F0D1FC1F236B
:10187800A5F8D830DBE60029A4D10121164A0D4885
:1018880073F0C6FC6FF004047CE6039804F078FB60
:1018980021464FF6024003AA08F01EFD0446F8B19F
:1018A8000E4ABEE7AFF30080908800020080002057
:1018B80010020020786B0900CF600A004002002067
:1018C8000E1207002E1207001088000295610A0008
:1018D8000802002015610A0072610A00B9610A0055
:1018E8000398C368B3F80130A5F8753004F048FBD5
:1018F80095F875305A0798D521464FF6034003AA44
:1019080008F0EAFC08B11A4A8BE70398C3685B78C9
:1019180085F8743004F034FB87E72E78002E87D1E1
:1019280095F875309B061FD54FF0FF304FF0FF310B
:1019380008F000FB044610B96FF0680422E606219F
:101948000C3072F01FF9D5F8013021460360094BBD
:1019580032469B8883804FF6064008F0BDFC04465B
:1019680000283FF465AF0DE66FF085040AE600BF76
:10197800E2610A00810100204FF0FF329FED0A7BEF
:101988000D4B00211A6000200C4B002283ED007BD8
:101998009FED077B0A4BC3E900010A490A4B81ED19
:1019A800007B1A6016F08EB9FFFFFFFFFF1F0000D3
:1019B8001F000000000000007487002000030020C2
:1019C800803E0020F80200206C8700200000000004
:1019D8002DE9F047044640F2712690F8623090F8FD
:1019E800382023F00103C3F3800060F386128CB023
:1019F80004F1460184F8623084F8382014F0E6FED9
:101A0800B4F84C300022A3FB0663A36D484D236550
:101A180003F5D673B34228BF33464649A4EB050500
:101A2800A1FB051594F83810C5F3471501F07901A5
:101A3800DFF81091C4E90222227032BF6360666049
:101A4800226584F8381005EB4502246149F82230F4
:101A580014F016FE63694FEA450A00F5D677002BA5
:101A68004BD00DF12C089121AA4409EB8A034FF0C1
:101A780000094FF0020A0993CDF820800694B4F8C3
:101A88004C302D4A2D480792A3FB000201FB03218D
:101A98002B4BCDF80C9005936368CDF82CA00493DC
:101AA80021A3D3E90023FFF737FB104619464FF46B
:101AB8007A720023FFF730FB0535EDB20321CDE93B
:101AC80001603B462A464846CDF8009014F05EFC7B
:101AD800414615F08DFC60B994F8623043EA0A0378
:101AE80084F8623019F0E0FBB8B100200CB0BDE812
:101AF800F0870C200CB0BDE8F0870DF12C08CDE97B
:101B08000A330320434661680AAA23F011FB002820
:101B1800A9D1DDE90A371F44A5E7504624F034F976
:101B2800E3E700BFAFF3008000CA9A3B0000000063
:101B3800E08A00201F85EB514D680100002AE784E8
:101B480055D50100D48A002070B50D46044600F131
:101B58008F06334600223B3105F12B002AF05AFE4E
:101B680000229FED2D7BD4F89B30D4F89710C4F851
:101B7800BC30D4F8AC30D4F89300C4F8CD3094F825
:101B8800C830D4F88FC043F0010384F8C83094F803
:101B9800A730C4F8B810D4F8A81062F30003C4F84A
:101BA800B400C4F8C9102046294684ED307BC4F837
:101BB800B0C084F89F2084F8A02084F8A12084F87D
:101BC800A22084F8A32084F8A42084F8A52084F80F
:101BD800A62084F8A7301FF08DFA0646B8B1301D4C
:101BE80020F08CFEF37931466B7320461FF098FA8B
:101BF800204620F097FB40F206636B8194F88E3004
:101C080023F0180343F0180384F88E3070BD00DE0B
:101C1800E5E700BFAFF3008000000000000000000F
:101C280070B504460D461FF05DFA10B90623AB7275
:101C380070BD04F18F063346002205F13B0105F122
:101C48002B002AF0E7FD00229FED2B7BD4F89B3078
:101C5800D4F89710C4F8BC30D4F8AC30D4F893005A
:101C6800C4F8CD3094F8C830D4F88FC062F30003BC
:101C780084F8C83094F8A730C4F8B810D4F8A8107D
:101C880043F00103C4F8B400C4F8C910204629463B
:101C980084ED307BC4F8B0C084F89F2084F8A0207D
:101CA80084F8A12084F8A22084F8A32084F8A42032
:101CB80084F8A52084F8A62084F8A7301FF01AFA23
:101CC8000646A8B1301D20F00FFEF37931466B733C
:101CD80020461FF025FA204621F0F8FF4FF4C16393
:101CE8006B8194F88E3043F0080384F88E3070BD11
:101CF80000DEE7E7AFF3008000000000000000000E
:101D08002DE9F04F03699146D3F8A460436891F830
:101D18002000D3F800B000F07F0440B20028B8BF1C
:101D2800A2464FF0010396F8C623A9BF04F158074D
:101D380004F1480704F1100A0BEB4717B8BF0BEB87
:101D4800471712F0100288463D6803FA0AF185B079
:101D580006F1F40334D0A4000028344417DBD4F887
:101D68003C2222F00042B9F1000F0DD042F40012DB
:101D7800C4F83C22184676F0F3FB0021404605B033
:101D8800BDE8F04F76F01FB842F00062F0E7D4F8F3
:101D98007C2122F00042B9F1000F0ED142F000621E
:101DA8000120C4F87C21C2F3835200FA02F2B6F88B
:101DB8009E030243A6F89E23DCE742F00262EFE7A7
:101DC8009FED377B18468DED007B0391029379F0E8
:101DD80042F9DDE90231D8B1B9F1000F02D045F47A
:101DE80000153D6001224FEA5A130AF01F0A02FA51
:101DF8000AF2D24306EB830303F58073D3E8EF0FAF
:101E08001040C3E8E10F0029F8D105B0BDE8F08F14
:101E180098F92020002A32DBEFF31180202282F388
:101E28001288BFF36F8F0122A240B6F8984392B28E
:101E38001443A6F89843B9F1000F04D0B6F89A43B2
:101E48002243A6F89A23DBF8042842F40072CBF860
:101E5800042880F31188BFF36F8F40F635440025BE
:101E680000221846CDE9004579F0F5F8002884D11C
:101E780098F820200C490D4876F00EFB7DE7B9F163
:101E8800000F09D145F00065AA0303D5002DB8BF9E
:101E980045F080453D60E0E745F00265F4E700BFA6
:101EA8000000000000000000F8800A00986C09009B
:101EB8002DE9F04F984685B000F15803C0E9163374
:101EC800129B0026838104239FED257B073222F095
:101ED800070A0374119B01EB0A090F4680ED087B82
:101EE8004946C0E9066686608373C6730446DDF812
:101EF80038B003F087F8109BC51D25F00705C4F816
:101F08008850C4E9207A02930F9BA9EB0505CDE917
:101F180000B32A4643463946204603F06DFB0F9B23
:101F2800C4E91B8B6367109B6665A367EFF3118297
:101F3800202383F31288BFF36F8F0B4B596A5C62BF
:101F4800E16782F31188BFF36F8F9B680BB1D3F8F9
:101F58008C302846C4F88C3005B0BDE8F08F00BF3F
:101F6800000000000000000024A500200000000080
:101F780030B5144617A3D3E9002385B0FFF77CF8E2
:101F8800054601A928464CF04BFD9DF807309DF801
:101F980006201B0443EA42539DF808200C4943EAF3
:101FA800C2239DF8092025F0010543EA42139DF854
:101FB8000A20A5FB010143EA5203BDF80420A2F25E
:101FC800BC7243EA4263236005B030BDAFF30080C2
:101FD80000CA9A3B00CA9A3B0000000000000000BB
:101FE8002DE9F0412DED028B90F8A5300446B0EEB6
:101FF800408A86B01BB9F7EE007A37EEC08AD4F86B
:1020080084202F4B9A4213D118EE100AFEF7BCFB1E
:1020180029A3D3E90023FEF79FFE011E18BF012163
:1020280004F1840038F050F984ED268A012005E097
:10203800B4F89C30B3F5807F05D1002006B0BDEC24
:10204800028BBDE8F08104F15008404651F05EFC77
:102058000028F2D0DFED1B7A68EE277AFCEEE77AEB
:10206800CDED037A94F8806094F89C209DF80C30AC
:10207800276E206D6EB18DF8153002238DF814206F
:1020880000210122009305ABB847404684F00AFEC0
:10209800CAE7012531468DF813208DF814302A46F9
:1020A8000DF113030095B847009532462946276E6F
:1020B800206D05ABE8E700BFAE47E17A14AEEF3F0D
:1020C80088F2090000007F432DE9F04F044685B0EF
:1020D80008466160062190461D469DF838709DF8B7
:1020E8003CB03AF035FEA060067C16F0010602D03E
:1020F8007F483BF0F7FF9DF8403005FB08F084F877
:102108002A309DF844307D3084F828307E2390FBB7
:10211800F3F0C0011630B0F5D07F38BF4FF4D0705F
:10212800C4E90485277360627FF02AF90DF1080A73
:102138000622C4E907066F492046A66191F0C7FE4A
:10214800022251462046ADF8088091F0C0FE0222D6
:1021580051462046ADF8085091F0B9FEF623032207
:1021680069462046ADF800308DF8026091F0AFFE68
:102178007B1EDBB2082B05D840F25515DD4015F063
:10218800010501D15C48B4E7052F09D0072F06D017
:10219800032F73D1012384F82930002502E02E464D
:1021A80084F82960002646F34F10C0EB0020FEF7A4
:1021B800D9FA0022514BFEF789F90022504BFEF75D
:1021C80065FCFEF7D3FD5FFA80F8C6F38200C0EB2A
:1021D8000020FEF7C7FA00224A4BFEF777F90022E3
:1021E800494BFEF753FCFEF7C1FDC7B206F00300EA
:1021F800C0EB0020FEF7B6FA0022404BFEF766F966
:1022080000223F4BFEF742FCFEF7B0FDC0B2002DA6
:102218005ED08DF808008DF809808DF80A700322C9
:1022280051462046013691F052FE802EBBD1BBF1BB
:10223800000F1AD0354D01A92A88AB782046ADF891
:10224800042003228B7091F042FE0B222046304975
:1022580091F03DFED5F80300EB7902900522514636
:1022680020468AF8043091F032FE204691F01DFE97
:10227800A06991F03EFE05B0BDE8F08F092F84F803
:1022880029608AD10FF25809D9E90089354616A77D
:10229800D7E900672846FEF765FA42464B46FEF73F
:1022A80015F932463B46FEF7F1FBFEF75FFDC0B27B
:1022B8008DF808008DF809008DF80A0003225146B0
:1022C8002046FF3591F003FEB5F5FF4FE2D1AEE7AA
:1022D8008DF808808DF809708DF80A009FE700BF17
:1022E8000000000000C04F400000000000C05F4038
:1022F80011E60A0009C90A00DCDD0A000000F83FFF
:102308000000084000000C4000001C40556E090009
:10231800FDC80A000000000010EE103A33F0004239
:1023280010B52DED028B06D10120BDEC028BBDE866
:1023380010406EF0A7BE002B05DABDEC028BBDE89D
:1023480010406EF0ADBEB3F1FF4F06DB30EE008AF1
:10235800B0EE480ABDEC028B10BDB3F5000F604922
:10236800BBBFDFED607A6FF01802002260EE277ABB
:10237800B8BF17EE903AF7EE007ADC15C3F31603F0
:102388007F3C1944144401F4000282F07E5204EBAD
:10239800D15403F10F011A4307EE102A524A0A409A
:1023A80037EE678AB2BBB5EE408AF1EE10FA0FD16C
:1023B800002C00F08C8007EE904A9FED4C0A9FEDB0
:1023C8004C7AF8EEE77A27EE808A07EE878ABFE72D
:1023D80041A1D1E90001FEF7F1FCB6EE007A07EE63
:1023E800900A07EEC87A68EE087A27EE277A14B9B9
:1023F80038EE478AACE707EE904ADFED3C6AF8EE24
:10240800E77A07EEE67A37EE488A9FED397A17EED3
:10241800878A9DE7F0EE007A9FED365ADFED364A5F
:10242800364A78EE277A1A44C3F5571388EE276A96
:1024380007EE904A03F522731343F8EEE76ADFEDDF
:10244800307A002B66EE065A25EEA57A07EE275A53
:10245800DFED2C7A45EE077A9FED2B5A07EE875A67
:10246800DFED2A7A47EE274ADFED297A44EE877AAC
:1024780067EE877A45EE257A1ADDB6EE007A28EE01
:10248800077A27EE087A77EE877A67EE867A14B9A4
:1024980037EE677AACE79FED156A46EE867A37EE37
:1024A800677A37EE488ADFED127A16EEA78A4FE789
:1024B80078EE677A67EE867A14B938EE678A47E766
:1024C8009FED0A7A46EEC77A37EEC88AEBE79FEDAA
:1024D800118A3DE7AFF30080555555555555D53F01
:1024E80020FB4A000000004CF0FF7F00D1F71737AF
:1024F8008071313F25333A3E298E633E305CCFFFF1
:102508009788173E2549923EABAA2A3F4FD01C3EDA
:10251800CDCCCC3E00000000F8B510EE904A10EE8D
:10252800103A34F000472DED048BB0EE609A0DD1CF
:1025380083F480035B0013F5000F40F2AA8230EEAB
:10254800098AB0EE480ABDEC048BF8BD23F00041BF
:102558001846B1F1FF4F02D8B7F1FF4F08D9B3F1D0
:102568007E5FECD184F48004640014F5000FE4E786
:10257800002B25DAB7F1974F80F09482B7F17E5F90
:1025880039D3FA15C2F1960247FA02F505FA02F2B2
:10259800BA4229D105F00105C5F10205B7F17E5F00
:1025A8002AD1002C80F27B82B5EE400AF1EE10FAB7
:1025B8001CD1D80FBDEC048BBDE8F8406EF062BDAD
:1025C800B7F1FF4F10D1B1F17E5F00F0628205D9FB
:1025D800002CDFEDD17A29FE278AB2E7002C80F2A1
:1025E8005B82B1EE498AACE70025D7E7B7EE007AFF
:1025F80087EE008AA5E70025B4F1804F0A4640F02F
:102608005782B1F1BF4F0CD2B1F1D05F02D920EEA1
:10261800008A96E7B0EEC08A59BB012D00FE088AF1
:102628008FE723F04046B0EEC08AB6F17E5F17D13F
:10263800002CBCBFB7EE007A87EE088A002B80DA40
:10264800A1F17E51294305D1BDEC048BBDE8F840CA
:102658006EF026BD012D7FF474AFB1EE488A70E7A5
:1026680039B9002CD9DA002BA4D06B1E5842584136
:10267800A0E7DE0F013E55EA0600E5D0B7F19A4F14
:1026880071D9A64B994208D8002C0BDA0020BDEC72
:10269800048BBDE8F8406EF0E7BCA14B994208D91D
:1026A800002CF3DC0020BDEC048BBDE8F8406EF094
:1026B800CDBCB7EE007ADFED9B7ADFED9B9A38EE62
:1026C800478A93A1D1E9000168EE278AFEF776FBD5
:1026D800B5EE007A07EE900ADFED946A68EE299A63
:1026E80048EE477AB6EE007A07EEC87A68EE087ABE
:1026F80027EE277AF0EE687A47EE667A39EEA77AFF
:1027080017EE103A6FF30B0307EE103A77EE699A5B
:1027180077EEE97A013DF7EE006ABFEE008A6FF3C3
:102728000B04354367EE890A08FE268A06EE904AAE
:1027380039EE666A67EE267A46EE070A30EEA77A21
:1027480017EE101A002921F0004340F31381B3F16A
:10275800864F40F2CC80B5EEC08AF1EE10FA4CBF3D
:102768000120002093E713F0FF4F05BF9FED707A1B
:102778006FF01701002168EE077A08BF17EE902A5C
:10278800D315C2F316027F3B42F07E500B446949D1
:102798008A4206DD68498A4240F3A7800133A0F5E2
:1027A80000000021654A06EE100AF7EE006A02EB07
:1027B8008102D2ED005A75EE867A36EE657AC6EE5B
:1027C800A74A27EE245A15EE102A6FF30B0206EEDD
:1027D800902A5B4A02EA600242F0005202F5800247
:1027E80002EB415207EE902A06EEE77A77EEE57A99
:1027F800DFED545A36EE676A65EE057A06EE667ABC
:102808009FED516A47EE865A9FED506A27EE247A6B
:1028180066EEA64A05EEA76ADFED4D5A46EE275A40
:102828009FED4C6A05EEA76ADFED4B5A46EE275A34
:1028380036EE856A67EEA77A26EE076A05EEA76A7E
:10284800F0EE085A74EEA57A77EE867A17EE902A9B
:102858006FF30B0207EE902A77EEE55A27EE277AF8
:1028680066EEA76A75EEE45A36EE656A06EE057AF4
:102878009FED3A6A76EE877A17EE902A6FF30B028D
:1028880007EE902A364A77EEE66A02EB810227EED7
:10289800866A37EE667ADFED336A67EEA67ADFED91
:1028A800326A47EE267A92ED007A77EE877A07EE5B
:1028B800103A2E4BF8EEC76A03EB810336EE277AFF
:1028C800D3ED005A37EE257A37EE267A17EE103A0E
:1028D8006FF30B0307EE103A77EE666A76EEE56A59
:1028E80076EEC66A77EEE67A14E701215AE755D103
:1028F800DFED1F6A37EE677A70EEA66AF4EEC76AF4
:10290800F1EE10FA3FF727AF86234BE0AFF30080D4
:10291800E13D55555555D53F00000000F3FF7F3F79
:102928000700803F70A5EC3600AAB83F3BAAB83F25
:102938000000804B71C41C00D6B35D00FC390A004E
:1029480000F0FFDF55326C3E42F1533E05A38B3E4B
:10295800ABAAAA3EB76DDB3E9A99193F0040763F75
:10296800EC390A00C623F6B84F38763FF4390A0026
:102978003CAA3833534A934207D9B5EEC08AF1EEE0
:1029880010FA4CBF012000208DE607D137EE677A98
:10299800B4EEE07AF1EE10FAB6DBEEE7B3F17C5F65
:1029A80072D9DB157E3B4FF40000474A002940FAF4
:1029B80003F00844C0F3C753A3F17F0342FA03F2BC
:1029C800C3F1170302EA0002C0F3160040F4000046
:1029D80007EE102A40FA03F077EEC77AB8BF4042F4
:1029E80037EEA07ADFED396ADFED395AB7EE000A23
:1029F8009FED386A17EE103A6FF30B0307EE103AA3
:102A080077EE677A67EE266A70EEE70ADFED327ACC
:102A180027EE277ADFED317A00EEA77A76EE877A0D
:102A280077EEE66A37EE667A67EEA76A07EE877A88
:102A380016EEA56ADFED2A5A46EE265A9FED296A58
:102A480015EEA66ADFED285A46EE265AB0EE676AFA
:102A580005EEE66AF0EE006A67EE865A36EE666ABA
:102A6800C5EE866A36EEC77A77EE677A30EE670A81
:102A780010EE103A03EBC053B3F5000F06DA6EF010
:102A880069F920EE088A5CE50020A9E700EE103A13
:102A9800F7E7B7EE008A54E59FED148A51E5B0EEEA
:102AA800408A4EE5B7F1FF4F3FF48DAD0A46022547
:102AB800B4F17C5F7FF4B5AD002BFFF6B2ADB1EE9B
:102AC800C08A3EE500001643000080FF0072313FD7
:102AD8004CBB31330EEADD358CBEBF351872313F41
:102AE80055B38A38610B363BABAA2A3E000000007A
:102AF80010EE103AB3F1FF4F10B52DED048BB0EE88
:102B0800408A06DB30EE008AB0EE480ABDEC048B42
:102B180010BD774A934276DC23F00042B2F17E5F23
:102B280013D3FFEE007AB4EE670AF1EE10FA06D17D
:102B38000120BDEC048BBDE810406EF0A3BABDECDB
:102B4800048BBDE810406EF0ABBAB2F1645F0FD2EF
:102B5800B2F14A5F24BF20EE007AF6EE007ABDECAF
:102B6800048B28BF07EE670ABDE810406EF0ACB8CA
:102B7800604A134493424ED8F7EE007A38EE277A2B
:102B880017EE103ADC157F3C002CD5BF77EE677A3C
:102B980037EE488A78EE677A77EEC87A87EE879AB2
:102BA800C3F31603544A9342CCBF43F07C5243F01C
:102BB8007E52F7EE007AC8BFC3F5000307EE102A6D
:102BC800C4BF01349B1037EE678AF6EE008A68EEC0
:102BD800288A68EE888A002B44D1B5EE408AF1EE47
:102BE80010FA1DD1002C7AD007EE904AB0EE498A2F
:102BF8009FED427AF8EEE77A07EE878A9FED407AF2
:102C080007EE878A80E7B3F1B44FB5DBDC159FED9B
:102C18003D9A7F3CC4E7012300249FED3A9AD4E70C
:102C280031A1D1E90001FEF7C9F8B7EE007A07EE45
:102C3800900A07EEC87A27EE287A14B938EE478A40
:102C480062E707EE904ADFED2D6AF8EEE77A07EEC5
:102C5800A69A37EE497A37EE488A9FED297A17EE19
:102C6800878A51E7F0EE007A9FED276A9FED277A71
:102C780078EE277AC8EE276A66EEA67A07EE867A95
:102C88009FED236A07EE276A9FED227A06EE277AE0
:102C98009FED216A07EE276A9FED207A06EE277AD4
:102CA8009FED1F6A07EE276AB0EE687A06EE277A6C
:102CB80027EE267A24B978EEC78A38EE688A23E7A1
:102CC80007EE904ADFED0D6AF8EEE77A07EEA69A6E
:102CD80039EE079A78EEC98A38EEC88ABDE79FEDC3
:102CE800098A11E7AFF30080555555555555E53F0D
:102CF800D613D43EE0096A41F6043500D1F71737F8
:102D08008071313F000000009788173E4FD01C3E6D
:102D180025333A3E298E633E2549923ECDCCCC3EA2
:102D2800ABAA2A3F2DE9F0470546884600AF6EF06A
:102D3800F8FDA9680646B1F5004F36BFA8F10403AF
:102D4800002303F00703B1F5004F34BF0420082027
:102D580002F0070407341C440444E40804EBD204DA
:102D68008C4228BF0C460122314628466EF093FD5E
:102D780010EA020A16D1E94688B06A46504BCDE9F6
:102D88000538032342F8103F4FF4C25153464D48CB
:102D980001F006FACD468AF31188BFF36F8F04233A
:102DA800184602DF314628466EF08BFD06EB000917
:102DB8004946002228466EF06EFDA9EB00094E45F3
:102DC80018D0E94688B069463F4BCDE9053803235A
:102DD80041F8103F3B4813460A464FF4C25101F0F0
:102DE800DFF90023CD4683F31188BFF36F8F0423E7
:102DF800184602DF314628466EF063FD844280465D
:102E080023D028D234443146224628466EF01BFE91
:102E18000122314628466EF05AFD21466EF051FDDA
:102E280026180122314628466EF035FDC30708D41E
:102E3800314628466EF0B7FD3246214628466EF0E8
:102E480029FE214628466EF043FE4FF00109484608
:102E5800BD46BDE8F08706EB000A01225146284628
:102E68006EF019FD10EA020927D1514628466EF086
:102E780028FD40448442EAD8514628466EF093FD26
:102E8800514628466EF01DFDA4EB0808804509D27E
:102E980034445146284622466EF0D5FD2146284640
:102EA8006EF016FE5246314628466EF0F3FD0122BA
:102EB800314628466EF00BFDC7E74FF00009C6E71C
:102EC8005A440A00586C09007E440A002DE9F84368
:102ED800884600AF00297DD00568012228466EF09B
:102EE80020FD0146044628466EF0D5FC10EA02068D
:102EF80016D1E94688B06A46384BCDE90538032330
:102F080042F8103F4FF4C2513346354801F048F9B2
:102F1800CD4686F31188BFF36F8F0423184602DF6E
:102F2800214628466EF0CDFC261831460022284658
:102F38006EF0B1FC361AB44218D06E4688B06946B5
:102F4800284BCDE90538032341F8103F24481346A0
:102F58000A464FF4C25101F023F90023B54683F322
:102F68001188BFF36F8F0423184602DF0022214621
:102F780028466EF0ACFC21466EF0A3FC2618012210
:102F8800314628466EF087FCC20708D431462846E9
:102F98006EF009FD3246214628466EF07BFD002280
:102FA800214628466EF077FC261A0122314628462B
:102FB8006EF071FCC30709D4314628466EF0F3FC65
:102FC8002246314628466EF065FD3446214628469D
:102FD8006EF07EFDBD46BDE8F88300BFA7440A0039
:102FE800586C09007E440A0008B502486FF00DF9D4
:102FF800002008BDD4440A000E4A0346904202D37A
:103008000D4A904211D30D4A22B1934202D30C4A81
:1030180093420AD30B4A52B10B48834234BF012072
:103028000020934238BF00207047012070471046A7
:10303800704700BF00660900B8FF0A0000000000E2
:103048000000000000000000000000002DE9F04F23
:103058009BB000AF04468B46D7F890A0FA637B6319
:1030680049B903784678807800EB830020445E45B0
:1030780022D8A0EB040B0AF0010394F80280FB624B
:10308800E378B8F1000F0CBF4FF000090AF001090E
:103098003B6313B11AF0020F17D1B9F1000F14D125
:1030A800FB6B1BB1594620467A6B98475D4628460C
:1030B8006C37BD46BDE8F08F451C2846FEF798F8EA
:1030C800013028440BF1010BD1E7CAF3C003FB61BF
:1030D8002378BB629B00BB6163683B62BB6A04EBFD
:1030E8008301FB6B002B7DD15D468844B9F1000F4D
:1030F8001DD08B469946A94E1BF8013B54F8230076
:10310800002808BF3046FEF773F8D7F8943001302E
:103118004BB1D7F898304B4582BFD7F8943023F895
:10312800190009F10109C3450544E5D1D8461AF04B
:10313800050F0CBF4FF0020B4FF0010B00260AF0F1
:103148000203FB633B6B9E42B1D298F8013008F151
:10315800020854F823A05046FFF74EFFFA690346C9
:1031680002B3B86318F8021C386A6FF02DF8BB6B0D
:10317800C0B1EA468AB06A46894B05933B6ACDE9F5
:1031880006314FF40073ADF82030864B42F8103FFB
:1031980000234FF41251844801F002F8D546023D4D
:1031A8000136CFE723B1FB6A2BB9A5EB0B05F7E78F
:1031B800FB6B002BF4D07948BAF1000F18BF5046CA
:1031C800FEF716F8D7F8943053B1D7F898309945E8
:1031D8003FBFD7F89420431C22F8193009F10109A0
:1031E8000544DDE7B9F1000F6DD04346102B28BF29
:1031F80010230026BB6397F8389007F14800BA6B94
:10320800796292F021FF796A00227A620AF002025A
:1032180001EB08033A610AF004027B61FA600233A9
:103228007A6A396B8A4267D36378F96A1AF0020FAF
:103238007B624B4418BF0022DBB208BF720800292A
:1032480040F0A9801AF0040F14BF314600216370C2
:10325800A170E27020467A6BB969FB6B9847051E2E
:10326800FFF625AFBB6A314623707B6A7A6B6370C1
:103278003B6B84F80280E37007F15800FB6B9847BA
:10328800061EC0F2C5803A6BBB69386B03EB42037C
:10329800ABEB0301D7E90D23C91A7B6903EB4000A7
:1032A800FB6B98470028C0F2B5804FF000082E4409
:1032B800351807F1480AC84578D300217A6B0846C3
:1032C800FB6B9847F3E6B8F1000F0CD01AF0040F27
:1032D8000ED04346102B28BF1023BB6397F83860E5
:1032E80007F158008BE74646C146C7F838808BE798
:1032F8004E46C7F8388087E713F8015C13F8021CBC
:1033080054F82500BB60FFF777FE0246F869BB68F2
:1033180038B1386AC7E901326EF056FFD7E9013291
:10332800F0B912B3FA6A72B1B9F10F0F18D809F1EE
:10333800280107F1400009F10102014401F8205C6D
:103348005FFA82F90CE0FA6852B10F2E08D806F13C
:10335800280107F14000721C0E1806F8105CD6B25E
:103368007A6A023301327A625AE73A69002ADBD173
:103378000F2EF5D806F1280007F1400C6044721CA6
:1033880000F8101C07F16801023651FA82F2F6B211
:1033980002F8105CE4E7002159E700BF02450A0083
:1033A80009450A0004000001D06B090018F80A302A
:1033B80054F823B087F84730D7F8943033B3D7F8A8
:1033C8009830984522D2D7F8943033F81860012104
:1033D8007A6BFB6B07F14700984700281ADB0E4B06
:1033E8000544BBF1000F08BF9B4626B95846FDF7B8
:1033F800FFFE461CB6B2314658467A6BFB6B9847BF
:10340800002807DB054408F1010854E70026DEE739
:1034180035464CE605464AE602450A00014B186067
:10342800704700BF98030020044608B5EFF31183E6
:10343800202383F31288BFF36F8F2CF047FF2046B9
:1034480002F074FE02486EF0E0FE70F0AFFAFCE79E
:10345800BD450A002DE9F047058B044628071746A5
:103468000CD501290CBF45F0100545F02005258332
:1034780087F31188BFF36F8FBDE8F087022905F045
:10348800070540F0948020466FF0D1F9052864D8EC
:1034980001A353F820F000BF79340000B7350000CD
:1034A80063350000253500003F3500005135000028
:1034B80001F007035A1F012A1FD8002221F0070133
:1034C800062BD4F8008089B2C4E9002209D143460A
:1034D80003E0628B013262831B68002BF9D141F053
:1034E8000201204621836FF0A2F94FF0000900285D
:1034F8006DD041F02001218369E0042B0AD121F02D
:10350800070189B2204621836FF091F910B141F08B
:10351800200121834FF00008C14658E02369D3F801
:103528000090238B23F0070343F006034FF00008B5
:10353800238346464BE02369D3F80490238B23F07A
:10354800070343F00403F1E72369D3F80890238BBA
:1035580023F0070343F00503E8E74FF00008C146EE
:10356800E7E7012243F00803238387F31188BFF3B9
:103578006F8F002A3BD1B8F1000F4AD1B9F1000F83
:1035880002D020462C49C847EFF31187202383F344
:103598001288BFF36F8F238B23F008039BB223831A
:1035A800D9063FD523F01002228303F00705666988
:1035B800218B002EBFF67CAF00239946D4F80080FB
:1035C80021F00701C4E9003341F001012183238B75
:1035D80003F0070AAA4502D0A268002AC1D1B8F1AF
:1035E800000F02D1B9F1000FDAD00022BAE7A168C2
:1035F8000029C0D00D680029BDD033465246204668
:103608004F68B8471DB12B6829461D46F3E72B467E
:10361800FAE74146334652462046D8F800806FF014
:1036280032F9A8E79A067FF523AF23F02002228318
:1036380003F0070527E700BFBB28070037B5044696
:103648000821C06A6FF0D2FB00234FF6FF72104DBD
:10365800ADF804306368ADF800208DF80620E26804
:1036680019182B401344181A60606846ADF8021008
:103678006FF010FB694620466FF0D7FB2046211DEE
:103688006FF0E2FA63682B40A36003B030BD00BF5F
:103698000000FFFF2DE9F7430F4681460821C06A65
:1036A8006FF0A4FB80463C68124D241A3C6004EA83
:1036B8000506B4421CD3A0B210B903B0BDE8F0832C
:1036C80008236A46214648466FF085FA0028F4D157
:1036D8006946A0B26FF076FB38B1BDF80230BDF88C
:1036E80004202E4013441E443C60A4EB0804E0E789
:1036F8000020E2E70000FFFF2DE9F04704468AB00A
:1037080000F11407384676F0AEFFA06A83681B699B
:103718009847E06248B9A849A8486FF04FFB6FF096
:10372800150528460AB0BDE8F087A06A83681B69BA
:1037380098470368013B1F2B01D9A149ECE7E368CF
:10374800B3F5803F08D94FF48032012100929B489D
:103758009C4A6FF009FEE2E7A06A216807AA75F0A3
:1037680002FB08B19849D7E7E5682DB1089BB5FB7E
:10377800F3F203FB12550DB19449CDE7238A012BCF
:1037880001D89349C8E7E36A029593F805804FF09A
:10379800FF334FF0FF3238462EF0EAFE0821E06A88
:1037A8006FF024FBA9460646238A1FFA85FA53457B
:1037B80044D8238A4B4500F00F8153450BD1029919
:1037C800082342462046891B6FF013FA18B9204691
:1037D80002A96FF039FA204602A9FFF75BFF0546F8
:1037E800002840F0FB8002994FEA11494FEA094945
:1037F8006160C4F80890A3688B420DD8082320465E
:1038080003AA6FF0E8F9B8B903AB13F8012B904598
:1038180032D101300828F8D1636820466FF30F03CE
:1038280002A902936FF010FA42462046E368029913
:103838006FF0DFF900283CDA0546CFE0E1682B0499
:10384800891B13FA81F142460823204602916FF042
:10385800D0F978B1204602A96FF0F6F909F101090B
:1038680008234246204602991FFA89F96FF0C1F9E8
:1038780000289ED0013597E7A08803A96FF0A2FA27
:10388800626810B9911B6160B5E7BDF810A0BDF87A
:103898000E10E06AC4F8089051446FF0A7FA484443
:1038A8008242A060EED1BAF1000FEBD06FF01C0598
:1038B80094E05DD04FF6FF79636806EB0308E36890
:1038C8001FFA88F29B1B9A42CDF808801CD34FF050
:1038D80000086168B8F1000F30D06FF30F0120467F
:1038E800029102A96FF0B0F9204602996FF0B9F978
:1038F8000028A1D1E368A288A3EB46039A426DD1C0
:1039080020466FF0AFFA97E708234146204605AAFC
:103918006FF061F900288FD105A91FFA88F06FF0C0
:1039280051FA30B1BDF814304B4502D1BDF818300A
:103938000BB1B044C3E74FF00108CAE720466FF067
:1039480090F900287FF478AF6368224AE168134051
:103958000B44A3EB46036360134041462046A36033
:103968006FF004FBC4E7E26AA36812681344A3601B
:10397800D4E901318B4208D9424620465B1A6FF0E0
:1039880038F90028FFF658AFEDD16168E36801EB1C
:1039980046029A42AED10F4BA06801EA0302904258
:1039A800A8D020466FF05DF900287FF445AF626823
:1039B800084B1A40A2609DE705460A00006C090002
:1039C80027460A0044460A006D460A0085460A0052
:1039D80099460A000000FFFF6FF02C0538462EF0CC
:1039E80039FE002D7FF49DAE0123A37499E600BF34
:1039F8002DE9F04F1E46837C04468946904695B0D3
:103A08004BB96A496A486FF0D9F96FF00C05284636
:103A180015B0BDE8F08FC26A082110466FF0E6F9CC
:103A2800B1B2019010466FF0E1F9E368019A0746D8
:103A3800A3EB82038342C0F0B6801EB1B8F1000F39
:103A480000F0B180D4F804A0CDF810A0204605AA53
:103A580004A96FF041FA05460028D8D1BDF8143002
:103A68004B4507D0DDF810A063685345EED1002E12
:103A780039D1CCE705A91FFA8AF06FF0A3F900281D
:103A8800F0D0BDF8183066B3B3422CD1B3464FEA34
:103A98001A43BDF816A01B049A44E36ACDF80080C7
:103AA8001B685B4203F020030293029B51465B456F
:103AB80028BF5B4620460CAA03936FF08CF80028B9
:103AC8004DD1039B00981A460CA992F0EBFA50B915
:103AD800039B009ABBEB030B1A449A440092E4D16F
:103AE80095E7002B93D0002F3CD1BA4604F1140B74
:103AF8004FF0FF324FF0FF3358462EF039FD238A3E
:103B08009D424DD0D4E901320AEB02018B422ED3FB
:103B18009BB263B3FF230021ADF81E200CA8182226
:103B28008DF82230ADF81C90ADF8206092F0B2FA12
:103B380020460CA9CDE90E866FF062F9074648B910
:103B480007A86FF0A7F8204607A96FF06EF9074697
:103B580000B9374658462EF07DFD3D4657E7C2DC92
:103B6800054654E7019B1F441FFA87FABEE7204623
:103B7800FFF764FD3DB9ADF82490CDF82880ADF885
:103B88002C608DF82E50204609A96FF0EFF90746F2
:103B98000028DFD19DF82E300135002BAFD0D8E7B3
:103BA8006FF01B07D6E76FF0150530E7F1450A00FF
:103BB800006C09002DE9FF471E46837C04460F462A
:103BC8009046BDF8309043B9274828496FF0F6F879
:103BD8006FF00C0004B0BDE8F0870821C06A6FF0F0
:103BE80005F9E368A3EB4003B3423AD34FF0000A68
:103BF80065680195204602AA01A96FF06DF90028B1
:103C0800E8D1BDF80830BB4206D102A9A8B26FF0CE
:103C1800D9F850441FFA80FA019B62689A4219D079
:103C2800CA4515D9BDF80C30C3B1CA4516D3BDF87D
:103C38000A10B3426FF30F0528BF334642462046A9
:103C480029446EF0C8FF0028C4D1BDF80C00C1E7B4
:103C58001D46CFE7BDF80830BB42E3D06FF0010046
:103C6800B8E76FF01500B5E7006C0900F1450A00E8
:103C78002DE9F047044607464FF00109DFF84C806C
:103C880094FAA4F5B5FA85F509FA05F32E0108EBBF
:103C980005156FEA030A24EA03042B7B63B158F87D
:103CA80006301B696BB946447368022228461968B6
:103CB80007EA0A076FF0D5FA002CE1D13846BDE8CB
:103CC800F087284698470028F6D1ECE7106D0900E0
:103CD80010B5002288B00E490E4877F0C4F80022CB
:103CE80000230024CDE906230E234FF44072CDE9CA
:103CF8000334CDE90144084B0849009408482FF0E3
:103D0800B5F80849064876F009FF204608B010BD06
:103D1800313D0000A82A00205140000070D4002046
:103D2800C0250020C3460A0001482EF019BD00BF77
:103D3800901E00202DE9F047804621480F466FF07D
:103D480074FA0646002833D000252846BDE8F087D7
:103D5800237B83B12368DB680BB1204698476368EF
:103D680083F8069023681B69D3B96368022220464A
:103D780019686FF076FA013610345445E8D3B8F173
:103D8800000FE2D0002DDFD02846FFF771FF05466F
:103D9800002FF7D0002140F2391076F0C1FFF1E78B
:103DA800204698470028E0D009FA06F31D43E2E7C9
:103DB80005464FF00109034CDFF80CA0DDE700BF12
:103DC80078540020106D0900206D0900014B53F84C
:103DD800200070473C71090008B5034608462BB11E
:103DE800044A136000F04CFC002008BD6FF0150079
:103DF800FBE700BF9C03002010B5044C237813B9DF
:103E080003482EF0ADFC0123237010BD12CE002014
:103E1800901E002010B5044609486FF006FA3CB120
:103E2800084BD3E8EF1F0139C3E8E21F002AF8D195
:103E380005482FF03DFEBDE8104004482EF090BC28
:103E48007054002074540020A82A0020901E0020DE
:103E58000022044BD3E8EF0FC3E8E12F0029F9D182
:103E6800704700BF7054002070B5FFF7F1FF05469A
:103E7800074C084EB44200D370BD63685B792BB120
:103E880023685B6813B12946204698471034F1E748
:103E9800106D0900206D090010B5044C0449204636
:103EA8006EF0CEFA034B1C6010BD00BF401D002011
:103EB800287109006854002000230D4A10B51370BA
:103EC8000C4A0D4913600D4A0D481360FFF784FF33
:103ED800FFF7E2FF0B4B0C4918468B4200D310BD8D
:103EE8001A1A5C681211013222711033F5E700BF0B
:103EF80013CE00207054002040420F00745400205C
:103F08002F320700106D0900206D0900014647F6A1
:103F18001222002301486EF0B4BA00BF401D0020F1
:103F280001486EF04ABB00BF401D0020024B01460D
:103F380018686EF09DBB00BF6854002001486EF001
:103F4800D2BB00BF401D0020F8B5284B1B78002BC2
:103F58004AD0FFF7E5FF0446002842D1244B254DFF
:103F68001B68002B19DD76F036FF4FF47A76A0FB3C
:103F7800060747F61222002306FB0171FDF7CCF86D
:103F8800D5E90032C01A40F2E93361EB02019842E8
:103F980071F1000101D3FFF767FFD5E9003213F58E
:103FA8007A7342F10002C5E90032ECB1BDE8F8408D
:103FB800FFF7C4BF6B685B7923B12B68214628469D
:103FC8001B6898471035B542F4D32046FFF7AEFF7B
:103FD800094BD3E8EF1F0139C3E8E21F002ABDD01F
:103FE800F7E7064D064EEEE70020F8BD12CE00209A
:103FF80070540020A02A002074540020106D09007D
:10400800206D090070B50D4D297861B90120FFF7C1
:1040180091FE0B4C0B4EB44206D3FFF795FF0028D8
:10402800FBD101232B7070BD63685B791BB12368DA
:1040380020469B6898471034EDE700BF13CE002058
:10404800106D0900206D090000212DE9F84308468C
:10405800FFF770FE044648B340F21B684FF00009B2
:1040680001F0D8FB1A4B1B4A1B58136033B11A4B8B
:104078001B68092B02DD19482EF072FB0025184F2A
:1040880044B12046FFF7F4FD044618B94FF0FF3855
:104098004FF0FF39FFF758FF064628B9B5B90F4862
:1040A80042464B462EF098FB3546E9E74FF0FF387D
:1040B8004FF0FF39D4E72B689B691BB100222846D3
:1040C800114698471035BD42F5D3E8E7054DFAE7A4
:1040D800080000006C54002074540020901E00203A
:1040E800206D0900106D090013B518486FF09DF890
:1040F800174B1B7873B1EFF31184202383F31288D5
:10410800BFF36F8FFFF720FF84F31188BFF36F8F22
:1041180002B010BD0F4B1B68002BF9D050B900221C
:1041280000230D48CDE9002347F6122200232FF083
:1041380099FCEDE70928EBD107482FF0B9FC0748AF
:1041480002B0BDE810402EF00BBB00BF7454002035
:1041580013CE00206C540020A82A0020901E0020B6
:1041680010B5064B04461B6898472146A0600448D2
:104178006EF004FABDE81040FFF7B6BF9C030020BC
:10418800401D0020044A054B9B1AB1EBD30F34BFE6
:1041980052F8310000207047106B0900106D0900BB
:1041A8002DE9F04F8FB0C1F34A2604AF0D46904673
:1041B800B8607B600C0D002E61D04FF000090A2317
:1041C8004FF0040B07F1140AFE60C7E90799C7F816
:1041D80024900093CDF808B0CDF804A007F11C0393
:1041E8004A464046F968FEF731FFB0F5006F0346CE
:1041F8001CD36C468AB0D8F8041004AB24481A467D
:10420800C3E9050140F2FF71D9614FF400711984C7
:10421800204B42F8103F4FF412514B461E48FFF70F
:10422800BFFFA5462C37BD46BDE8F08FC0F30A0690
:1042380004F11700184420F0070080083B60FFF7DE
:1042480065FE66F35325044680B13B6800F1100112
:10425800C7E908390A23F961CDE901AB0093404663
:104268000E4AF96807F11C03FEF7F0FE66F35325C2
:104278002A4620467B68B9686FF013F8D2E704F144
:10428800170020F007008008FFF740FE0446EDE71E
:10429800D4460A0004000001206C09007D320700A2
:1042A8002DE9F04F87B00546DDE9106BDDE9127A9C
:1042B800884614469946BFB110213B465A4600200D
:1042C800CDF800A0CDF814A06DF0A5FDB0F5006FF5
:1042D80001460BD340F2FF730221184A184807B071
:1042E800BDE8F04F6FF036B83946384604F007039A
:1042F80005F00704E40044EA831444EA402444EA4D
:10430800065406F11700084420F0070080080391BE
:10431800FFF7FCFD054640B13FB13B465A460399BD
:10432800CDF800A010306DF076FD4B462246414690
:10433800284607B0BDE8F04F6EF0B3BF13470A0038
:10434800206C0900406820B1034BC01A40F3CF002D
:1043580070474FF0FF307047106B09000EB403B57B
:1043680003AB53F8042B01460448019301F086FC83
:1043780002B05DF804EB03B0704700BFBF3307001D
:10438800CA0605D48B064CBF02490349FFF7E6BFAE
:10439800704700BFE2920A0002890A002DE9F04F37
:1043A8008BB099469DF85880179B044607930D4695
:1043B800DDE918A31A9F06920593B8F1000F00F0E3
:1043C800BC80834B07F0020B13F80830089307F4FE
:1043D800807309936EF043FF024600287AD0204686
:1043E8007C49FFF7BBFF0646BBF1000F08D017F06A
:1043F800440F71D12A4620467749FFF7AFFF06449C
:1044080007F0010353B1754B204653F82820744B2D
:104418007449002A08BF1A46FFF7A0FF07F4807303
:10442800002B07F0080318BF4FF00009002B7FD0BE
:104438006D4B204653F828206C49FFF78FFF05463F
:10444800069B2BB11A4620466949FFF787FF0544AA
:10445800B9F1000F0DD0089B002B6CD06549664B55
:10446800B8F1040F18BF19464A462046FFF776FFF1
:10447800054462483544079B1BB1224660496DF0EC
:1044880072FE059B002B00F08E80059B3946102B91
:1044980028BF1023204699460026FFF771FFB54232
:1044A80052DC0026334620461AF803205549FFF708
:1044B80055FF0136102E4DD0710703D120465249C1
:1044C800FFF74CFF4E453346EDD320464F49FFF7E3
:1044D80045FFEEE7064687E74D4B186800288ED063
:1044E8004C4B4FF47A7B1B684FF03C0CB5FBF3F553
:1044F800B5FBF0F14FF4616300FB11550BFB05F5BB
:10450800B1FBF3F2B5FBF0FE03FB121100FB1E55E5
:10451800B1FBFCF30BFB05F5B5FBF0F50CFB131138
:1045280020460091CDE901E53B49FFF717FF66E713
:1045380007F0080584E7304996E7B9F1010F4546C9
:104548000CBF2E48354896E720462F49FFF706FF4F
:104558000136A4E7002620463149FFF7FFFE33461F
:104568001AF803202046A2F120035F2B28BF2E2231
:104578002C49FFF7F3FE0136102E0DD0720703D138
:1045880020462149FFF7EAFEB1453346E8D82046E0
:104598001D49FFF7E3FEEEE7059BCA44B3EB0903A9
:1045A80005937FF472AFB8F1000F0AD0FB0704D56A
:1045B80020460B4A0B49FFF7D1FE39462046FFF744
:1045C800DFFE20460BB0BDE8F04F6EF0E7BE00BF3F
:1045D8005CC90A0059470A005D470A004C71090086
:1045E8004B470A0098910A006071090083470A0046
:1045F80089470A0050470A0054470A00BF3307009A
:10460800855C00008D470A0078C80A0076C80A0051
:10461800805400207C54002067470A00ED330700CF
:1046280093470A00DB900A0042F20F7373B58B427E
:1046380028BF0B4605680446052168460D4A69F0FF
:1046480005FA0646636828460B225B680A496EF03D
:1046580097FE63683246694628465B686EF090FEAE
:1046680063681B2228465B6804496EF089FE02B025
:1046780070BD00BF15930A0050C90A0034C90A006A
:1046880000210123064A904206D8064A01B90123AF
:104698001360054B18607047012140085B00F2E782
:1046A80040420F007C54002080540020F8B50D468D
:1046B8000446064F4618B44201D12846F8BD14F8FE
:1046C800011BBB6801485B689847F4E7D06709009D
:1046D800014B036000207047A871090070B5104BAA
:1046E8000D461C68B4B10F4B196800238B4202DBDE
:1046F8006FF0010070BD224612F8146B864202D09A
:1047080014460133F2E7E06875F06EFE28B1002028
:104718002C60EFE76FF00C00ECE76FF01200E9E7B0
:10472800A8030020A871090010B5436888B0029357
:1047380083680C46CDE9033200230A68C068CDE9D6
:104748000623054901AA059374F011FB079808B9D7
:10475800059B236008B010BD7F35070010B54FF4E6
:104768002814DFF820C086B0CDE904C408240294D8
:1047780004AC0194BDF82040009472F0F1FB06B03F
:1047880010BD00BF180028002DE9F8430646FCF7C5
:104798002FFD0546EFF31188202383F31288BFF31A
:1047A8006F8F114B1C68D3F804909C4208BF0024FB
:1047B80034B988F31188BFF36F8F2046BDE8F883BA
:1047C800A7683846FCF714FDA84206D12A463946A0
:1047D800304691F084FC0028EBD04C4501D0246889
:1047E800E6E70024E5E700BFC40300202DE9F04117
:1047F8000E461546FFF7C8FF044628B3C3681BB327
:104808005F690FB3062E07D0072E20D02A463146FF
:104818003B46BDE8F0411847838A3BB92A463146F2
:10482800B84750B9A38A0133A38206E04FF6FF7256
:10483800934204D00133A3820020BDE8F081012116
:10484800114A12486EF07DFD6FF01500F5E745B18D
:104858002A7832B10022828231462A465B6998471B
:10486800EAE7A38A012B08D12A4607212046B84740
:104878000028E2D1A38A013BD6E70BB1013BDAE776
:104888000221034ADDE700BFE9470A00E86B090097
:104898000B480A0010B5044608B1806838B9104AB8
:1048A800104801216EF04DFD6FF0150010BDFFF7A7
:1048B8006BFF08B10C4AF3E7A082EFF311812023C4
:1048C80083F31288BFF36F8F084B5A68C4E900322C
:1048D80014605C6081F31188BFF36F8FE6E700BF57
:1048E80029480A00E86B090042480A00C40300206E
:1048F8002DE9F0410C4B05461C680E4617467CB165
:1049080000F06AF963682046D3F8108032463B46C7
:104918002946C047044600F069F92046BDE8F08101
:104928006FF00104F9E700BFB054002000230360D2
:10493800044B5A6812B9C3E9000070471060586008
:10494800704700BFB4540020014B1860704700BF87
:10495800B0540020002330B585B0CDE902330546B8
:10496800019000F039F9094B1C6844B9284600F059
:10497800D5F8044600F03AF9204605B030BD636822
:1049880020461B6801A998472468EEE7B454002024
:104998001FB5CDE90101039200F01EF9074B1C6811
:1049A80024B900F023F9204604B010BD63682046FE
:1049B8001B6801A998472468F2E700BFB454002097
:1049C8000022024BC3E90022704700BFB454002004
:1049D8000022024BC3E90022FFF7F2BFBC540020BB
:1049E8002DE9F74307460C4609B100230B60002662
:1049F8001E4DDFF880904D450FD31D4B1D6885B3C4
:104A080055F8188C3846414601AA183D6EF099FEB3
:104A180010B3D6B914BB2E461EE0D5F80080384630
:104A2800414601AA6EF08DFE50B116B954B92E4612
:104A380006E00022404631686EF083FE0028F5D17A
:104A48001835D8E7019B2360F1E70022404631681A
:104A58006EF077FE0028DDD1AD69D0E7019B2360B9
:104A6800D9E7304603B0BDE8F08300BF206D0900E8
:104A7800BC540020B06D09002DE9F04784B002AFA6
:104A8800D7F8289004460D46164698467860B9F13E
:104A9800000F07D0D9F8001031BBD9F804A0BAF13B
:104AA800000F28D12046391DFFF79AFF08B3D0F828
:104AB8000C904346324629467868C847C8B16D46C7
:104AC8008AB002AA124BD061C2E905344FF40073D0
:104AD8001384104B42F8103F00234FF411510E4835
:104AE800FFF75EFBAD4604E03A1D6EF02AFE002893
:104AF800D3D1002007E0D9F8083032460093294680
:104B080043467868D0470837BD46BDE8F08700BF00
:104B18006B480A0004000001606C09002DE9F047A9
:104B280080464FF000470026DFF8A490DFF8A4A0E5
:104B38003D46264C4C450DD3DAF80040002C40D0B9
:104B4800183CB8F1000F24D1226952BBA469F5E7DB
:104B58002F46EDE7B8F1000F03D122694AB918349E
:104B6800E8E70022414620686EF0EBFD0028F4D10A
:104B7800F5E76368BB4206DDAF4202D0AB42A8BF8F
:104B88002B461D46EBE7EAD19047002E08BF0646A4
:104B9800E5E70022414620686EF0D3FD0028D3D116
:104BA800D4E76368BB4206DDAF4202D0AB42A8BF80
:104BB8002B461D46CAE7C9D19047002E08BF0646B6
:104BC800C4E7AF42C4D13046BDE8F087206D090084
:104BD800B06D0900BC5400204FF0FF324FF0FF3396
:104BE80001482DF0C5BC00BF1C1E002001482DF057
:104BF80031BD00BF1C1E002038B5094DFFF7ECFF82
:104C08002B785BB9FFF7E4FE00F06AF8044608B9B0
:104C180001232B70FFF7EAFF204638BD0024F9E78F
:104C280015CE00202DE9F04306460F46048F99B0B3
:104C38000134A4B200F10808651EADB2B5F5004F05
:104C48004AD04A23294605AA40466EF0D3FA04F50D
:104C58007F543F34A4B281462146012340460DF1DA
:104C68000B026EF0C7FAB9F1000F014610DC0028FC
:104C780010DC338FAB4209D132466B1E22F8383F25
:104C88004FF4004102234046FEF7B2FE2C46D3E71C
:104C9800002808DC294640466EF0A8FA214640461E
:104CA8006EF0A4FAE5E7B9F1490FEFD809F160030E
:104CB8000DEB03090023094A09F84C3C05A80097A5
:104CC80003ABCDF80C80ADF81040FFF7D5FE0028F7
:104CD800DCD019B0BDE8F0830020FAE7BB37070045
:104CE8007FB50123694604200193FFF7F7FC0446CA
:104CF80068BB042002AA01A96EF05FFC044610B14B
:104D080010F10C0F23D10399B1F5803F24D2002371
:104D18001846009A9468084484421BD30133B3F5BB
:104D2800807FF8D10E4D69612B8353682846AB60AC
:104D3800D368EB636EF0D5FD044640B9094E2846AA
:104D48006E60FFF7F3FD28466E60FFF7FDFD204615
:104D580004B070BD9BB2E5E76FF02004F7E700BF31
:104D6800C45400209C7209002DE9F04F8BB0914685
:104D7800D0F808A01E4600AFDAF8103080460D467D
:104D88009847B9F1000F05DA2B4A01212B486EF03C
:104D9800D8FA0AE0036846EA09045A1E14400BD000
:104DA8000121274A25486EF0D5FA6FF015052846E7
:104DB8002C37BD46BDE8F08FDAF80CB0BBF1000F18
:104DC80006D0294633464A464046D8470546EEE7C8
:104DD800202B01D91B4AD8E72946202207F10800D1
:104DE80091F058F92546A642E1D9331B202B28BF5C
:104DF800202309EB040BDAF804505946404607F122
:104E080008027B60A847051E7B6812DA6C4688B0EA
:104E18006A460D4BCDF81CB0CDE90538042342F89D
:104E2800103F00234FF401510448FFF7B9F9A54694
:104E3800BDE71C44D7E700BF90480A00F06B0900A3
:104E4800AD480A00DF480A0005490A0080B5054652
:104E58000E46174698462EF029FB034600F0DAFC6A
:104E68000446DFF81890424649F800303946304683
:104E7800A84754F8090000F045FC00BF08000000EE
:104E880008B50348034A0021121A6EF066FD08BDF2
:104E98008022002070D40020074808B5074A084936
:104EA800121A6EF05CFDBDE808400648064A07493C
:104EB800121A6EF054BD00BF0000002048220020E6
:104EC800B8FF0A000000002000000020B8FF0A0018
:104ED8002DE9F84F80460C4600AF00296AD0D1E989
:104EE8000012E9468AB0A3686D464FF0050A6E467F
:104EF8003948CDE90723CDE9050146F810AF00236D
:104F080032464FF421513548FFF74AF9D4E90312E4
:104F1800CD466369AD463248C5E90723C5E90501B1
:104F2800C5F810A0002332464FF421512B48FFF753
:104F380037F9CD46E36901212A4A28486EF00AFA72
:104F48000121294A25486EF0FCF9264600254FF034
:104F58000A0ADFF8A4B0E946D6E908C0D6E90A1378
:104F68008EB06A46CDF81CC005F1010CCDE908C029
:104F7800A81CCDE90A01E91CCDE905B5CDE90C135A
:104F880042F810AF002345F2400114480435FFF7FA
:104F980007F9102DCD4606F11006DCD1236E01214C
:104FA800124A0E486EF0D6F9A3690121104A0B483F
:104FB8006EF0D0F9B8F1010F07D1EFF305830D4A70
:104FC80041460648103B6EF0C5F9214640462CF094
:104FD800FFFFBD46BDE8F88F2C490A00506C090058
:104FE8005B490A008A490A0099490A00164A0A00D8
:104FF800254A0A00534A0A00D3490A0030BFFFF77E
:10500800FDBF00BF2DE9F04105460B4EDFF83080AB
:10501800324606EB0807CC1B2046084991F014F8E5
:10502800A01942460021083C91F034F8C5F8904098
:1050380007F10800BDE8F08100000000B06D09002C
:105048000800000010B5244C244925486EF094FC53
:10505800A36A99013ED5224822496EF08DFC1E2094
:10506800A36ADA0104D51E481F496EF085FC1F208B
:10507800194CA36ADB0204D519481C496EF07CFC64
:105088000220A36A1C0304D5154819496EF074FC64
:105098002120114CA36A590304D5114815496EF013
:1050A8006BFC2220A36A9A0304D50D4812496EF0BE
:1050B80063FC2320084CA36ADB0304D508480F4986
:1050C8006EF05AFC2420A36A6FEA03436FEA134385
:1050D800A36210BD1D20C3E700ED00E0664A0A0088
:1050E800506C09007E4A0A00914A0A00AB4A0A003D
:1050F800D54A0A00F34A0A00184B0A00324B0A0044
:1051080070B506460D46294C29492A486EF034FCEC
:10511800A36ADB0647D5274827496EF02DFC1120E6
:10512800A36A1C0704D5234824496EF025FC1220E5
:105138001E4CA36A990712D521491E486EF01CFC23
:10514800636BA26A120609D501211E4A19486EF03E
:1051580001F91EB1A36A23F08003A3621320134C44
:10516800A36ADE0704D5134817496EF005FC14201E
:10517800A36A9C0604D50F4814496EF0FDFB152060
:105188000A4B9A6AD10658BF9A6A9A6A920642BF2F
:105198005A6A22F400525A629A6A42F0FF029A62EC
:1051A80000232B7070BD1020BAE700BF00ED00E0AF
:1051B8005D4B0A00506C0900734B0A00A64B0A00AD
:1051C800B94B0A00D14B0A00E74B0A00064C0A000B
:1051D80070B506460D46284C284929486EF0CCFB88
:1051E800A36AD9043CD5264826496EF0C5FB17208A
:1051F800A36A1A0504D5224823496EF0BDFB18207E
:105208001D4CA36A9B0512D51D4820496EF0B4FBBE
:10521800A36BA26A100409D501211D4A18486EF033
:1052280099F81EB1A36A23F40043A3621920124C13
:10523800A36A590504D5124816496EF09DFB1A2039
:10524800A36ADA050ED50E4813496EF095FB1B20AC
:10525800094A936A43F47F43936200232B7070BD1D
:105268001620C5E7A36A9B04F2D505480B496EF0E2
:1052780083FB1C20ECE700BF00ED00E0354C0A0082
:10528800506C09004B4C0A00A64B0A005C4C0A0003
:10529800754C0A008A4C0A00A54C0A00064C0A0004
:1052A800F0B59DB0664B05465868002600AFC0F3C0
:1052B800080386F31188BFF36F8F02F07F44B4F1BF
:1052C8007F4F07D102F00C04082C0ED15D495E48CF
:1052D8006EF052FB5D495C486EF04EFB00210846BB
:1052E800FFF7F6FD7437BD46F0BD14074CBF0D46F9
:1052F8000126002DEED00022FA71DA1E092A7ED886
:10530800DFE802F0057578717D7D7D7D7D7B5049F4
:105318004D486EF031FB0023494CFB71E36A9A0754
:1053280005D54C4948486EF027FB00242DE0E36A78
:10533800002B01DA4849F5E7E36A5B00F5D54749F0
:1053480041486EF019FB6369AA6943F4807363618D
:10535800BFF34F8FBFF36F8F32F8023C626922F4BC
:1053680080726261BFF34F8FBFF36F8F03F47F4288
:10537800B2F55F4F21D1DBB2022B1ED12B68012180
:10538800374A31486DF0E6FF2C68FB79002BA9D12C
:105398006822294607F1080090F056FE7B6A002E25
:1053A8004AD0C3F3080222B96FEA53236FEA4323B2
:1053B8007B62204607F1080192E7214B9A6AD2B234
:1053C80022B10120F91DFFF79BFE0EE09A6A12F444
:1053D8007F4F04D00120F91DFFF7FAFE05E09B6A14
:1053E800B3F5803FA1D3FFF72DFE0446CDE700209B
:1053F800F91DE8E70020F91DEEE71A4992E71A4A75
:105408006C4610F4F87F8AB0184918BF11466A46EE
:10541800103B07934FF400731548ADF82030154B37
:10542800CDE9050142F8103F00234FF41151064819
:10543800FEF7B6FEA54678E76FF30803B8E700BFA6
:1054480000ED00E0EB4C0A00506C0900164D0A0014
:10545800524D0A00694D0A008A4D0A00984D0A000B
:10546800B74D0A00D34D0A00D24C0A00BD4C0A00C1
:10547800F74D0A0004000001064B5A6942F0100279
:105488005A615A6942F480625A615A6922F00802E4
:105498005A61704700ED00E0EFF30880EFF30981EF
:1054A80001B57246FFF7FCFE01BD00BF0B4880F353
:1054B80008882AF091FF202080F3118808484FF4CB
:1054C8000061401880F30988EFF314800221084333
:1054D80080F31488BFF36F8F00F068F880720120A2
:1054E800600A01201EF0040F0CBFEFF30880EFF3F1
:1054F8000980816911F8021C0229FFD001B57246A2
:105508006EF02FFA01BD00BF0028ACBF00F160406B
:10551800064B4FEA4111C9B2ABBF00F5614000F03C
:105528000F0080F800131954704700BF14ED00E015
:1055380000B2002807DB01234109034A00F01F00DD
:10554800834042F82130704700E100E000B20028B3
:105558000CDB01220649430900F01F00824020337A
:1055680041F82320BFF34F8FBFF36F8F704700BF01
:1055780000E100E0054B420953F82220012300F026
:105588001F0003FA00F01040704700BF00E100E080
:10559800044B054A23F07F039360BFF34F8FBFF39B
:1055A8006F8F70470000000000ED00E008B5FFF7BE
:1055B800EFFF104BD3F8882022F47002C3F888203C
:1055C800D3F8882042F4A002C3F888204FF0404264
:1055D800C3F83422BFF34F8FBFF36F8F0023E1EE80
:1055E800103AFFF74DFCFFF757FC00F0F3F82CF0EA
:1055F8001BFE00BF00ED00E08189203A41F0020166
:1056080081814FF47D41C0F8DC101360009B08498C
:105618005360019B21F001019360029B9161D3606B
:105628004FF08073D36100230265C0F8943070474F
:10563800554E0000104B9B6883421AD1EFF305804A
:10564800B8B9EFF31181202282F31288BFF36F8F6C
:105658009A8922F002029A81EFF3148323F004035B
:1056680083F31488BFF36F8F81F31188BFF36F8FB3
:1056780070476FF01500704724A500200E461546A8
:10568800002300B5E1EE103AEFF3148323F004038E
:1056980083F31488BFF36F8FBFF36F8F0C4BD0F871
:1056A800902098600B4B1A60D0F8803083F30B88F9
:1056B8002C4686F309880020034B98472046002192
:1056C80000220023014C2047A7390700554E00004F
:1056D80024A50020045500201022014B1A617047B0
:1056E80000ED00E0054B9A699B689A421FBF044A87
:1056F800536843F080535360704700BF24A50020CF
:1057080000ED00E0084B9B6883420BD1EFF3058363
:1057180043B1064B5A6842F080525A605A6A22F4E2
:1057280000425A6275F0FFB924A5002000ED00E0A0
:1057380025498A6882F8DDE04FF030001044EFF325
:10574800098C80E8F01F1EF0100F03D102F19C00B5
:1057580080EC108A202080F31288BFF36F8F1B4FD4
:105768004FF000668A698A603E60D2F89000184C53
:10577800206092F9DDE0D2F894000023C2F894305A
:1057880080F311881EF0100F03D00023E1EE103AC9
:1057980003E002F19C0090EC108AEFF3148323F0ED
:1057A800040383F31488BFF36F8F02F1300090E88D
:1057B800F01F8CF3098802F1000004B56EF0E8F8D8
:1057C800BDE804407047000024A5002004ED00E077
:1057D80004550020002320210448C2180133B3F5E2
:1057E800917F82F80013F8D1704700BF00E100E014
:1057F80008B5EFF30583064A103B02EBC30152F8E4
:10580800330049688847BDE80840FFF76BBF00BF11
:105818000C1400200148006870470000045500205F
:105828001FB50121094B0A4A0A4800F00FF9002365
:10583800064A0393084B0121019301A8D31A029346
:1058480000F00EF905B05DF804FB00BF00FC07206E
:1058580000000020B8720900802200200A7A0B6834
:1058680010B562F304031C46CB68520923F01F03EA
:1058780043EA4203044A43F00103C2F89800C2F81D
:105888009C40C2F8A03010BD00ED00E010B50A4BF6
:10589800D3F89030C3F30723013B984208D901217C
:1058A8000346064A06486DF055FD6FF0150010BD19
:1058B800FFF7D4FFFBE700BF00ED00E00E4E0A0043
:1058C800386C09002DE9F04F8946144606464FF01A
:1058D80000084F4D85B0C84527DAD6F804A0BAF1BC
:1058E800000F44D0BAF11F0F17D91AF01F0F14D1A7
:1058F800D6F800B01BF01F0F0FD158466EF072F8A3
:1059080007460AEB0B0001386EF06CF8874210D09E
:105918006FF015073F4A3B4601E043463E4A0121E6
:105928003E486DF017FD6FF01504204605B0BDE840
:10593800F08F17F1160FEDD0BC42EBDDC5F898706B
:10594800D5F89C10C5F89870D5F8A03021F01F0143
:1059580043F01F0BD6E900321A44994202F1FF3A8C
:105968001AD1D34507D13146F8B26EF044F808F1A0
:1059780001080C36AFE73146C5F89870D5F89C3069
:10598800E0B263F30402C5F89C206EF034F810F11D
:10599800160FC8D0441CEAE7C5F89870D5F8A020BF
:1059A800013B23F01F0302F01F021343D345314686
:1059B800E0B2C5F8A030E8D06EF01DF810F1160F6F
:1059C800B1D0C5F89870D5F89C209DF808300BF137
:1059D800FF3B62F304038DF80830D5F8A0309DF83A
:1059E80008205B0863F347128DF80820D6E90032D7
:1059F8001344009323F01F035B44A3EB0A03013015
:105A080023F01F036946C0B20393FFF73FFFBEE7C9
:105A180000ED00E05A4E0A00344E0A00386C0900C6
:105A28000522044BC3F89420BFF34F8FBFF36F8F49
:105A3800704700BF00ED00E0BFF35F8F0022024B0C
:105A4800C3F89420704700BF00ED00E010B5034C88
:105A58002278FFF737FF207010BD00BF16CE002058
:105A68002DE9F74F294D8A4606464FF00008AB4608
:105A7800274FD0451BDAD6F80490B9F1000F3FD074
:105A88003168084601916DF0ADFF0199044609EBB4
:105A9800010001386DF0A6FF84424FF014021D4B3F
:105AA80008D002FB08F36FF015024BF8032003B08F
:105AB800BDE8F08F14F1160F2C60F8D01978A142C8
:105AC800F5DD02FB08B0C7F89840C7F89840D7F84A
:105AD8009C4000F10801007B64F304000871D7F8CA
:105AE800A0000C79400860F347140C71D7F89C109B
:105AF80021F01F016960D7F8A01021F01F0129616A
:105B080008F1010814350C36B3E700BF085500202A
:105B180000ED00E016CE0020F0B55349534DD1F802
:105B280090302C68C3F307239C4287B000F2998019
:105B38000020FFF781FF4E4BC1F8C030844216D1D8
:105B48004C4D01A82C70FEF7C3FD002607464A4CB1
:105B5800B74213D100202B784349D1F89020C2F3E3
:105B68000722934277DBFFF75BFF002046E0696876
:105B780001EB0011FFF772FE0130DFE701993001F8
:105B880001EB0613DA682240B2F1807F52D00AD8BE
:105B9800B2F5001F34D0B2F5800F3ED0B2F5801FA9
:105BA80012D00136D4E7B2F1006F43D0B2F1805F72
:105BB800F7D15A689B680958013B22F01F0003443B
:105BC80023F01F03012032E05A689B680958013B03
:105BD80022F01F0003440120844623F01F0340EAFB
:105BE8004C10CDE902218DF8100002A92878059300
:105BF800FFF74CFE00282ADA6FF0150007B0F0BD59
:105C08005A689B680958013B22F01F0003444FF073
:105C1800020C012023F01F03E1E75A689B6809582A
:105C2800013B22F01F000344022023F01F034FF022
:105C3800000CD4E75A689B680958013B22F01F0002
:105C480003444FF0030C012023F01F03C7E72B7810
:105C580001332B70A5E7C1F89830C1F8A0000133D3
:105C68007BE74FF0FF30C9E700ED00E0C4720900A0
:105C7800AAFF440016CE00200000F0FFF0B587B060
:105C880007460E4614460021102268461D4690F02D
:105C980001FA02238DF80230054B2A462146684650
:105CA800CDE90476019368F063F807B0F0BD00BF52
:105CB800373A070008B5024B1B689847002008BD13
:105CC8001C550020034B044A1860937843F00203E4
:105CD800937070471C550020CC03002008B5054878
:105CE8006CF093FA002383F31188BFF36F8F0423BA
:105CF800184602DF8C4E0A0008B50549054A21F00E
:105D080007010548521A6CF034F8002008BD00BF9E
:105D180053BD012000FC0720205500204FF0FF3222
:105D28004FF0FF3301482CF023BC00BFDC030020F8
:105D380001482CF08FBC00BFDC03002038B50546B5
:105D4800FFF7ECFF2A46082107486BF058FF044686
:105D580028B925B1FFF75EFD0C22044B1A50FFF756
:105D6800E7FF204638BD00BF205500200C0000008A
:105D780038B504460D46FFF7D1FF21462B460822C9
:105D880007486BF0BEFF044628B925B1FFF742FD6E
:105D98000C22044B1A50FFF7CBFF204638BD00BF3A
:105DA800205500200C00000010B50446FFF7B6FF90
:105DB80021460348FDF78AF8BDE81040FFF7B8BF51
:105DC8002055002070B5A0FB015434B92846FFF7D0
:105DD800B5FF064640B9304670BDFFF71BFD0C22E3
:105DE800044B00261A50F6E72A46214690F052F94D
:105DF800F1E700BF0C00000070B541690446867ADF
:105E08000A4D59B1437ADB0706D42C2303FB06530A
:105E18005B6A1B689B689847002363612C202146B6
:105E280000FB0650BDE8704074F0EDBCFC1E00207D
:105E38002C22024B02FB0030704700BFFC1E0020E2
:105E48002C21827A054B01FB02339A6A1B7F801A48
:105E58001B3323F00303B0FBF3F07047FC1E002054
:105E680038B52C24827A064B04FB02335B6AD3E9EB
:105E780001240C601568FFF7E3FF04FB005038BDF0
:105E8800FC1E00202DE9F04385B005466846904683
:105E98001C46039174F0A1FFDDE90067EFF3118957
:105EA800202383F31288BFF36F8F6B8B002B41D0B5
:105EB8002A8B9A4225D90022002328462CF01AFC66
:105EC8000446F0B189F31188BFF36F8F039B002B51
:105ED80041D032463B46684674F0A4FF2C21A27A92
:105EE800254B204601FB02335B6A03A91B681D682A
:105EF800DDE90023A847606170BB2046FFF77CFFFF
:105F080024E0698B4B1E6B8389F31188BFF36F8F75
:105F18002B7F2A8BAC6A1B3323F00303521A02FB34
:105F28000344154B154AEB1A9B105343A3722B7F5E
:105F3800E372CBE789F31188BFF36F8F234642469C
:105F480028462CF0D7FB04460028BFD10024204661
:105F580005B0BDE8F0836361012300252381039B1D
:105F680029466382E27A656004F1180090F092F89D
:105F780063692582E360EAE7FC1E0020A38B2EBA42
:105F8800F8B500242C260F4D00B9F8BD476800F17C
:105F98000802D2E8EF3F591EC2E8EC1FBCF1000F1F
:105FA800F7D1DBB2012BF0D1837AC46006FB03532F
:105FB80044601B6A13B198473846E5E7FFF71CFFB2
:105FC800FAE700BFFC1E00202DE9F84F06460D46F3
:105FD80017460446A3466468002CFBD14FF02C09F1
:105FE800DFF878A0BBF81030BBF81220DBF81410EB
:105FF800D21ADBF80C300BF10C005B1AD21AAA4249
:1060080028BF2A461FFA82F8394642466DF0C0FD7D
:10601800B5EB0805444447441DD00C9B53B1DDE95A
:106028000A010D9A98478346A8B1014630466DF09B
:1060380071FDD7E7B07A09FB00A0436A9B6843B1BA
:10604800AB4228BF2B461946DDE90A23FFF71AFFA2
:10605800E9E72946F8E72046BDE8F88FFC1E00204E
:1060680008B5244A244B1A6028F0A2FC4FF47A6140
:106078002248D0F82436C3F30802C3F309434B433C
:1060880082F480721E49883201FB02334FF4FA21F0
:106098005B00B3FBF1F201FB12331A49B3F57A3F07
:1060A80028BF0132C1F80429D0F820364FF47A60AD
:1060B800C3F30802C3F30943434342F21C5082F47A
:1060C800807202F2172200FB02334FF47A701B0A27
:1060D800B3FBF0F200FB12330020B3F5FA7F4FF068
:1060E800010328BF0132C1F81C27C1F80009C1F813
:1060F800003608BD0020A107340E002000C0FF00B4
:10610800F82A00800000125048B1054B054A1B6868
:10611800B3FBF2F35843044B43F0010318477047AD
:10612800340E002040420F00706E0900BFF34F8FFD
:106138000549064BCA6802F4E0621343CB60BFF31B
:106148004F8F00BFFDE700BF00ED00E00400FA0537
:10615800F7B506460D461446124F384674F044F912
:10616800E0B1BB68314638461B68AAB29847002898
:1061780002DB002003B0F0BD002CFBD1AC42F8D20A
:106188002F1B042F28BF042773F0BBFC3A4601904D
:1061980001A930198FF058FF3C44EFE76FF0120067
:1061A800E8E700BFB467090038B504462DF05AF98E
:1061B80020466DF057FDA069C8B194F86C30DB0734
:1061C8000DD50221154A16486DF04AFD6FF0770586
:1061D800201D6DF04EFD2DF059F9284638BD74F09C
:1061E80003F938B901210F4A0D486DF039FD6FF0F8
:1061F8001205EDE7204600F0B5FF05460028E7D177
:106208000146242204F128008FF044FF94F86C30F2
:1062180043F0010384F86C30DAE700BFA84E0A00A7
:10622800D06C0900D24E0A0070B504462DF01AF958
:1062380020466DF017FD94F86C30DA070DD4022172
:10624800254A26486DF00CFD4FF0FF35201D6DF0F6
:1062580010FD2DF01BF9284670BDC3F340019B07C4
:1062680007D502211E4A1D486DF0FAFC6FF077052C
:10627800ECE7A06971F07EFF0646A06972F00AF8A3
:10628800054628B10121174A14486DF0E9FCDDE7FD
:10629800A36F4BB1314620466DF0C5FE0546A0B14F
:1062A800A06972F01FF8D1E7A06971F09BFFA067A1
:1062B8000028EFD101210C4A08486DF0D1FCA069F3
:1062C80072F010F86FF00B05C0E794F86C3043F0EB
:1062D800020384F86C30B9E7F54E0A00D06C090067
:1062E8001B4F0A00414F0A005D4F0A0038B590F86D
:1062F8006C3004469B0708D40221144A14486DF0F8
:10630800AFFC6FF07705284638BD6DF0ABFC002177
:10631800204601F0C1F820B101210E4A0C486DF069
:106328009FFCA06971F0DEFF054620B101210A4AF1
:1063380007486DF095FC94F86C30201D23F002039B
:1063480084F86C306DF095FCDDE700BF794F0A00EA
:10635800D06C0900A04F0A00BE4F0A002DE9F04397
:1063680085B006460C4690466DF085FC0546B8F1AA
:10637800000F07D030466DF083FC012810D1B5FA24
:1063880085F56D09013429463046E2B26DF064FEA8
:10639800814650B901212346324A33486CF0DAFF6E
:1063A8000024204605B0BDE8F0834768B8F1000F27
:1063B80009D03868796801AB03C33A7A01AF1A701B
:1063C80007238DF80530F18D7B883046994228BF28
:1063D80019466DF093FF04460028E1D0038A428AEB
:1063E8004169D21AC36800F10C085B1AD21A3B78CB
:1063F80039469A4228BF1A4640466DF0C9FBD9F87B
:106408000C90B9F1000F08D1218AF38D9942C8D9AF
:106418004046C91A6DF0E3FBC3E7D9F80400836866
:106428001B6B13B9D9F80090EBE729469847002869
:10643800F8D0071F57F8041F0029F3D00878002860
:10644800F0D0628A238AA2EB030C6269E3689B1A84
:10645800ACEB0302904294BF024692B240466DF004
:1064680097FBE7E7EE4F0A00B06C090038B5044621
:10647800806F6DF037FB05466DF0EDFA2046294632
:1064880001F052FA044638B104480121044A6CF07C
:1064980058FF2846FFF774FD204638BDB06C090048
:1064A80014500A0038B580210446806971F0BDFE99
:1064B800054678B10146204601F036FA044638B15F
:1064C80006480121064A6CF03CFF2846FFF758FDB4
:1064D800204638BD6FF00B04FAE700BFB06C090026
:1064E80033500A0000232DE9F04F93B005930B7E3B
:1064F800044633F080060F4615460AD00121AD4AFE
:10650800AD486CF01EFF6FF00406304613B0BDE8CE
:10651800F08F82B10846FFF733FD7B7EDA0704D49B
:106528009D07F2D53B7E002BEFD1204613B0BDE886
:10653800F04FFFF79BBF4A7E00F12809900705D569
:10654800802B09D13846FFF71BFDDEE7910700F0E5
:106558003884002B40F03584D3071ED53B8A082B9E
:1065680012D1FA68394613680020A3625368C9F843
:1065780004306DF0E1FA059080B18F4801218F4A0F
:106588006CF0DFFE059805E08B4801218C4A6CF021
:10659800D8FE3846FFF7F4FC1EE00597FFF73AF9F6
:1065A800002394F82850874A15F0600F8350C5F3EC
:1065B80041131CD0032B40F064836FF08505FFF76F
:1065C80029F9804B1B58002B00F0A183002D00F007
:1065D800698305980028DDD148466DF084FC0346A0
:1065E800A069002B00F02884802100F02EBC4846CA
:1065F8006DF079FC94F82930002840F02C81013B9B
:106608000A2BDAD801A252F823F000BF5367000022
:10661800C3650000D9670000C3650000416600003B
:10662800C3650000C3650000C3650000A7660000DD
:10663800C36500001B670000A069618D03697F299D
:1066480093F88030B9D8A28D002AB6D1E28D002AFD
:10665800B3D1EE06B1D194F83020022A02D14FF01E
:10666800FF35ACE71D070BD5C9B26DF072FC0546C6
:1066780048B1638D0121544A4F486CF06BFE9EE788
:10668800012384F8393094F83030012B05D1638D1B
:106698001BB984F83030002591E70123F9E720463B
:1066A8006DF0E9FA628D0146FF2A86D8E38D002B4A
:1066B80083D194F82830D8067FF47FAF94F830302F
:1066C800002BCCD092B9618D94F838308B42E2D04F
:1066D8002046C9B200F0E0FE638D054668B101218D
:1066E80000903A4A34486CF03FFE68E72046D2B240
:1066F8006DF0D8FC0028E6D1B1E7002B14BF0222C8
:106708000122052184F8302020461A466DF03FFE0C
:10671800C1E705F01F05012D7FF44FAFE38D002B76
:106728007FF44BAF628DFF2A3FF647AFA18DFF295B
:106738003FF643AF94F83030022B90D12046D2B2C6
:10674800C9B26DF05FFD054639E7E38DA68D002BD4
:106758007FF433AF94F83030002B80D0012B02D176
:10676800002E7FF47CAF15F01F0515D0022D92D1B5
:10677800B4F82A80B8F1000F8DD1F6B23146204620
:1067880001F03AF9421C05463FF419AF424631463A
:1067980020466DF0AEFB12E7002E7FF460AF638DEC
:1067A800012B7FF478AF94F86C3066F3C30384F858
:1067B8006C3070E756500A00B06C09008E500A0021
:1067C80077500A000C000000B0500A00D2500A00AE
:1067D800A38DE28DDEB2002A7FF4EFAE628D022A2D
:1067E80011D105F01F0535434FEA13217FF4E5AEBB
:1067F8000122A0696DF08DFB00287FF4DEAE012335
:1068080084F8393047E794F8301000293FF427AF6F
:10681800012902D1002B7FF422AF15F01F050FD0FC
:10682800022D7FF438AF002A7FF435AF3146204679
:1068380001F0C0F8431C05463FF4C1AE0122A6E7AB
:10684800002B7FF40CAF012A7FF425AF94F86C304D
:1068580043F00803ABE70A2B63D8DFE813F00B001B
:10686800620062006200620062003A006200DD01BC
:106878006200F201E38D022B53D194F83030002BE3
:106888004FD0012BA18D01D100294AD115F01F0548
:106898000ED0022D17D00026022120466DF02EFDC5
:1068A800054618B131460C306DF083F90595F2E6CE
:1068B800002936D194F86C309E0806F00206C3F31E
:1068C80000131E43E8E72046C9B26DF03BFD0646BB
:1068D800E2E7618DED064FEA1123C9B207D0002324
:1068E80020460AA90A936DF04DFB0A9DDEE7013B9D
:1068F8000E2B16D8DFE813F00F0030003800150013
:106908001500D200360015001500150015001500F9
:10691800150015000F0120466DF0ADF918B10128DA
:1069280018D00025C2E7266F002EFAD0B4F82E80C2
:1069380033782046984528BF984641466DF0DEFCDE
:1069480005460028B2D04246314605F10C006DF0EC
:106958001FF9ABE7666FE7E700222046FFF7FEFC6A
:106968000546A3E70122F8E70A46204603216DF011
:106978000EFA80460028D4D06DF0B0FAE58D98F86C
:106988001530B8B998F814608DF82930AE428DF8F2
:10699800286028BF2E46D8F8103031461B8820467C
:1069A800ADF82A306DF0AAFC05460028B9D0324669
:1069B8000AA9CAE74FF0000AB44A8DF81130D8F88E
:1069C80008308DF810A01A40B14B9A4255D11021C9
:1069D80006A828F0C5FE061E36DB0AAB102E984620
:1069E80028BF1026AB4806AA564503F1020334D83F
:1069F800B6000236F6B28DF81060AE4228BF2E46B9
:106A0800204631466DF07AFC0546002889D0022ED2
:106A1800B34628BF4FF0020B5A46A6EB0B06C346F7
:106A280000F10C0A504604A96DF0B2F8730808EB9F
:106A380056025A4528D1F0077FF538AF504618F866
:106A480003106DF0AEF831E758367FF46AAF0121D4
:106A5800914A92486CF075FC63E712F8011B0AF141
:106A6800010A4FEA111C01F00F0110F80CC0415C3B
:106A780003F802CC03F8011CB6E798F81460D8F8BC
:106A880010808DF81060B8E750461BF8011BCDE95F
:106A980002236DF08EF8DDE90223CAE720466DF087
:106AA800EAF8D4E91C53002808BF1D460A2300262B
:106AB8008DF8283006232046CDF82A60CDF82E60C0
:106AC8008DF829306DF0DCF801287FF42AAF002D0D
:106AD8003FF4ECAE6B882046ADF82A302B798DF860
:106AE8002C306B798DF82D30AB798DF82E30EB7911
:106AF8008DF82F306B7C8DF83030E68D9DF828307E
:106B08009E4228BF1E4631466DF0F8FB0546002818
:106B18007FF44DAFCAE620466DF0ADF820B10128EC
:106B28007FF4FFAE636F00E0236F002B3FF4F9AEF4
:106B38005B88B3F5007F7FF6F4AE594B04F14C0641
:106B48000A9300238DF82C30E36C9E4208BF002383
:106B5800BDF82A2093B1597D0F2908D1197D0A441F
:106B6800ADF82A209DF82C2001328DF82C20226DBA
:106B78009A4201D01B68EBE7BDF82A20B4F82E80B2
:106B88002046904528BF904641466DF0B7FB054624
:106B980000283FF4C6AE9DF8282000F10C0A4245B3
:106BA80028BF424650460AA96CF0F2FF9DF82830EB
:106BB800434594BFA8EB0308A8EB0808B8F1000FF9
:106BC8003FF474AED4F84CB0B3453FF46FAEBBF1AC
:106BD800000F3FF46BAE9BF815300F2B15D19BF8C7
:106BE80014205046424528BF4246DBF810106CF08E
:106BF800CFFF9BF81430434594BFA8EB0308A8EBDC
:106C08000808B8F1000F3FF451AE236D5B453FF41F
:106C18004DAEDBF800B0DAE794F83030002B3FF4E3
:106C280080AEE18D01297FF47CAE94F8386020466F
:106C38006DF064FB054600283FF438AE31460C3051
:106C4800FFE605F01F05012D7FF46BAE20466DF0C1
:106C580017FA00283FF465AEA38D4268FF2B3FF674
:106C680060AE12799A42FFF45CAEDAB20F2A3FF6B0
:106C780058AEE18D01297FF454AE234493F83A606D
:106C8800D5E7204605A96DF07DF95CE500FF020017
:106C98000003020061C90A00F5500A00B06C09003F
:106CA800050F050074F097F84FF47A76A0FB060CF0
:106CB80047F61222002306FB01C1FAF72DFA654BAD
:106CC800D3E8AF1F41F28732461A9642624A39D951
:106CD800D3E8EF6F8E4204D1C3E8EC0FBCF1000F8C
:106CE800F6D12FD1D2E8EF3FC2E8E15F0029F9D110
:106CF80023B10221594A5A486CF02CFB0221594A07
:106D080057486CF01EFBFEF785FD574B1D58002DAC
:106D18007FF45FAC7B7EE28DD9071BD548466DF0CA
:106D2800E2F8B8B9BAB12946A06971F06AFA014621
:106D3800059000283FF450AC204613B0BDE8F04F52
:106D480000F0F2BDD2E8EF3F0133C2E8E13F00298D
:106D5800D9D0F7E73AB92046FFF7A4FB00287FF41B
:106D68003BACFFF7E2BB48466DF0BDF8059D18B98E
:106D78002846FFF705F9EEE7002D3FF42DAC29462C
:106D8800204600F0D1FD08B1284603E4A069036954
:106D980093F8801011F004017FF4C7AB71F045FA45
:106DA800054600283FF418AC0146204600F0BCFD1B
:106DB80000283FF4BAAB01212C4A29486CF0C1FAEB
:106DC800E2E752077FF508AC002B3FF4BBAB38462F
:106DD800FFF7D6F894F83930002B3FF496AB94F8C7
:106DE8002930052B0CD1618DA069C9B26DF0B1F8BD
:106DF800054628B1638D01211D4A19486CF0AAFA8D
:106E080094F82930032B11D1638D022B0ED1A18D5B
:106E180000220E0A3146A0696DF07BF8054628B1BC
:106E280001213346134A0E486CF094FA00232E468B
:106E380084F83930FFF769BBE38D002B3FF4D4ABFE
:106E48000599003918BF0121C90171F0F1F8FFF760
:106E58006CBB00BF305500202C55002017510A008C
:106E6800B06C09002B510A000C00000054510A00B4
:106E7800B0500A0078510A000B7810B4062B14D1D0
:106E88000369D3F89C20EFF31184202383F312883D
:106E9800BFF36F8F00204B681860506A60B9C2E971
:106EA800083384F31188BFF36F8F0022002304484E
:106EB8005DF8044B73F097BB03605362F1E700BFC2
:106EC800601E002030B589B0002200230024CDE9DF
:106ED80006236FF007034FF48062CDE90334CDE950
:106EE8000144154B1549009415482BF0BFFF15496F
:106EF800134873F013FE144B14498B4207D3002038
:106F0800134B14498B420CD3002009B030BD03F158
:106F18001402D2E8EF0FC2E8E54F002DF9D118337B
:106F2800EBE703F11402D2E8EF4FC2E8E50F002DBA
:106F3800F9D11833E6E700BFB96F000070D7002019
:106F4800E02A00201F8F0A0088210020E821002065
:106F5800E82100204822002038B50D466DF090F851
:106F680030B90121BDE838400F4A10486CF0E9B942
:106F7800C46804B938BD2B78032B05D0052B0ED077
:106F8800022B08D02468F4E7606883685B69002BEB
:106F9800F8D09847F6E7606883689B69F7E7606808
:106FA8008368DB69F3E700BF9F510A00C06C0900E2
:106FB8002DE9FF4120274FF0FF334FF0FF3264489F
:106FC80001A92BF071FA039B1B69D3F89C40236A33
:106FD80093B1EFF3118287F31288BFF36F8F216AA1
:106FE80029B1606A0B688142236208BF636282F339
:106FF8001188BFF36F8FC9B99DF80430062BDAD01A
:10700800072BD8D801A252F823F000BF597000000E
:107018004D700000817000005F700000B5700000C6
:10702800A3700000BF6F0000497100000B7E20466E
:107038005D06D1F81E2002D1FFF754FAC7E76DF0BC
:107048006FF8C4E70022012120466DF0A0F9B2E7ED
:1070580000221146F8E794F86C3043F0040384F8F2
:107068006C3094F83030022B03D1204601A9FFF789
:1070780073FF00220321E7E794F86C3023F0040340
:1070880084F86C3094F83030022B03D1204601A9E3
:10709800FFF762FF00220221D6E794F83030022B76
:1070A80089D1204601A9FFF757FF84E794F86C308F
:1070B800A66923F0040384F86C30D6F80880336995
:1070C800A033D3E8AF3F9A071ED53046D8F83C30F6
:1070D8009847D8F824300021304698470546D8F814
:1070E80040303046984795B11A4A01211A486CF049
:1070F80028F90022042120466DF049F9002D3FF4BB
:107108005AAF2A4607219FE74FF0FF35ECE729469B
:10711800204600F0C1F9054608B1104AE5E7A06924
:1071280071F0A2F8831E5842584194F86C3084F8E4
:10713800305023F0680343EA401384F86C30D8E7F2
:107148000121074A04486CF0FCF80621029A7BE703
:10715800601E0020CE510A00C06C0900FC510A00D4
:1071680028520A0038B5024605460C49806971F074
:10717800D9F8044630B10121094A0A486CF0E1F80F
:10718800204638BD85F83800284600F043F9044603
:107198000028F5D0A86971F0F4F8F1E7816E0000D5
:1071A80038520A00C06C0900F8B501231D460C6866
:1071B800002C35D063F07F02D6B202F07F02103285
:1071C80024FA02F7FF0716D5046824FA02F7FF0726
:1071D80008D4334613480121134A6CF0BBF86FF00A
:1071E8001500F8BD05FA02F224EA020404600C68EE
:1071F80024EA02040C60DC40E6070ED5026822FA95
:1072080003F4E40700D4E5E705FA03F422EA0402EC
:1072180002600A6822EA04020A600133102BC6D110
:107228000020DEE7F06C09005F520A002DE9F04FFC
:107238000026536891B0D4680A9008910692029388
:107248000E96039674B9039B029A09339BB2937006
:107258001B0AD370069B1671DC68002C40F0C780AF
:10726800A346AEE04FF0000A6068CDF83CA0836802
:107278001B6B002B00F0AC8008999847002800F0A1
:10728800A7803546C4E903AAA0F1040959F8043FC8
:107298000BB11A789AB9B54240F29780E3680F9A11
:1072A8001343E360606883689B6A002B00F0928058
:1072B80098478346002800F09080534A7DE05A782A
:1072C8000B2A08BF9D70D9F800305A78042A10D1CB
:1072D800E2680F990A43E260DA78002A5CD1012259
:1072E8009D702369AA40134301352361EDB2CDF89F
:1072F8003CA0D9F800707B78052BC7D16FF0120B32
:107308004FF001080A9B9B69099379793A790E9B9A
:1073180042EA0122ADF8362097F902205FFA88F197
:10732800002AACBF424641F080010493B7BF4BB27C
:107338004FFA88F321F080020793A8BF0793049BB4
:10734800B8BF103223FA02F0C0072CD40F9B23FADF
:1073580002F20593D30726D4BB79FA7809980093EB
:107368000DF136030B9170F0D9FD0B998346D0B916
:10737800079BB970002B4FF00103BCBF21F08001BF
:1073880010318B4004980599BDF8362019431843ED
:10739800CDE90E01BA8079E76A1E9A700FA90EA886
:1073A800FFF702FFA3E708F10108B8F1100FACD10D
:1073B800BBF1000F3FF46AAF144A012114486BF087
:1073C800C0FF584611B0BDE8F08F6FF0150BF3E71A
:1073D800354667E76FF0850B6FE7606808996CF0D2
:1073E8006FFE039B2E460344246803932AE7E36851
:1073F80004F10C01A3600EA8FFF7D6FE08B92468B3
:107408002BE76FF0150BDCE7A0520A007C520A004C
:10741800F06C090070B5836905461B69026F93F823
:107428008030C3F34113022B0CD0032B0CD0012B5B
:107438000CBF10230823D371EE6D3EB96E6DBEB933
:10744800344611E02023F6E74023F4E732460121D1
:107458002846FFF7EBFE044640B173685B790B4A98
:1074680001210B486BF076FF204670BD3668E4E7D3
:10747800324600212846FFF7D9FE044618B1736842
:107488005B79044AECE73668D9E700BFC4520A00C2
:10749800F06C0900E7520A002DE9F04105460E4656
:1074A8006CF0E9FB95F83830804633B328466CF029
:1074B800E7FD0746F0B1014628466CF051FE102260
:1074C8000446002105F13A008EF0E4FD002385F81A
:1074D8003830FF683FB984B119491A486CF0AFFDDC
:1074E8002046BDE8F081786883685B6A03B19847F5
:1074F8003F68EFE76FF03C04EEE71EB985F83860A7
:107508000024EDE73246414628466CF0A5FD0746C3
:1075180090B1024628466CF04DFE04460028DFD1A3
:1075280085F83860FC68002CEAD0606883681B6ABC
:1075380003B198472468F6E76FF03C04D0E700BF32
:10754800A04F0A00A86C09002DE9F04105460F4636
:107558001446D2F804806CF076FD95F86C30D907A3
:107568000BD5474947486CF06AFD6FF00F07281D97
:107578006CF070FD3846BDE8F081012F0AD128462D
:107588006CF07EFB30B940493E486CF058FD6FF016
:107598008507ECE798F807309A0607D5AB691B69A9
:1075A80093F880309B0701D43849EDE71FB1012FCC
:1075B80006D03749E8E7EB6D2BBB05F1540603E02D
:1075C8006B6DABB905F15C06002233680BBB002F6D
:1075D800D5E91C2308BF13465B7C626803F10103ED
:1075E800DBB25371D5E91C1208BF0A46537422E076
:1075F8009C4206D1274923486CF021FD6FF01507FE
:10760800B5E71B68DDE79C4201D12349F3E71B6816
:10761800D2E79C4221D12368CAB972683360944288
:1076280000D173600023236063685B7902211B4AE1
:1076380014486BF08FFEA168B9B128466CF0C1FB05
:10764800074668B116490F486CF0F9FC8FE71360DC
:1076580073689C4208BF7260E4E71A461B68B5E786
:10766800A0686CF03BFC88F8060000232360736870
:107678001BB9C6E90044002779E71C607460FAE783
:1076880038530A00A86C09005A530A0014530A0018
:1076980078530A0098530A00B5530A00D2530A00D7
:1076A800EF530A00F8B5054600AF29B301290BD1FD
:1076B800184C194E2BE0636828461968F9F786FDBF
:1076C800B8B11834B442F6D36C4688B06A46134B46
:1076D800CDE905354FF40073ADF81C30104B42F876
:1076E800103F00234FF4E2510E48FCF759FDA54620
:1076F80000242046BD46F8BD0B4C0C4EE2E76368FB
:1077080028461968F9F762FD0028F2D01834B44207
:10771800F5D3D9E7E82100204822002026540A00A2
:1077280003000001B86C090088210020E82100202E
:1077380070B5012501F07F0311F0800F18BF1033D9
:107748009D4090F830300446022B06D001210C4AA7
:107758000C486BF0F6FD002070BD90F838606CF0B6
:107768008AFA3246014620466CF076FC0028F2D0B0
:10777800C0680028EFD083681D42EDD10068F8E7A3
:1077880044540A00B86C09002DE9F8430546084638
:10779800114616469846FFF785FF0446002843D051
:1077A80028466CF086FC95F86C30DA0702D5204A3A
:1077B800012109E0D4F8049004F11407D7E8AF3F99
:1077C800DB070CD502211B4A1B486BF0BAFD6FF092
:1077D8000F04281D2AF03EFF2046BDE8F883D9F89B
:1077E80004301BB1AB4201D0144AE1E742463146AE
:1077F80028466CF031FCA0B10023236003696BB903
:10780800C0E90344D7E8EF3F43F00103C7E8E23F8C
:10781800002AF7D10024C9F80450DAE71C60046193
:10782800F0E76FF03C04D4E76FF01204D4E700BF30
:1078380038530A0069540A00B86C09008B540A00CE
:107848002DE9F04F83B000AF7B6097F830304C687B
:107858000E463B60814690466CF00DFAA3680146DF
:107868001B6B33B96FF0150420460C37BD46BDE8D5
:10787800F08F204698470028F4D00024051F06F111
:107888000C0A55F8041F09B10B782BB9002C14BF4A
:1078980000246FF03C04E7E74B78042B0ED1002C52
:1078A8003CD18B787A689342EBD1CB783A68934293
:1078B800E7D10B79002BD7D00124E2E7052BE0D1E3
:1078C800002CDED0B8F1010F91F802B009D0B8F160
:1078D800020FF1D152465946D9F818006CF0F8FC5D
:1078E80004E05246D9F818006CF0D6FC044600288B
:1078F800E2D06D468AB06A46F368CDE907B306233D
:1079080007490990CDE9051842F8103F00234FF4C4
:1079180041510448FCF744FCAD46A5E70024A3E721
:10792800CB540A00E86C09002DE9F0410B7E0C46A7
:107938005906054637D16BB36CF0DDF940B11B48E9
:1079480001211B4A6BF0FDFC4FF0FF30BDE8F081D0
:107958002846D5F87080268AEF8D6CF08CF9F8B13E
:10796800421E534253419B01228A9AB1BE4232467B
:1079780028BF3A46E98D91420CD9B2FBF3F103FBDB
:1079880011223AB994F91830002BBEBF637E43F038
:10799800080363762146A869BDE8F04170F0A4BBEE
:1079A80098F80730E0E76FF01500CFE7D86C0900CA
:1079B80007550A0070B5064680690C4670F038FB1A
:1079C800054638B102212346094A0A486BF0C2FC31
:1079D800284670BD012214F0800F18BF24F08004DF
:1079E800736B18BF1034A2401A437263F0E700BFEC
:1079F8001B550A00D86C090070B5054680690E460B
:107A080070F041FB044638B102213346054A064866
:107A18006BF0A0FC204670BD314605F134006CF0D7
:107A28002DFCF7E732550A00D86C090070B50646F8
:107A3800EFF31181202383F31288BFF36F8F1B4D5F
:107A48002A6881F31188BFF36F8F526892F86C200F
:107A5800D20705D4BDE87040202200232BF056B988
:107A6800EFF3118283F31288BFF36F8F2C682CB168
:107A7800696823688C422B6008BF6B6082F31188A9
:107A8800BFF36F8F44B1606804F10801C369984778
:107A98002146074872F044FD2B6833B13046BDE8F3
:107AA8007040002200232BF0F9B870BD3455002037
:107AB800D81D002030B585B0CDE90012054600225A
:107AC8000023144803A92AF055FC0246E8B9DDE969
:107AD8000001039B5D60083383E80300EFF3118026
:107AE800202383F31288BFF36F8F039B1A600A4A1F
:107AF800516861B9C2E9003380F31188BFF36F8F11
:107B08000022002305482BF0C9F805B030BD0B60F2
:107B18005360F1E7D81D00203455002000000020F4
:107B280073B5202504698DF80710EFF3118685F3E6
:107B38001288BFF36F8F0122206C0DF107016AF0E4
:107B4800DFFF86F31188BFF36F8F012812D072F020
:107B5800DFFFC8B10122104BD3E8EF1F002903D182
:107B6800C3E8E02F0028F7D104D102210B4A0C48C2
:107B78006BF0E7FB237F2BB12022002304F14800A0
:107B88002BF08CF802B070BDA37E002BE2D0002150
:107B9800202073F0C5F8C8E73C5500205C550A0062
:107BA800A06C090038B5002405690E492B6C05F155
:107BB8004800C3E90144DC60AB6BC3E90144DC6005
:107BC80072F04EFF05F17800074972F0ECFE0749A4
:107BD80005F1280072F0E7FE28466CF0FDFB204610
:107BE80038BD00BF197D0000617E00002D7F0000B8
:107BF8002DE9F341036906460D46D0F804801C6957
:107C08000F7E002A32D00B8A71323E480BBF022108
:107C180001213D4A3D4A00933B466BF0A5FB3046A7
:107C28002F7E6CF042FC874204D1042104F18800C5
:107C38006CF0E8FC30462F7E6CF045FC874204D19E
:107C4800052104F188006CF0DDFC30462F7E6CF0D5
:107C58001EFC874203D104F18C002AF0E3FD29467B
:107C6800404602B0BDE8F0416CF069BB6CF01DFC09
:107C7800B84214D12A8AE968A06B6AF041FF28B19A
:107C8800236A1BB104F128002AF098FF04F1880048
:107C980004216CF0B7FC04F178002AF08FFF30461D
:107CA8002F7E6CF010FC874215D1236A1BB104F1BA
:107CB80028002AF083FF052104F188006CF0A2FC5B
:107CC800237F9BB9002340F6354204F148002AF08F
:107CD800E5FF0123237730462F7E6CF0D8FB8742DF
:107CE800BDD104F18C002AF03BFDB8E7236C5A891A
:107CF800DB889A42EFD00022002304F148002AF0E2
:107D0800CDFFE8E7A06C09007B550A009F550A00E3
:107D18002DE9F04750F8483C00F140075B680546FC
:107D280000213846D3F800906CF0ABFB002864D0F3
:107D3800012138466CF0A5FB804600285DD155F836
:107D4800083C5A89DB889A4203D115F82D3C002B50
:107D580053D0D7E8EF4F44F02003C7E8E23F002AAA
:107D6800F7D114F0200448D148466CF0ACFB00224F
:107D78008246002322486BF073FE064650B9384607
:107D880005216CF03FFC2846BDE8F047202200237F
:107D98002AF084BF80F818A015F82C3C33B1428A29
:107DA800C16855F8080C6AF0CBFE0446214606F176
:107DB8000C006BF0E7FE5CB1D9F804006CF000FC35
:107DC800B4FBF0F303FB1044B4FA84F84FEA5818F4
:107DD8003146484605F82D8C6CF099FA68B10121B6
:107DE800084A09486BF0ADFA3046FEF7C9F838463C
:107DF800BDE8F04705216CF005BCBDE8F08700BF81
:107E0800541F0020C0550A00A06C090038B503466D
:107E18001B6940685D68AC68A37A84F8223094F8DE
:107E28002D3084F82330A376696849B1237C3BB9A7
:107E38006BF0C7FF30B10121054A06486BF081FAA3
:107E4800002038BD68686CF049F82074F8E700BF76
:107E5800D2550A00A06C090070B550F8782C00F1D2
:107E68001004526803460021204615686CF009FB8F
:107E780000284DD0012120466CF003FB002847D193
:107E880053F8402C68689388918916695B1A9BB2ED
:107E9800F61A6CF095FBB0423AD8D4E8EF3F43F0BD
:107EA8001002C4E8E12F0029F7D1DB0606D5BDE8AA
:107EB80070400221174A18486BF043BA28466CF004
:107EC800F4FA00220646002314486BF0C9FD044664
:107ED800F0B1067668686CF073FB638A984203D247
:107EE80068686CF06DFB83B22146284663826CF0AB
:107EF8000EFA68B128466CF0D8FA03460648012104
:107F0800074A6BF027FA2046BDE87040FEF738B8FC
:107F180070BD00BFFC550A00A06C0900541F00206A
:107F28001C560A0038B550F8083C044633B9BDE879
:107F3800384001212A4A2B486BF003BA50F8283CF4
:107F480000F160055B6802211A680023838283833D
:107F580028466CF096FAB8B154E90231106998478E
:107F6800637D1BB104F150002AF028FE0521284644
:107F78006CF087FA98B9637F6BB10022002304F193
:107F880020002AF08BFE0AE0032128466CF079FADB
:107F98000028E1D1E4E714F80D3C002BEDD10221D3
:107FA80028466CF06EFA38B12369DA885B899A4200
:107FB80002D020462AF002FE032128466CF061FA1E
:107FC80060B1A2699388918912695B1A9BB29A423F
:107FD80004D02046BDE838402AF0F0BD38BD00BFC7
:107FE80041560A00A06C0900D3B5002600270446B4
:107FF800CDE9006705486BF037FD28B1230658BF67
:108008000023047658BF038202B0D0BD8820002028
:108018002DE9F04383B000234FF0010805691C4C9B
:108028001C4E02AF28602B7785F8203005F1240913
:10803800B442234601D3002019E095F820201034DB
:10804800CAB16C4688B01B6802AA1349C2E9051375
:108058004FF400739383114B42F8103F10480023EC
:108068004FF4E251FCF79CF86FF00B00A54604377B
:10807800BD46BDE8F08385F8208054F8043C4846A6
:10808800009354F8101C54E903236CF087FDCFE7E4
:1080980000220B0010220B00A3560A000300000167
:1080A800F86C09001FB5CDE9010103924FF0FF32CA
:1080B8004FF0FF3301A9034872F095FA002005B08C
:1080C8005DF804FB301E00201FB500230190CDE9A8
:1080D80002334FF0FF324FF0FF3301A9024872F02C
:1080E80082FA05B05DF804FB301E00202DE9F0414E
:1080F800044617460E4600686CF0B8FB31463A460F
:108108008046FFF771FFD4F87B300546DB1B01463C
:10811800C4F87B3020686CF0FAF888B10B4A434603
:1081280001210B486BF016F9314620466CF069FCCA
:108138002846FDF725FF2046BDE8F0416CF02DBC30
:10814800A37F0133A377BDE8F08100BF1C560A0066
:10815800F86C09002DE9F84F044600686CF09BFBA9
:108168004FF030090746E37F012B1ED82368D3F868
:1081780010B0D3F804A09BF8616009FB06B624365A
:1081880030466CF031FD31460246804650466CF070
:1081980098FB9BF81F30054633B1A8EB0002314627
:1081A80050466CF08EFB05460DB9BDE8F88F2046A9
:1081B8006CF044FB2A46014606463846FFF714FF92
:1081C8000546014620686CF0A2F880B101213B46C3
:1081D800094A0A486BF0BEF82846FDF7D1FE314639
:1081E80020466CF00EFCBDE8F84F6CF0D6BBE37F80
:1081F8000133E377B7E700BF1C560A00F86C0900A3
:108208002DE9F04FB94F89B04FF0FF324FF0FF33EF
:10821800B74805A92AF048F9059E069D3469002D3E
:1082280040F09080257704F1240694F820309D4290
:10823800C0F2828004F11803D3E8EF2F22F0020283
:10824800C3E8E12F0029F7D1D3E8EF1F21F004019B
:10825800C3E8E21F002AF7D104F11803D3E8AF3FBF
:10826800DB07D1D5237F022B00F08E81032B00F092
:10827800878153BBDDF814A0DAF81050EB7F23BBDD
:1082880050466CF008FB814628466CF0D7FA4FF44C
:108298000072014606464846FFF7A6FE804601469C
:1082A80050466CF034F8002800F0668101214B46F6
:1082B800904A91486BF04EF84046FDF761FE314612
:1082C80028466CF09EFB6CF068FBA37F002B9BD1CB
:1082D800237F012B40F07D81302304F1630694F85D
:1082E8006150304694F8621003FB054500F060FACF
:1082F8002435024631462369284600F077FA0646B7
:10830800C4F8840028466CF065FC814628466CF069
:1083180066FC804628466CF067FCE26D3044002A13
:1083280040F03B81002840F0338128466CF083FC04
:10833800003818BF01202CE130466CF042FC0135B2
:10834800303672E7DDF81C80D6F804A095F818904E
:10835800B8F1000F21D02B8A18F1710F66480093ED
:1083680008BF02214B4616BF0121644A644A6AF0DD
:10837800FBFF304695F818806CF08DFA804540F088
:10838800EF80E37F013BE377204669696CF039FBB6
:10839800294650466BF0D3FF5EE730466CF07BFA17
:1083A800484540F09580237FD5F80C80B5F810B08B
:1083B800002B49D1BBF11F0F42D1D8F80030BB4286
:1083C8003ED1414604F1540308F11C0251F8040B54
:1083D800914243F8040BF9D10A881A808A7842211D
:1083E8009A70552384F87330532384F8743084F8D2
:1083F8007630A36DE26DC4F877300023C4F880307E
:1084080094F86030C4F87B209A0684F875100FD170
:1084180094F8612094F820309A4209D294F8623096
:10842800013B0F2B04D8012384F87F302377A0E782
:1084380020686CF026FA022384F87F300423F5E7DD
:1084480020466CF0AAFA94E7032B92D1302394F8D3
:10845800619003FB0949D4F8803009F124095B4491
:10846800C4F88030BBF1000F16D048466CF0BCFB56
:1084780090B141465A4648466CF0C8FB804628B938
:1084880002215B461F4A1C486AF064FFD4F87B301F
:10849800A3EB0803C4F87B30D4F88020E36D9A423C
:1084A8000DD248466CF0A0FB00287FF462AFD4F8E8
:1084B8008020E36D9A4202D220686CF0F8F94846B1
:1084C8006CF0B9FB003818BF012084F87F00B5E7CD
:1084D800304695F818906CF0C9F981457FF449AF9A
:1084E800237F052B10D184F81C8042E75553424363
:1084F800301E00201C560A00F86C09007B550A0043
:108508009F550A00BA560A00022B7FF432AF4FF08B
:1085180030092A8AD4F8803094F861801344C4F86A
:10852800803023681969D3F804B091F8613009FBE9
:1085380003112431084603916CF056FB0399024657
:1085480058466CF0BEF900287FF413AFD4F87B309E
:1085580013B120686CF095F909FB08402430AFE7A7
:10856800304695F818806CF081F9804502BFA37FEA
:1085780003F1FF33A37707E7EB7F0133EB77A4E63B
:108588002046FFF7E7FDA0E620466CF04AFA9CE695
:10859800022084F87F0004231AE094F9601040B99F
:1085A8000029206802DA6CF06CF9BEE66CF07FF9FD
:1085B800BBE6002914DA904202D8B9F1000F06D1BF
:1085C80020686CF05EF9022384F87F30E3E7022329
:1085D8002377237F022B0ED120466CF022FA13E674
:1085E800904202D8B8F1000F03D120686CF05FF90F
:1085F800E9E70323ECE7032B03D12046FFF7AAFDA5
:1086080002E6042B7FF400AEA37F2BB101211D4AA3
:108618001D486AF096FEF7E520686CF027F9804659
:1086280020466CF00BF90546024604F1730304F189
:108638007F0153F8040B8B4242F8040BF9D11B78E5
:108648002946137040460D22FFF7CEFC0646014628
:1086580020686BF05CFE78B10C4A434601210A4859
:108668006AF078FE3046FDF78BFC294620466CF010
:10867800C8F96CF092F9C7E5A37F0133A377052306
:108688002377C1E5E0560A00F86C09001C560A0079
:10869800802938B50D46144621D083290DD019BB41
:1086A8008023537183230320117193710023E07099
:1086B80023706570A370043038BD02231371012341
:1086C8005371002393710A23D37108224168A018BB
:1086D8008DF017FD064B0E201B882382E6E7044B1E
:1086E80002201B889380E1E76FF08500E4E700BF74
:1086F80077C80A002DE9F0418769D0F82480BA428A
:1087080028BF3A46B2FBF8F40646C2692346006819
:108718006AF0F9FF0546C0B9B7FBF8F7A7420BD1D5
:10872800002205213068FCF761F828B101210A4AC6
:108738000A486AF006FE0125F3692344F3613DB156
:108748000020074BB362BDE8F08100240125E7E76C
:10875800706A6043F7E700BF01570A00F86C090028
:108768000203000C81420B4607B509D302210D4ACA
:108778000D486AF0EFFD6FF0150003B05DF804FBDB
:108788006AB101391144814201D28B4207D90221D1
:10879800009305481346054A6AF0E6FDEBE700201A
:1087A800EBE700BF18570A00F86C09002F570A00BA
:1087B8000C290346084616D11B78252B12D009D858
:1087C800122B10D8084A42FA03F313F0010F08BF1E
:1087D8000620704703F0FD02282A03D05A2B08BF51
:1087E8000A2070470A207047F6FFFBFF2DE9F04189
:1087F800984690F82C3086B023F00C0380F82C3083
:108808000023C0E904338361062A04460F460B7827
:1088180040F010810BBB4B795B0724D490F82C30C7
:108828009F070DD402234FF468521946002584F897
:10883800283084F829106285284606B0BDE8F08102
:108848006CF02EF90028EDD1002319461A46EDE701
:108858000223052145F20232E8E7032B36D14E798F
:1088680016F0040604D0022305214FF41052DDE768
:1088780090F82C308DF8076043F0040380F82C3012
:108888007023ADF8043090F829300D7903F00F0308
:108898008DF806300A23122D28BF12258DF80B30CB
:1088A800438D2A465BBA404601A98DF808608DF8C9
:1088B80009608DF80A600396ADF81030ADF81260C3
:1088C800ADF814608DF0C0FBA662B5E71B2B00F075
:1088D800898009D8122B1AD01A2B61D00121B24AEB
:1088E800B2486AF037FDBEE71E2BF7D14B795E0719
:1088F800B9D40B7913F0030300F09780012BA3D1AF
:1089080090F82C3043F0010380F82C309CE74B7929
:108918005E07A8D490F82C3043F0040380F82C307C
:108928004A7812F002061FD1D5078B7822D5B1F804
:10893800035042461946FFF7ABFE6DBAADB2854209
:108948000BDAB7F803506DBAADB200231A4684F8B3
:10895800283084F8296062856EE742462046B97857
:10896800FFF796FE051EF0DA022305264FF4105293
:108978000025ECE72BB102218D4A8C486AF0EAFC0D
:10898800F2E7B1F8035041466DBAADB26CF0BEF8EB
:10899800232DD6D9414620466CF0B8F82425D4E7D3
:1089A8004D7915F004057FF45EAF90F82C3043F054
:1089B800040380F82C308B783F2B0ED1CE78002E14
:1089C800D2D10D790323042D28BF042540462A4619
:1089D80001A901938DF038FBB7E7022305264FF470
:1089E8001052B4E74B7959073FF53DAF3B791A0967
:1089F8000CD19A070AD5DB0715D494F82C3003F06C
:108A08000303032B3FF424AF002305E094F82C2044
:108A18009707C2F34003F0D594F82C2063F3410282
:108A280084F82C2010E70123F6E790F82C2063F354
:108A38000002F5E70A2A7FF451AF2A2B1AD8222B15
:108A48007FF64CAFA3F12302072A3FF647AF01A1F7
:108A580051F822F0D38A0000E5880000558B000009
:108A6800E5880000E5880000BD8B0000E58800006F
:108A7800158C00005A2B7FF431AF4D7A15F00405A0
:108A88007FF4F1AE90F82C3043F0040380F82C30DA
:108A98008B783F2B40F0DD80CE78002E40F0D980D7
:108AA8004FF4C063CDE90136B1F8075040466DBABE
:108AB800ADB2082D28BF082501A92A468DF0C4FAB1
:108AC8003246334684F8282053E07B7A13F00403B7
:108AD8007FF4C9AE01AEADF80430B370082390F846
:108AE8002C208DF8073042F0040280F82C206BF01F
:108AF800D7FF0028B5BF4FF0FF3302220322236AB5
:108B08008DF80C20A8BF1BBA0293636A31461BBAC2
:108B18008DF80D30C3F30722C3F307438DF80F30E8
:108B280094F82C308DF80E2043F0040384F82C3090
:108B3800B7F8075040466DBAADB20C2D28BF0C25CA
:108B48002A468DF081FA0023A36275E67E7A16F034
:108B580004067FF488AE90F82C3043F004039D0798
:108B680080F82C3009D402264FF46853002584F885
:108B7800286084F8296063855EE66BF091FF002821
:108B8800F1D1236A03B1013B94F82C10626A1BBA35
:108B980012BA41F0040184F82C100825C8F80030F6
:108BA800C8F804200023E2E776570A00F86C0900A9
:108BB80059570A007B7A58073FF555AE94F82C3080
:108BC800D7F8026043F004039907B7F8075084F810
:108BD8002C307FF527AE20466BF062FF00287FF42B
:108BE80021AE6DBA36BAADB22A463146206AFFF7D1
:108BF800B9FD20B1022305214FF4045216E6174BA4
:108C08002361636AE6616B43A3611DE67B7A5A07B9
:108C18003FF529AE90F82C30D7F8026043F00803EE
:108C2800B7F8075080F82C309B077FF5FBAD6BF049
:108C380037FF00287FF4F6AD6DBA36BAADB22A46D2
:108C48003146206AFFF78EFD0028D3D1044B6361BB
:108C5800D7E7022205264FF4105333E7774B070076
:108C6800FD86000010B504690346204640F8143B11
:108C78000122002171F0EBFD04F12C00024971F092
:108C880092FE002010BD00BF1D8E000038B50346BF
:108C98001B6940685C681B6925685A681AB19A683C
:108CA8000AB1DA683AB913480121134A6AF049FB54
:108CB8006FF0150038BD1033D3E8EF1F41F0010104
:108CC800C3E8E21F002AF7D1216909B90020F1E7BA
:108CD8002B7A002BFAD16BF074F828B10121074ADE
:108CE80004486AF02EFBF1E720696BF0F7F8287268
:108CF800ECE700BFE06C090091570A00D2550A0062
:108D080038B504694068006804F11005D5E8AF5F1C
:108D1800ED071FD40BB15D683DB9104A1048012119
:108D28006AF00FFB6FF0150038BD90F820501DB1A8
:108D3800DD680DB90B4AF1E785791DB19D690DB95B
:108D4800094AEBE7C4E9021263600274120A42742A
:108D58000020E9E76FF07700E6E700BFBB570A009D
:108D6800E06C0900DA570A00F9570A002DE9F347C1
:108D7800D0F804A00669884615467768DAF80440F2
:108D880006F11003D3E8AF3F9B073BD52369606822
:108D98005B68D3F800906AF06EFF00220023012878
:108DA80029460CBF99F81B9099F81490DAF80C0032
:108DB800CDE9002342466AF057FE054650B9012125
:108DC800124A13486AF0BDFA6FF00B04204602B04D
:108DD800BDE8F087014680F8189020466BF097FAB6
:108DE800044618B12846FDF7CBF8EFE7FB69002BDE
:108DF800ECD14FF0FF324FF0FF3306F1140029F0A9
:108E0800EBFCE3E76FF00C04E0E700BF1A580A0038
:108E1800E06C090070B550F82C3C5C6865681C383B
:108E2800D0E8AF3F9B0725D52B6968685B681E684B
:108E38006AF021FF002201284FF00003A0680CBF50
:108E480096F8296096F822606AF00AFE044630B95E
:108E5800094A0121BDE8704008486AF072BA014623
:108E6800067628466BF053FA20B12046FDF788F8BD
:108E7800034AEEE770BD00BF35580A00E06C0900F0
:108E88004F580A0070B50B7892B006460C4607ADED
:108E9800032B31D8DFE803F0022A2C2E1949284683
:108EA800F8F79EF905956378174A0493A3781E216D
:108EB8000393E3780AA80293237910AD01936379A9
:108EC8000093A37964F0C2FD32460AAB1C4603CC7A
:108ED800AC4210605160234602F10802F6D12068C6
:108EE80010603046A388938012B070BD0749D6E75A
:108EF8000749D4E70749D2E70A212846064A64F019
:108F0800A5FDCFE784580A009F580A00AABA0A00AC
:108F18008B580A0095580A003C7A0A000E4B4029E3
:108F280028BF402170B51D460C4C4618B04203F1CD
:108F3800020304D1002305F81130074870BD0278F8
:108F48001209A25C03F8022C10F8012B02F00F02A0
:108F5800A25C03F8012CE9E717CE0020BAC90A0081
:108F680010B50024094B86B009480393CDE90444A1
:108F780071F06FFD03AB00934FF440620A2305497B
:108F8800034829F021FE204606B010BDC9580A0042
:108F9800A02C002070E100200146014829F054BEB1
:108FA800A02C00200146014829F07EBEA02C0020FC
:108FB8000146014871F022BDA02C00202DE9F7439D
:108FC80006468946174698463C4DD5E8AF3FDA072E
:108FD80022D548B901213A4A3A486AF0B2F96FF005
:108FE800010003B0BDE8F08301A96AF0CEFB0228B6
:108FF80004462BD10246344930468DF053F80028F8
:10900800EDD1D5E8AF3FC3F3C0061B0706D52F4AFD
:1090180021462C486AF095F90020E2E7A5F188047A
:10902800072221464046B84706280AD80121284A7F
:1090380024486AF086F945F8886CE671C4F803603C
:10904800EAE70723B0FBF3F0E071E5E7042818D15D
:109058000246204930468DF025F804460028BED146
:109068001C22404605F1A001B847031E05DA01217C
:10907800194A14486AF06EF9CEE72B4483F8A040E9
:10908800CAE70A28ABD10246144930468DF00AF8DF
:109098000028A4D1B9F1020F07D00A480121104ACB
:1090A8006AF04FF96FF015009BE74A46404605F114
:1090B800BE01B84700EAE07093E700BF080200204D
:1090C800D2580A00B06B090092580A00F3580A00F7
:1090D80017590A00025F0A003C590A006E590A0033
:1090E80079590A002DE9F04389B0DDF840909D795F
:1090F8005E791F7993F803C093F802E093F8018032
:109108000C461B78B9F1000F15D0CDE90639CDE929
:1091180004E81346CDE9027CCDE900560D4A64F017
:1091280095FC002813DBA0422CBF6FF0150000202F
:1091380009B0BDE8F083CDE90583CDE903CE134638
:10914800CDE90167044A009564F080FCE9E76FF017
:109158001500EDE7B0590A00D4590A0010B5FBF71D
:109168004BFD044628B101210346034A03486AF02F
:10917800F1F8204610BD00BFF5590A00B06B090090
:1091880070B504461E4615468CB0AAB129B10A46E8
:1091980002A8042169F0BFFA02A900912B462246D1
:1091A800242103A8FFF79EFF70B93146109A03A83F
:1091B800FBF79EFB0CB070BD03462421044A03A8AC
:1091C80064F044FC2328F0D96FF01500F2E700BFE3
:1091D8001A5A0A0007B50B4B0B48DA79C2EBC202E0
:1091E800009200221146FFF7CBFF034638B1012158
:1091F800064A074803B05DF804EB6AF0ABB803B061
:109208005DF804FB8001002092580A00205A0A00E9
:10921800B06B090030B5044615468DB09AB129B136
:109228000A4602A8042169F076FA02A900912B46A1
:109238002246242103A8FFF755FF60B903A86AF066
:109248007CFA0DB030BD03462421044A03A864F01B
:10925800FDFB2328F2D96FF01500F2E71A5A0A002D
:1092680007B5009313460A4601460348FFF788FFEF
:1092780003B05DF804FB00BF7B770A000A4601468D
:109288000148FFF7C7BF00BF7B770A0007B5009307
:1092980013460A4601460348FFF772FF03B05DF81C
:1092A80004FB00BF75770A000A4601460148FFF72C
:1092B800B1BF00BF75770A0007B5009313460A4689
:1092C80001460348FFF75CFF03B05DF804FB00BFED
:1092D800A6750A000A4601460148FFF79BBF00BF72
:1092E800A6750A0007B500220346009103481146F7
:1092F800FFF746FF03B05DF804FB00BF6D770A0077
:1093080007B500220346009103481146FFF738FFCE
:1093180003B05DF804FB00BF025F0A0007B5002236
:109328000346009103481146FFF72AFF03B05DF892
:1093380004FB00BF6E590A0008B5024829F03EFC3C
:10934800002008BD5C080020F8B51E4DD5E8AF3FE9
:1093580013F0010F2F4632D095F8A040A5F18806EA
:109368003CB91C22184906F594708CF0CAFE86F8A0
:109378004441F3798BB902F04BF8044630B101212E
:10938800124A134869F0DDFF2046F8BDF37923B986
:1093980002F04EF804460028F1D1D5E8AF3F5A074D
:1093A80001D400F0CBFED7E8EF3F23F40062C7E812
:1093B800E12F0029F7D11B0501D5FFF7BDFF0024D8
:1093C800E2E700BF080200203B5A0A00425A0A009E
:1093D800B06B090007B5009313460A4601460348D7
:1093E800FFF7CEFE03B05DF804FB00BFAC7C0A00BB
:1093F8000A4601460148FFF70DBF00BFAC7C0A00D2
:1094080030B50378012B11D0022B21D06BB90A4655
:10941800144B03F1100453F8045BA34242F8045BB5
:10942800F9D143881A0A8A70CB7030BD0A460D4BB1
:1094380003F1100453F8045BA34242F8045BF9D12A
:1094480043681A0C180E4A700870C3F30722EAE73B
:1094580000F11003013913F80129984201F8012F8E
:10946800F9D1E2E7CBC90A0010B56BF047FE71F0FD
:109478004FFB044608B929F0F5FF064BD3E8AF3F88
:109488000BB10A2098471CB9BDE8104029F0FEBF6F
:1094980010BD00BF0062002038B5044608486AF0D5
:1094A800DFFA054648B1631EDBB21F2B96BF054A9B
:1094B8000021D15C0C306AF074FB284638BD00BF2F
:1094C80004200020DBC90A000F2810B50CD80D288D
:1094D8000CD90A486AF0C4FA044618B104210C30C1
:1094E8006AF05FFB204610BD1328F2D009B104488A
:1094F800F0E70220BDE81040FFF7CEBFB4200020FF
:10950800801F0020C3681B780221024A02486BF0C2
:1095180093BE00BF845A0A00786B0900F8B5064666
:109528000F4604F01DFB044690B9394630460BF04F
:1095380003F80546F0B93946304608F0D9FF164B0E
:109548001B6823B153F80C4904B10C3CB3B9F8BDFE
:1095580083781321012B4FF0000312BF1D46D0F86A
:10956800A450C0F8A4306CF094FA204603F06EFEC4
:10957800002DDAD028466EF01FFBDCE79B6813B19C
:109588003946304698472CB1E26802B10C3A234676
:109598001446DBE72246FAE70863002010B50024EA
:1095A80086B003AB00934FF480624FF0FF33054958
:1095B8000548CDE90344059429F006FB204606B08A
:1095C80010BD00BF70ED0020A02D002038B5C46884
:1095D8002378ABB9B4F801500F21284603F09CFF5B
:1095E800E278044688B90D4B194633F8024B44B962
:1095F8006FEA05536FEA135321F81030084B1A54D9
:1096080038BD01300528F0D1FAE70273012103F0D3
:1096180069FE2046BDE8384003F018BE84CB002020
:1096280098CE002070B5C3681D787DBBB3F8016083
:109638000F21304603F070FF044638B90121334644
:10964800BDE87040124A13486BF0F6BD294603F096
:1096580049FEA378012B04D02046BDE8704003F0F2
:10966800F5BD201D6BF0D1FDC307F5D503212046BC
:1096780003F038FE032002F025FF03460028EBD054
:109688000221054A03486BF0D7FDE5E770BD00BF2E
:10969800AC5A0A00786B0900D25A0A0010B5C368A0
:1096A8000121B3F80140204603F036FF38B9012103
:1096B8002346BDE81040044A04486BF0BDBDBDE830
:1096C800104003F0C3BD00BFF85A0A00786B0900C8
:1096D80010B5C36801211C88204603F01DFF38B966
:1096E80001212346BDE81040034A04486BF0A4BD9D
:1096F800BDE8104003F0AABDF85A0A00786B0900CB
:1097080010B501210C306AF08AFA03780121BDE80E
:109718001040024A02486BF08FBD00BF1C5B0A0074
:10972800786B0900014610B508486AF0B0F9084995
:10973800084871F063F9031E06DABDE810400121FC
:10974800054A06486BF078BD10BD00BF84020020B2
:109758007C080020A02E00203E5B0A00786B0900E0
:109768000121024A02486BF053BD00BF5B5B0A004F
:10977800786B090070B5C5680121B5F801603046FD
:1097880003F0CAFE044638B901213346BDE87040EB
:109798000B4A0C486BF050BD2B783BB9D5F8033019
:1097A800C0F89930D5F80730C0F89D30201D4FF427
:1097B80000316BF036FD2046BDE8704003F046BD31
:1097C800F85A0A00786B090008B502F031FE064B1A
:1097D80018466BF01AFD00F00B00D3E8EF2FC3E832
:1097E800E10F0029F9D108BD080200200B46B0B5E9
:1097F8000D8A00AF04462946D868FFF78FFB8AB068
:109808006A460A4BCDE90750CDE9053440F20243D8
:10981800ADF82430064B42F8103F00234FF4325184
:109828000448FAF7BDFCBD46B0BD00BF755B0A0031
:1098380005000001786B09002DE9F84FD0F80C906D
:10984800018A99F8004000AFA30001338B4260D928
:109858006D468AB06A46CDE9073105232E48CDE921
:10986800050442F8103F00234FF421512B48FAF722
:1098780097FCAD46BD46BDE8F88F01212B46284A26
:1098880026486BF0D9FC013699F800309E42F1DA8F
:1098980009EB8603B3F801500F212846B3F803807B
:1098A80003F03AFE04460028E7D000F1C00AB8F1F8
:1098B800000F06D0656945B901211A4A17486BF0AF
:1098C800A7FC204603F0C2FCDDE7A2692B6895429D
:1098D8002046636108BFA36103F0D8FB28F040FF6E
:1098E800C5F800B0236A8BB9C4E90755DAE8EF3F39
:1098F800013BCAE8E23F002AF8D10021204608F1DE
:10990800FF3803F0CDFB1FFA88F8D0E71D60256209
:10991800ECE70026B346B7E7975B0A00786B0900C7
:10992800C25B0A00DE5B0A0080B500AF8AB06A46F7
:10993800094BCDE90530094B079340F20133ADF8E7
:109948002030074B42F8103F00234FF412510548CE
:10995800FAF726FCBD4680BDF55B0A0007890A00B8
:1099680004000001786B090037B50446084602EB8D
:10997800C3039A4202D16FF05E0010E0114611F85D
:10998800085BA54211D1038A5178994209D9084840
:109998000121084A009469F0E7FC6FF0150003B054
:1099A80030BD536898470020F9E70A46E1E700BF51
:1099B800786B0900115C0A002DE9F0470C4629F084
:1099C80051FDE5682B78022B72D0042B07D00121BA
:1099D8003B4A3C486BF030FC6FF015040EE0B4F8DD
:1099E8001080B8F1020F0ED84346374A3548012196
:1099F8006BF022FC2046FCF7C3FA002429F046FD50
:109A08002046BDE8F08768783E280CD1B8F1030FEE
:109A180002D12E4A4346E9E7EB78012B01D00A2B05
:109A280046D1032704E06BF0DDFB0746F8073FD576
:109A380004F10C0601213046D4F814A06AF0E7F8C6
:109A4800022130466AF0EBF8814600783E2807D1BB
:109A5800E3681B78012B01D00A2B06D1032614E0FA
:109A68006BF0C0FBC10706460FD441F28A13184AAF
:109A78001849194868F0D6FB002383F31188BFF30F
:109A88006F8F0323184602DF0226144A0623214655
:109A980099F800006BF0F1FBB2070DD56369A5EBEF
:109AA8000A0513FA85F5E560A4F81080BB07A4D56C
:109AB8002046FFF737FEA0E72046FCF761FAF5E7F6
:109AC800D95C0A00786B0900335C0A004F5C0A0015
:109AD8006F5C0A00A35C0A00BC5C0A00E87309001A
:109AE80010B5012104460C306AF099F82146BDE80A
:109AF80010400223014A00786BF0BFBB18740900BC
:109B080073B53E4869F0D8FF0446002873D000F1C9
:109B18000C0528466AF08BF80228034603D004286F
:109B280047D0374A03E0238A032B05D8354A012159
:109B380035486BF081FB13E0042128466AF06FF882
:109B4800FF23428806882376238AC6F30B009A42AD
:109B5800608309D0012100922B482C4A69F004FC4B
:109B68002046FCF70DFA12E00F2103F0D5FC05465C
:109B780010B9638B264ADAE703F002FD2146207606
:109B8800320B284603F0DEFA284603F05FFB214B30
:109B9800D3F804317BB32049204870F02FFF031E0F
:109BA80029DA01211E4A184802B0BDE870406BF05E
:109BB80043BB284602216AF032F8054600783E2861
:109BC80012D06BF00FFB10F002060DD140F6BC432B
:109BD800144A1549154868F025FB86F31188BFF328
:109BE8006F8F0323184602DF06232146104A287880
:109BF8006BF043FBB4E702B070BD00BF84020020E5
:109C0800825D0A00ED5C0A00786B09000E5D0A00AF
:109C1800325D0A00800100207C080020A02E002070
:109C28003E5B0A006F5C0A00545D0A00BC5C0A00D7
:109C38002874090010B5012104460C3069F0EFFFC3
:109C48002146BDE810400D23014A00786BF015BB92
:109C580058740900F8B50121044600AF0C3069F0CA
:109C6800DEFF0678002321463046114AFFF77CFEC6
:109C78005F301AD1258AE0682946FFF74FF96C460C
:109C88008AB06A460B4BCDE90750CDE9053640F25C
:109C98000243ADF82430084B42F8103F00234FF43C
:109CA80032510648FAF77CFAA546BD46F8BD00BF12
:109CB800C0740900965D0A0005000001786B090070
:109CC8002DE9F74F0023804689461746DFF810A193
:109CD800DAE8EF4FCAE8E23F002AF9D1264644B94C
:109CE800012143463A4A3B4803B0BDE8F04F6BF0C8
:109CF800A3BA2046FCF7A4F84FF00C0B364D0BFB2B
:109D08000050438843451BD02046FCF799F80BFBCD
:109D18000050438801210093304A43462D4869F09A
:109D280023FBDAE8EF3FCAE8E26F002AF9D1002BFB
:109D38004BD01E46304603B0BDE8F04FFCF720B9C3
:109D4800A74208D0204669F086FE3A8AF96804F1ED
:109D58000C0069F01DFF2046FCF772F80C2707FB82
:109D680000504368ABB1B9F1000F12D12046FCF79F
:109D780067F8012107FB00504268536803F01F0091
:109D8800814010685B0900EB8300137ACBB16BF05C
:109D980048FA2046FCF754F80C2707FB0050836864
:109DA800002BC7D02046FCF74BF8784305F8009005
:109DB8002046FCF745F807FB0055A86828F0D0FCBA
:109DC800B8E7C9436BF03FFAE3E703B0BDE8F08FAB
:109DD800C85D0A00786B090004620020F05D0A0083
:109DE8008002002073B5C5680121B5F801603046CE
:109DF80003F092FB044640B9012133463D4A3E48F0
:109E080002B0BDE870406BF017BA2B78061D1A2B0C
:109E180019D1C378012B50D14FF4804130466BF0F3
:109E280000FA42040FD4D4F88C3069460093D4F871
:109E380094302046019304F0EBFB204602B0BDE8C5
:109E4800704003F003BA2B78BBBB40F2E242B5F88E
:109E580003302A495343C4F88830B5F80520A4F8DC
:109E68009020B5F80720A4F89220A3F5EA520C3AFE
:109E78008A4204D90221224A1F486BF0DDF9B4F85E
:109E88009030B3F5FA7F04D302211E4A1A486BF0CA
:109E9800D3F940F67641B4F89230A3F10A0292B2AF
:109EA8008A4204D90221184A13486BF0C5F96FF4A5
:109EB800805130466BF0C7F914E030466BF0A5F9D5
:109EC800C304F4D52B78202BF1D194F89830002BCB
:109ED800EDD0013B84F898300C4A002304F140008F
:109EE80028F0DCFE2B78002BA7D1204603F01EFDBE
:109EF800A3E700BFF85A0A00786B090095F03C0008
:109F0800235E0A004A5E0A00715E0A005A62020075
:109F180010B5C1E900239DF808300C460B72FBF719
:109F28008FFF0C22024B02FB00335C6010BD00BFA8
:109F380004620020F8B502460B46104869F090FD0F
:109F48000446C0B104210C3069F011FE2046FBF72D
:109F580077FF0C2700260A4D07FB00504680204655
:109F6800FBF76EFF07FB005086602046FBF768FF93
:109F780007FB00556E602046F8BD00BFD81F0020C3
:109F8800046200200138C0B202289ABF014B185C55
:109F98000020704725CA0A0037B50C468DF807001F
:109FA80000F0FF05A0B929B1072220460A498CF024
:109FB80079F840B9002009490DF107020AF004FABE
:109FC800002003B030BD21462846FFF7A7FAF7E77F
:109FD8006FF01500F5E700BFA7C90A004552070052
:109FE80029289ABF014B185C09207047FBC90A0051
:109FF80070B5C3680F21B3F801601D78304603F0CF
:10A008008BFA044638B901213346BDE87040184A36
:10A0180018486BF011B965B12846FFF7E1FF2946EA
:10A028000246204603F03AFD2046BDE8704003F0A2
:10A038000DB98378012B07D10AF076F820466BF02A
:10A04800B9F8002808BF05252846FFF7C9FF2946A3
:10A058000246204603F022FD002DE5D00121064AE4
:10A0680004486BF0D5F8052120466BF012FDDBE7BC
:10A07800AC5A0A00786B09009D5E0A002DE9F04190
:10A08800C6680F21B6F801703578384603F044FAEF
:10A09800044638B901213B46BDE8F0411E4A1F4835
:10A0A8006BF0CAB865B12846FFF79AFF2946024601
:10A0B800204603F0F3FC2046BDE8F04103F0C6B8A3
:10A0C800F278C37A934205D10221154A13486BF0FE
:10A0D800B3F8F0E78378C272012B08D10AB10AF00D
:10A0E80023F820466BF066F8002808BF05252846A7
:10A0F800FFF776FF29460246204603F0CFFC002DE5
:10A10800D9D00121074A05486BF082F8052120467D
:10A118006BF0BFFCCFE700BFAC5A0A00786B0900B0
:10A12800C35E0A009D5E0A00034B0146D3F8240172
:10A1380082689268104700BF8001002008B504219A
:10A1480003486BF06EF8BDE8084002F071B900BF33
:10A158000802002008B503486BF057F8C0F38000E8
:10A1680008BD00BF0802002038B50546F7F740F8DB
:10A178001C2804461BD829460E48F7F727F8A0B133
:10A18800224629460B488BF05FFF00220A482146E9
:10A19800031900F5947083F82821FFF7B1F820B16E
:10A1A8000221064A06486BF033F8002038BD6FF0EC
:10A1B8000B00FBE7A802002080010020F25E0A00E5
:10A1C800786B090000487047A8020020014BB3F8DB
:10A1D800460170478001002037B50F4DADF80600E5
:10A1E800B5F84631834203D10024204603B030BD80
:10A1F80002210DF10600FFF791F8044630B1012164
:10A208000346064A06486BF017F8EEE7BDF8063035
:10A21800A5F84631E8E700BF80010020075F0A0083
:10A22800786B09000149024870F0E8BB6C0800200F
:10A23800A02D002070B505460C4639B1CB684A6997
:10A248009B1A032B0ED86FF0150509E04FF0FF306D
:10A258004FF0FF31FFF76EFE044618B96FF068053E
:10A26800284670BD2046FBF7EBFD0C22164BA618BE
:10A2780002FB0033032130465D8069F0B7FC05809E
:10A28800238A0121033B8370304669F0B7FC40F60E
:10A2980035439D420FD12046FFF746FF054600286B
:10A2A800DED001210346094A09486AF0C5FF204665
:10A2B800FBF766FED4E72146064870F091FA0025C0
:10A2C800FFF7B0FFCCE700BF04620020385F0A0048
:10A2D800786B09008C0200202DE9F04786B0804693
:10A2E80091460C4600AF71B94FF0FF304FF0FF3187
:10A2F800FFF720FE044660B96FF068052846183756
:10A30800BD46BDE8F087887AFBF792FD3C4B834257
:10A318006FD101220021384670F099FA2046FBF7E8
:10A328008FFD0C23DFF800A103FB00A08760204607
:10A3380069F0D8FB01464046FFF77CFF054618B197
:10A348002046FBF71DFED9E7002338462D4A28F0A2
:10A3580043FA064690B140F2E3132B4A2B492C48A6
:10A3680067F060FF324641462A4867F05BFF85F395
:10A378001188BFF36F8F0323184602DF2046FBF7CF
:10A388005FFD0C2358431AF8006066B36D468AB027
:10A398006A46214B0796CDE90538204B089340F2D1
:10A3A8000243ADF824301E4B42F8103F00234FF40F
:10A3B80032511C48F9F7F4FE2046AD46093EFBF73A
:10A3C800DFFD092E0CD8DFE806F0050B0B08170B8C
:10A3D8000B0B0B146FF06E0590E76FF00C058DE713
:10A3E8006FF004058AE7B9F1000FA9D0C9F8004059
:10A3F80084E76FF0150581E76FF00B057EE700BF76
:10A40800D81F0020B4C404006F5C0A005A5F0A0019
:10A41800BC5C0A00635F0A00A85F0A0007890A009B
:10A4280005000001786B09000462002073B5064638
:10A438000D4642F22F00002101AAFFF74DFF044606
:10A4480038B10121144A15486AF0E2FE204602B0EC
:10A4580070BD0198C368B3F801203280B3F80330A7
:10A468002B80FBF78DFD3388A3F11B02E02A04D96A
:10A4780002210B4A09486AF0DFFE44F248112B8892
:10A48800A3F5A47292B28A42E0D90221054A034890
:10A498006AF0D2FEDAE700BFC75F0A00786B0900EE
:10A4A800E75F0A000C600A002DE9F04385B0044616
:10A4B8000DF10301002001F029F8054600287CD1A0
:10A4C8004FF0FF304FF0FF31FFF734FD074600280B
:10A4D80077D000F10C080A21404669F053FB064684
:10A4E800056045600581384D023095F8DA3095F8F9
:10A4F800DB209A4294BF04F1700104F17E016AF0F6
:10A5080089FE9DF803307370AB6813F002091DD102
:10A51800012310214046737269F034FBAA89028036
:10A52800EA894280B4F88C208280B4F88E20C280F8
:10A53800B4F890200281B4F8922080F80C904281FF
:10A5480080F80D9080F80E9080F80F90AB68DB07CC
:10A558001CD5737A102143F004034046737269F0E6
:10A5680011FB2A8A02806A8A4280B4F88C20828091
:10A57800B4F88E20C280B4F890200281B4F89220FA
:10A5880042810022027342738273C2730F4B3846B2
:10A5980001930723029301238DF80C30FBF750FC3D
:10A5A8000C220B4B394602FB003301AA5A6042F2D7
:10A5B80043000022FFF790FE0546284605B0BDE897
:10A5C800F0836FF06805F8E780010020080200209A
:10A5D800046200203C2870B5054644D002283ED1CC
:10A5E80000210246084603F047FB044680B90121D2
:10A5F8001D4A1E486AF00CFE032001F063FF034663
:10A6080088B3BDE870400221194A18486AF014BEA0
:10A6180004306AF0FAFDC30707D50321204602F08B
:10A6280061FE204602F012FEE6E704F1400070F0F9
:10A6380023FA10F00C0607D10E4A29460B486AF097
:10A64800E7FD31462573E9E72046FFF72DFF00288F
:10A65800E7D00121084A05486AF0DAFDE1E7BDE8DC
:10A668007040FFF761B970BD2F600A00786B090070
:10A67800D25A0A004D600A0073600A0030B54FF0E4
:10A68800FF304FF0FF3185B0FFF754FC0446B0B1FE
:10A698000C4B0025019307238DF80C500293FBF710
:10A6A800CFFB0C22084B214602FB003301AA5A605B
:10A6B80042F20E002A46FFF70FFE05B030BD6FF0DC
:10A6C8006800FAE708020020046200202DE9F0473C
:10A6D8008CB0764AB0F8018005460023104600AFDA
:10A6E80048F4704132F8024BA14258D1002220F8B8
:10A6F80013206F4A12F8039000F07CFDEB782E1DB2
:10A70800012B08BF6B4B304614BF002493F822403E
:10A718006AF0F0FC3146002847D007F108006AF0DB
:10A72800DEFCD5F81130C7F80130B5F81530A7F8B8
:10A73800053001233B70E878002843D1022207F155
:10A74800080103F099FA0446EB7823B96FF0800109
:10A7580059486AF078FD002C49D107F110053146B7
:10A768002846FEF78FFB6E4688B06A46534BCDE904
:10A7780005354FF40073ADF81C30514B42F8103FCB
:10A788004FF4E2514F482346F9F70AFD1321B54625
:10A7980040466AF0ADFD3037BD46BDE8F08701336D
:10A7A800052B9FD14FF00009A6E720466AF03CFF31
:10A7B800014607F108006AF02DFD314638466AF077
:10A7C80029FDB8E7012810D1DFF8E8A006229AF899
:10A7D800220007F1080103F04FFA04460028B3D11C
:10A7E800052239499AF82200ABE70024ACE7204655
:10A7F80040F2E242B5F8013007F1080120F8703B59
:10A808006AF008FDB5F817305343C4F88830B5F836
:10A818001930A4F89030B5F81B30A4F89230002312
:10A82800EA782373012AE2702ED1394604F17700C1
:10A838006AF0F0FCD5F80B30C4F87F30B5F80F306B
:10A8480084F87E20A4F883300721204602F04AFDD0
:10A85800B9F1000F05D00121204684F80C9002F0D0
:10A8680041FD204602F0C8FEE3784BB9032001F011
:10A8780029FE034620B10221144A12486AF0DCFC82
:10A88800204602F0E3FC86E7002ADDD1394604F1D0
:10A898007E006AF0BFFC217A064BC1EBC101194466
:10A8A80004F177006AF0B6FCCEE700BF84CB002045
:10A8B80098CE002080010020080200208F600A0046
:10A8C80003000001786B0900A0C90A00D25A0A00E7
:10A8D80000B5C16889B0087820B109B05DF804EB0B
:10A8E800FFF778BEB1F801308DF80000ADF80130FF
:10A8F800CB7801A88DF80330B1F80B300431ADF8EE
:10A908001730B1F80930ADF81930B1F80B30ADF89F
:10A918001B304B7B8DF81D306AF07CFC084B684679
:10A928001A689B88CDF80B20ADF80F30CDF81120B0
:10A93800ADF81530FFF7CAFE09B05DF804FB00BF9B
:10A94800B4C90A0010B5F6F7BBFD034B1B6813B179
:10A95800BDE81040184710BD286200202DE9F341DA
:10A96800344D0646D5F824016FF03EFD50B901215B
:10A97800314A32486AF04CFC6FF01204204602B0AB
:10A98800BDE8F0816FF0020105F188006AF05BFC18
:10A9980001216AF046FCC30748D4FEF7DFFB0446F2
:10A9A8000028EBD1264B1E60012205F1E800114674
:10A9B8006FF04DFF234F05F586706FF0D3FE3846D4
:10A9C80070F047F838466FF007034FF400621E49ED
:10A9D800009428F0F9F8D7F8E0001C4970F09EF8C8
:10A9E800D5F824010769D7F80080B8F1000F15D110
:10A9F800174B3B6083681B689847044628B986B99B
:10AA080002B0BDE8F041F6F75BBDC7F80080012150
:10AA18002346104A09486AF00FFCAFE76FF0770445
:10AA2800F5E705F1780028F0C9F8A7E76FF0770493
:10AA3800A4E700BF800100200B620A00786B0900C0
:10AA480028620020A02E002070F1002023620A0056
:10AA5800C19900002C620A00F0B5C56801212F8851
:10AA680087B0BCB2204602F057FD064640B9012126
:10AA78002346274A274807B0BDE8F0406AF0DCBB08
:10AA880002ACD5F80220D5F8063001946989009106
:10AA98006CF0DCFE48B34FF0FF304FF0FF31FFF7AA
:10AAA80049FA054648B901211B4A1A486AF0B0FB21
:10AAB800304602F0CBFB07B0F0BD12210C3069F034
:10AAC80061F80346224623F8027B144603CC5960FA
:10AAD80006A98C421860224603F10803F5D12946DD
:10AAE80042F21A00FFF7A6FBE2E74FF0FF304FF003
:10AAF800FF31FFF71FFA04460028D4D002210C309A
:10AB080069F040F82146078042F21B00EAE700BFDF
:10AB1800F85A0A00786B090048620A0073B5C368DE
:10AB2800D9789A781E8842EA0122ADF8002059792E
:10AB38001A79B4B242EA0122ADF80220D9799A7999
:10AB4800204642EA0122ADF804201A7A5B7A0121F4
:10AB580042EA0323ADF8063002F0DEFC054658B998
:10AB680001211D4823461D4A6AF066FB0221204642
:10AB78006AF045FC02B070BD694602F023FF38B99F
:10AB88001E2120466AF03BFC284602F05FFBF1E7F5
:10AB98004FF0FF304FF0FF31FFF7CCF904460028A3
:10ABA800F2D00E210C3068F0EDFF00230680C0F8CB
:10ABB8000A30BDF8003021464380BDF8023083805A
:10ABC800BDF80430C380BDF80630038142F220008E
:10ABD800FFF730FBD8E700BF786B0900F85A0A0086
:10ABE80038B5042104460C3069F019F8034640884A
:10ABF8005D7818B122461978FFF762F835B1044834
:10AC080027F0AEFDBDE83840FFF70CBB38BD00BFEC
:10AC180068020020B0B50446032100AF0C3068F08C
:10AC2800FEFFE2680346117840F63542B0F80100AD
:10AC3800904217D16C468AB06A46114BCDE905316E
:10AC4800104B079340F20133ADF820300E4B42F819
:10AC5800103F00234FF412510C48F9F7A1FAA5460A
:10AC6800BD46B0BD1D7810B12246FFF729F8002D6A
:10AC7800F6D0074827F074FDFFF7D4FAF0E700BFD5
:10AC88005F620A0007890A0004000001786B090066
:10AC98006802002038B528F0E5FB314DD5F80C31B5
:10ACA800002B5AD00022002305F1E80027F094FD7C
:10ACB800002852D10022002305F5867027F01AFDDE
:10ACC800044668B940F6CC43264A2749274867F026
:10ACD800A9FA84F31188BFF36F8F0323184602DFA4
:10ACE800D5F800317BB1224A012122486AF090FA56
:10ACF8000022214BD3E8EF0FC3E8E12F0029F9D157
:10AD080008B1FBF73DF9204668F0ECFEC5F80001F4
:10AD18002046FFF709FA0346C8B10121174A15482A
:10AD28006AF08AFA164827F01BFD2046FBF788F8D8
:10AD38000C22144B02FB0033588818B122461F21FD
:10AD4800FEF7BEFF2046FBF71BF9FFF76BFAFFF78C
:10AD580069FABDE8384028F099BB02F05DFCF8E7D5
:10AD6800800100206F5C0A00785A0A00BC5C0A0067
:10AD780097620A00786B090080020020385F0A0099
:10AD8800680200200462002070B54FF0FF320D46C3
:10AD98004FF0FF3300210646FEF796FB044660B9E4
:10ADA8001A230A4A0A490B4867F03CFA84F31188C7
:10ADB800BFF36F8F0323184602DF022104F10C0052
:10ADC80068F0E0FE06704570204670BDFB620A0020
:10ADD800785A0A00BC5C0A00F8B506460024094DFA
:10ADE800EF79E3B29F4202D86FF0010007E02946ED
:10ADF80030466AF04EFB0735631C08B12046F8BDA3
:10AE08001C46EEE78001002037B504460D46B9B16F
:10AE1800284616496AF03DFB90B929461448C4EB08
:10AE2800C40420446AF02EFB12486AF028FB43074A
:10AE380003D5FEF781FA6AF0F5F8002003B030BDBB
:10AE480068466AF03EF90028F8D16846FFF7C4FF63
:10AE58000028F5DA064BC4EBC400694618446AF0CA
:10AE680011FB002DE0D001462846DBE7A7C90A0000
:10AE7800800100200802002070B5174E06223146D6
:10AE880005468BF00FF910B34FF0FF304FF0FF314C
:10AE9800FFF750F80446E0B1062229460C3068F066
:10AEA80077FE2146002242F20500FFF715FA044614
:10AEB80048B110F10D0F04D10221084A08486AF080
:10AEC800F0FA204670BD28683060AB88B380002453
:10AED800F7E76FF06804F4E79C01002031630A008B
:10AEE800886B0900064BD3E8EFCF4CF4806CC3E8BD
:10AEF800E2CF002AF7D1037A19430172704700BFE5
:10AF0800080200202DE9F3410021044602220846E8
:10AF180002F0B2FE054648B120460121FFF7E2FFE4
:10AF2800284602B0BDE8F04102F090B98DF8000063
:10AF380069464E4800F0ACFE9DF8003033B101215F
:10AF48002046FFF7CFFF02B0BDE8F08148486AF01D
:10AF580096FA8106C0F3401708D545486AF08FFA7B
:10AF6800420603D501212046FFF7BCFF00214148D6
:10AF780000F08EFE17B1002001F070FA3E4D95F8F2
:10AF8800DB309BB100206AF0CBFA78B102213B4A52
:10AF98003B486AF086FA17B1012001F05FFA0021F8
:10AFA800384802B0BDE8F04100F072BE95F8DB20E9
:10AFB80095F8DA309A4218D10221334A30486AF0BB
:10AFC80070FA002242F229001146FFF785F910B104
:10AFD80001212E4ADCE795F8DB30013385F8DB30B8
:10AFE800237A43F004032372D5E7224604F10108CB
:10AFF800414612F82E0B6AF056FA064610B1244A5A
:10B0080001210EE095F8DB30013385F8DB30237A37
:10B0180043F00403237295F85B305B0708D40221E0
:10B028001C4A17486AF03DFA01206AF079FAB2E73B
:10B03800414668466AF026FA01234FF0FF304FF088
:10B04800FF318DF80730FEF775FF044660B108221E
:10B0580069460C3068F09CFD3246214642F24E00AB
:10B06800FFF73AF90028DFD00B4AC9E71156070065
:10B0780008020020E15507008001002040630A0013
:10B08800886B09005B55070065630A0096630A0030
:10B09800B6630A00D6630A0000640A002DE9F74384
:10B0A800002104460222084602F0E6FD054648B1A2
:10B0B80020460221FFF716FF284603B0BDE8F043FB
:10B0C80002F0C4B88DF807000DF10701404800F000
:10B0D800DFFD9DF8073033B102212046FFF702FF5C
:10B0E80003B0BDE8F0833B486AF0C9F98206C0F3B3
:10B0F800401808D537486AF0C2F9430603D502213B
:10B108002046FFF7EFFE0021334800F0C1FDB8F1FB
:10B11800000F02D0002001F0A1F900206AF000FA27
:10B128002E4D0646C0B1012103462D4A2D4868F030
:10B1380011F995F8DB3013B101206AF0F1F9B8F193
:10B14800000F02D0012001F089F90021264803B040
:10B15800BDE8F04300F09CBD95F8DB3095F8DA20A7
:10B168009A420CD2013B85F8DB30237A024623F061
:10B17800040302201D49237209F048F9D9E74FF06A
:10B18800FF304FF0FF31FEF7D5FE04F10109074605
:10B1980068B107210C3068F0F5FC49466AF072F98D
:10B1A8003246394642F22800FFF796F828B10121C5
:10B1B8000F4A0C486AF075F9BBE795F8DB30013B9C
:10B1C80085F8DB30237A23F004032372B1E700BF4C
:10B1D8001156070008020020E155070080010020F1
:10B1E8001B640A00886B09005B55070013550700AC
:10B1F80048640A00084BD3E8EF2F22F48061C3E8C3
:10B20800E01F0028F7D1530504D500220220034986
:10B2180009F0FCB8704700BF080200205957070022
:10B22800002307B50549CDE900036A46022009F065
:10B23800EDF8019803B05DF804FB00BF85550700E1
:10B24800034610B470B10B4991F8DA4091F8DB204D
:10B258000CB1944209D2013281F8DB201A7A42F00B
:10B2680004021A725DF8044B70475DF8044BFFF74F
:10B2780049BE00BF80010020034610B4A0B10C4CA9
:10B2880094F8DA1094F8DB2031B101318A4204DCF9
:10B298005DF8044BFFF702BF12B1013A84F8DB20D6
:10B2A8001A7A22F004021A725DF8044B704700BF44
:10B2B8008001002038B50D460649CC7938B12B6895
:10B2C8009C4228BF1C46C4EBC4028AF0BDFE2C6019
:10B2D80038BD00BF8001002070B5044611BB20B303
:10B2E80025496AF0D6F800BB2046FFF775FD00280F
:10B2F8003BDA237853B92148C279002A35D121464F
:10B308006AF0C0F80123C371104670BD012B04D147
:10B31800A37903F0C003C02B07D00121184A1948AC
:10B328006AF0BFF86FF01500EFE7144DEB79012BC9
:10B338001ED005F188006AF0A2F8C30707D4002CD4
:10B34800F0D020460C496AF0A4F80028EAD1EE793A
:10B358002146731C3046EB71FFF756FD08B930469D
:10B36800D3E7EB79013BEB71CFE76FF07700CCE7E0
:10B378006FF00B00C9E700BFA7C90A0080010020D1
:10B388006D640A00886B09002DE9F341044640B951
:10B398001A4A02211A486AF084F8002002B0BDE86F
:10B3A800F081002141F2090001AAFEF795FF054648
:10B3B80008B1144AEDE7019E0622D6F80C8012491E
:10B3C80008F1010738468AF06DFE28B10622384692
:10B3D8000E498AF067FE18B93046FAF7D1FDDCE766
:10B3E800D8F801303046C4F80130BB882570A4F87D
:10B3F8000530FAF7C5FD0120D0E700BF9B640A00BD
:10B40800886B0900B4640A00B4C90A00AEC90A000E
:10B4180007B56846FFF7B8FF044BD87118B16946FD
:10B428000020FFF7F1FC03B05DF804FB8001002069
:10B438002DE9F041304E88B0F179002954D196F8C1
:10B44800764014F0010411D12C4A02212C486AF0EC
:10B4580028F80024F471162500240127F379E0B2B6
:10B4680083422BD8002B3FD000203AE06A464FF6A3
:10B478000940FEF731FF08B1224AE6E7DDF800C0CF
:10B48800DCF80C5095F80180B8F1000F0ED0AB1C19
:10B4980002AA1235174618685968083303C7AB4221
:10B4A8003A46F7D1186838609B88BB806046FAF73F
:10B4B80067FDB8F1000FCDD1134AC6E708AB05FB0D
:10B4C800003353F8182C33F8143C6946CDF80120A2
:10B4D800ADF805308DF80070FFF796FC01340028B0
:10B4E800BCD008B0BDE8F0810021084608B0BDE82E
:10B4F800F041FFF7F1BE00BF80010020D2640A00CE
:10B50800886B0900FE640A001E650A0038B50C46FF
:10B5180061B108480578012D05D10130FFF7ACFC71
:10B5280000B9257038BD00200870FBE76FF01500E2
:10B53800F8E700BF800100202DE9F0411D460E46C6
:10B548001746034648B145B10A0311D54C0708D53B
:10B558000121284A284869F0A4FF6FF01500BDE8CA
:10B56800F0816AF0D2F80028F9D101232B70F6E7B0
:10B57800B107047824D021492FB1B20603D591F838
:10B588009020500632D5C4EBC40411F80480B8F1F9
:10B59800010F09D10134184621446AF051F80028F6
:10B5A800DDD185F8008002E0B8F1000FF9D02FB1A5
:10B5B800B30642BF2B7843F002032B700020CEE77E
:10B5C800720710D50D49C4EBC4040F5D012F07D1D4
:10B5D800013421446AF034F80028C0D12F70E7E71D
:10B5E800002FE5D1FAE76AF090F8BEE76FF0850022
:10B5F800B5E700BF47650A00886B09008001002095
:10B6080070B500F10F0604460D46072230460C4976
:10B618008AF048FD0346207873B90522094902F0EB
:10B628002BFB044658B10573002101F05BFE204650
:10B63800BDE8704001F00ABE06223146EFE770BD52
:10B64800A7C90A00A0C90A00F8B5046906464568F2
:10B6580044B140F203432B4039D005F48263B3F57B
:10B66800806F34D015F4806302D115F4F84F2ED1D1
:10B67800184F3078FB79834229D9C0EBC0000722E4
:10B68800154938448AF00EFDA8B115F0030306D118
:10B6980097F82320082A02D8B2689F2A17D915F0EC
:10B6A800300F09D09CB1EB0608D405F46035B5F528
:10B6B800603018BF0120F8BD002CF6D1D6E902236E
:10B6C8009A4204D81F2A02D9B3F1807FEDD3002013
:10B6D800F1E700BF80010020A7C90A0038B50E4D68
:10B6E80028466AF054F810F0010412D1A5F11803A5
:10B6F8001846582221468AF0CDFC0346D5E8EF2F9C
:10B7080042F00102C5E8E12F0029F7D118465C7024
:10B7180038BD0020FCE700BFB82F0020F8B504466C
:10B7280014F80F7B154B06460D4607222046144990
:10B7380083F822708AF0B6FC70B93846114902F0D5
:10B74800E3F9044610B96FF00B00F8BD052101F0CC
:10B75800C9FD00202C60F8E72146384602F024FA9B
:10B7680040B92146307802F0CFF904460028EAD0E3
:10B778000621ECE76FF01500E7E700BF8001002025
:10B78800A7C90A00A0C90A002DE9F04F91B01546D3
:10B7980003905068002214460691824212D1FB2C75
:10B7A80018D89F4BB3F8D8309C421ED99D480093B7
:10B7B800022123469C4A67F0D7FD6FF0200011B0A4
:10B7C800BDE8F08F2968023401EBC2014B780132E1
:10B7D8001C44E2E7039B082103F1180069F0DAFF33
:10B7E8000028DED06FF00A00E9E7FB2C6ED8039B37
:10B7F8000B2103F1180069F0CDFF10B91F2C28BFE9
:10B808001F244FF0FF304FF0FF31FEF793FB04F198
:10B8180004080746002800F0FF8041460C3068F015
:10B82800B1F94FF000090646424600218AF032FC81
:10B838004946D5F8008006F1040B6B6899450FD38B
:10B84800039BF1705B7800223370032339467370D1
:10B8580001230698B37011B0BDE8F04FFEF73CBD68
:10B8680098F80120881C13189C4298F800C013D23D
:10B87800BCF1090FA4EB000201D1002A0ADC6948D7
:10B8880001216A4A67F05DFD3846FAF779FB6FF0E7
:10B89800150094E74FF0080C5FFA82FA0AF10103E9
:10B8A8000BF801300131C9B20BF801C0C3B2D8F8A6
:10B8B8000410584404938AF0C7FB049B09F101095A
:10B8C8009A445FFA8AF108F10808B6E700211022C5
:10B8D8000CA88AF0DFFB0027012340F272600B936B
:10B8E8003B4669680A958B4207D100240123A0468C
:10B8F800A34605935FB9384661E72A68023702EB29
:10B90800C302527817448742C1D80133EBE7FB2FB3
:10B918004FF0FF304FF0FF31BA4628BF4FF0FB0A17
:10B92800FEF708FB0AF104060490002874D031469B
:10B938000C3068F027F9039B81465B78002603707A
:10B948004FF000035FFA8AF283700792031D55F8DF
:10B958003B2005EBCB0102EBC8025278023294423D
:10B9680009D14A6808F10108904509BF002400245C
:10B97800A0460BF1010BBBF1010F12D055F83B208B
:10B988004FEAC80112EBC80C0BD09819FCB9012476
:10B998009CF8012001329A550136F6B2079AB24254
:10B9A800D5D8059BBF1B002B31D0002F0CBF03231C
:10B9B800012300220499069889F8036089F8013068
:10B9C800FEF78AFC00287FF4FAAE059092E7012C76
:10B9D80005D1525C013602240270F6B2DEE79CF80B
:10B9E8000120AAEB0601121B02328A4228BF0A462E
:10B9F800DCF804C0A11E6144099308928AF024FB74
:10BA0800089A099B14443244A4B2D6B2C6E7B7FADE
:10BA180087F35B095B00CCE76FF06800CFE600BFF7
:10BA280080010020106B09006C650A009A650A0005
:10BA38002DE9F3470F690D46496890463A1E18BF2D
:10BA480001224C020646016505D5EB787F33DBB24F
:10BA5800932B00F2048130460DF10303FFF76CFDD0
:10BA68000446002840F0E88006F10F03002F00F09C
:10BA7800E7802A6911684FF0FF30C6F80F109188E7
:10BA8800998092794FF0FF319A71FEF753FA814607
:10BA9800002800F0E78019210C3068F073F804469C
:10BAA800002119228AF0F6FA73782370AB68E370E4
:10BAB800C3F307221B0C22716371EB68A371C3F3F4
:10BAC80007221B0C2372E2716A6812F4004F14BF3C
:10BAD80006230723D00348BF03F00503910348BF9B
:10BAE80003F0FB0363729DF80330A3726B685A027C
:10BAF80054BF7F2395F90330E374012323756B68E2
:10BB080003F44063B3F5806F14BF01230223A375C8
:10BB18006B68DB0442BF03232375A3756A68C2F30D
:10BB2800802383F001031B0150049BB248BF43F0FC
:10BB38004003910448BF43F02003D20544BF0122CB
:10BB480022766A6890077DD043F0010A1FB9510533
:10BB580001D443F0030A900502D4B8F1000F03D0D2
:10BB68004AF0020A1FFA8AFA002F6DD0D1062A6914
:10BB780048BF4AF00403116858BF4AF00C03C4F8E0
:10BB88000B1091889BB2A4F80F10927962746A78AE
:10BB980001AFE275AA7849466275A4F801303A46C1
:10BBA80042F23600FEF798FB0446002844D1019B78
:10BBB800DB6893F90130B370D7E8EF0FC7E8E34FBC
:10BBC800002BF9D108B1FAF7DBF906F11807D7E825
:10BBD800EF3F43F00203C7E8E23F002AF7D16FF0D6
:10BBE8001001384669F0DDFDC2062FD46A680921C4
:10BBF80012F0030218BF0122384669F0DDFD0A2160
:10BC08003846CAF3400269F0D7FD2A790C21384634
:10BC1800C2F3800269F0D0FD6A790B213846C2F37D
:10BC2800800269F0C9FD9DF803200321531E5A4282
:10BC380038465A4169F0C0FD204602B0BDE8F08799
:10BC48000A4A17E79A4686E75346A0E7304606F1C0
:10BC5800090169F0F5FC0028C8D00446ECE76FF04C
:10BC68001504E9E76FF06804E6E700BFA7C90A0012
:10BC780008B520B9044869F08AFDC30701D400203B
:10BC880008BD0248FCE700BFB82F0020A02F002005
:10BC9800034610B5044869F07AFDC20703D5BDE82C
:10BCA80010400248184710BDB82F0020A02F0020D0
:10BCB80010B5054CA06930B16FF00101183069F07A
:10BCC80070FD0023A36110BD8001002010B5164B44
:10BCD8009C693CB90121154A154867F032FB0024DC
:10BCE800204610BD204669F0EDFD04F11802082138
:10BCF800104669F04FFD10B9FFF7DAFFEFE70921A9
:10BD0800104669F047FD18B100212046FFF778FC7E
:10BD180000222046114669F090FD04460028DFD134
:10BD2800FFF7C6FFDCE700BF80010020B3650A000B
:10BD3800106B090010B50A4B20389B6983420AD161
:10BD4800FFF7C4FF034648B1BDE810400221054A89
:10BD5800054867F0FFBA69F0B8FDF3E710BD00BF0A
:10BD680080010020EA650A00106B09002DE9F04FF8
:10BD7800DFF888B10646DBF818400F46904699462A
:10BD880085B0002C40F09E80FFF7A8FC0546CBF854
:10BD98001800002800F099800BF18800D6F810A050
:10BDA800ADF808408DF80A40039469F0F0FC4107AB
:10BDB80074D573685A0574D432690AB19B0770D078
:10BDC8003046FFF741FC00286BD005F1180B08211D
:10BDD800584669F0DFFC002866D1434869F0D7FC73
:10BDE800440501D5FFF706FA3378B9F1000218BF08
:10BDF8000122314628462B70FFF71AFE044660B927
:10BE0800BAF1000F0CD10E9B4246009339464B46BF
:10BE1800284669F085FD044680B1FFF749FF33E005
:10BE28007368D8060AD48023ADF80830DBE8EF3F02
:10BE380043F08003CBE8E23F002AF7D17368990703
:10BE480016D10121284602AA69F0F7FC0446B8B1C8
:10BE58000121264A264867F074FA039E002EDCD09A
:10BE68003046002101F03EFA304601F0EFF9D4E700
:10BE7800284603A9FFF752FC04460028E1D0CCE786
:10BE8800039808B101F0E2F93946002340F20110A5
:10BE980098450CD1204605B0BDE8F08F6FF00A0434
:10BEA800BBE76FF01504B8E76FF07704B5E70A88C9
:10BEB800824204D14A6812B11278D20708D40133F9
:10BEC8000831E5E76FF07704E4E76FF00B04E1E78A
:10BED8002035284607496EF0C3FD00232846064A48
:10BEE80026F014FFD6E700BF08020020CF650A003D
:10BEF800106B09003DBD00001C4E0E0080010020A3
:10BF08002DE9F341C6687078FFF7B2FE044638B9E8
:10BF18000121364A364802B0BDE8F04167F011BA4F
:10BF280004F11808758869F0CDFC6FF480714046FB
:10BF380069F037FC33782F4F1BBB2846012101F0ED
:10BF4800EBFA054650BB6FF08001404669F029FCCA
:10BF580003060ED5204669F0F1FBFFF74BF963683D
:10BF68003BB11B682BB1327920468DF8042001A91A
:10BF78009847BB699C4235D102B0BDE8F041FFF754
:10BF880097BE0921404669F005FC18B12046317872
:10BF9800FFF736FB3378002BD5D1CEE7236D00F1C0
:10BFA8007E0213F4002F12D0A368C0F87E30A38954
:10BFB8009380A37B937163682BB15B681BB12046A8
:10BFC800019501A99847284601F040F9BBE7037A93
:10BFD800C3EBC303F918FB58C0F87E308B889380F5
:10BFE8008B79E7E702B0BDE8F08100BF09660A0077
:10BFF800106B0900800100207FB5C5682878FFF71D
:10C0080037FE044638B90121134A144804B0BDE884
:10C01800704067F096B943688BB19B687BB1013576
:10C02800284669F067F802AE294650B1304669F0F3
:10C0380056F8636820469B68019601A9984704B0A2
:10C0480070BD207869F0F0FA0346006802909A887B
:10C058009B79B280B371ECE709660A00106B09009E
:10C06800034B1A7A012A04BF02221A72704700BFD2
:10C078009DCE002008B509486EF000FD031E04DAC5
:10C088000121074A074867F065F90022064B9968BD
:10C098009A801960054B1A7208BD00BFC8020020BB
:10C0A8001D660A00A86B09008C0800209DCE0020A0
:10C0B800F0B505460F464FF0FF304FF0FF3187B01F
:10C0C8001646FDF737FF0446C0B106210C3067F06D
:10C0D80059FD468000264770057006714671094A69
:10C0E800204603A905230095FDF712FF3246214695
:10C0F80042F24200FEF7F0F807B0F0BD6FF06800BA
:10C10800FAE700BF0802002038B50546407A0C4619
:10C11800FDF738FF2073A87AFDF734FF607395F9AF
:10C128000C30A37195F90D306371EB7A2371EB89AB
:10C1380063812B88103BDBB20B2B8EBF0523054A8E
:10C14800D35CE3712B8883F0100303F01F03238172
:10C1580038BD00BF28CA0A0008B50C4B0246400982
:10C1680003EB800069F008FC02F01F0340FA03F3B8
:10C1780013F0010006D122B9054869F0FDFB40F330
:10C18800C01008BD6FF07700FBE700BF2C620020ED
:10C19800080200202DE9F04788B0002200238E48CD
:10C1A80026F0E6F90646002840F0CB808B4869F077
:10C1B800E3FB10F0010F894D7ED02B1D93E807009B
:10C1C80008AB03E90700864869F0D6FBC0F34013C3
:10C1D800824869F0D1FB0446002800F0A3808BB1A7
:10C1E8000C22804905A889F05DFF0446002800F06C
:10C1F800A480002211461046FFF75AFF0446002883
:10C2080040F09B80764869F0B7FB410501D5FEF701
:10C21800F1FF9DF815502A0757BF9DF814300027E5
:10C228008DF80430BDF816305FBF01AFADF80530AA
:10C23800BDF81830ADF8073015F0040500F0C880D7
:10C24800BDF81C200AB9BDF81620BDF81E300BB980
:10C25800BDF818309DF81410ADF80D208DF80C10AD
:10C26800ADF80F3003AD002F6FD03B78012B71D0A4
:10C27800002D6AD10025BDF81A3006F0010043B13F
:10C28800574BD3E8EF1F41F04001C3E8E21F002AF3
:10C29800F7D10DF1030169F06BFA044600284CD17F
:10C2A8004FF0FF304FF0FF31FDF744FE8046002885
:10C2B80052D16FF0680440E0494869F05DFB10F026
:10C2C800800F494A0ED09089D18913694FF4807242
:10C2D800ADF81600ADF81420ADF81810ADF81A60D6
:10C2E800079370E7414C05AB2068616803C3A068F9
:10C2F800186092F8913039481F0744BF05238DF81C
:10C30800153069F039FB840706D53023ADF81830AD
:10C318006023ADF8163056E7304869F02DFB40072A
:10C32800F3D450E74BB102460146FFF7C1FE04467D
:10C3380018B92C4B2861C3E90100274826F08AF96F
:10C348002646304608B0BDE8F0872E78731E5E4258
:10C358005E4190E71E468EE700F10C09032148462E
:10C3680067F010FC9DF803309DF815A00370CAF320
:10C37800400306468470437037B101230522837059
:10C388003946484667F004FC45B1B378052243F0C6
:10C39800040329464846B37067F0FAFB0022414679
:10C3A80042F24100FDF798FF04460028C5D101205C
:10C3B800BDF81A200AF00101FFF77AFE04460028AA
:10C3C800BBD1084B08AA12E9070083E80700B4E7C5
:10C3D800002F7FF44AAF4DE7486200202C6200200E
:10C3E800080200203C62002080010020F06D090056
:10C3F800002347F6122210B5064826F087FC031ED4
:10C4080006DABDE810400121034A044866F0A2BFDD
:10C4180010BD00BFC80200204A660A00A86B0900C8
:10C428000022024B1A60FFF725BE00BF7862002089
:10C4380010B544220021084889F02CFE064B03F170
:10C448001C001C466EF00FF904F130006EF00BF979
:10C45800BDE81040FFF7E4BF2C6200200022044B27
:10C46800801A597C18BF012001F00101FFF720BE96
:10C478002C620020032870B5054603D1BDE8704042
:10C48800FFF788BEFFF768FE0446B0B9012605F03D
:10C498001F039E400A4B6D0903EB8505D5E8EF3F66
:10C4A8003343C5E8E23F002AF8D1FFF773FE04469C
:10C4B80018B1F143284669F062FA204670BD00BF02
:10C4C8002C620020032808B50AD0012100F01F03C0
:10C4D8009940054B4009C94303EB800069F04FFAC6
:10C4E800BDE80840FFF756BE2C6200202DE9F74F43
:10C4F80005465E4869F040FA00F001085B4869F0BB
:10C508003BFA0E46144699468246B8F1000F03D00E
:10C518000B895A0700F1A680284668F0EBFD6F46A4
:10C52800002868D02946684668F0D9FDB8F1000FA0
:10C5380002D11AF0040F28D14D4BD3F800B0BBF14B
:10C54800000F13D02268A368B4F804A0A4F80490DC
:10C55800A2EB030838462346F27996F90510D84726
:10C56800A368A4F804A013FA88F32360414B37604A
:10C578001A6842B152F80889B8F1000F01D0A8F141
:10C588000808002A47D1002333603848338969F006
:10C59800F3F910F0010665D1DB0763D503223946AC
:10C5A800304601F069FB044600285BD00220FFF703
:10C5B80089FF2B682046C4F87E30AB88A4F8823007
:10C5C800AB7984F8843068F091FE002843D01F23AB
:10C5D80031462373204600F085FE204600F036FEE3
:10C5E800FFF7D8FD034600283CD00221224A234801
:10C5F80066F0B0FE36E02B78FF2B07D1204B186889
:10C6080000909A889B79BA80BB718FE7294669F0B8
:10C618000BF80346F3E713688BB12168A368B4F8F5
:10C6280004B0A4F80490A1EB030A3046136821462D
:10C638009847A368A4F804B013FA8AF32360B8F102
:10C64800000F06D0D8F8083003B1083B4246984698
:10C6580097E74346FAE72046022100F043FE2046CA
:10C6680000F0F4FD03B0BDE8F08F00BF2C6200209D
:10C678007862002070620020D25A0A00A86B090074
:10C68800A7C90A0010B50020FFF71CFF58B16EF0CB
:10C6980069FA0020FFF716FF034620B10221124A6B
:10C6A800124866F057FE6FF04001114869F067F9CB
:10C6B8006FF480710E4869F062F9FEF79BFD0D4B2F
:10C6C8001B6823B153F8084904B1083C03B910BDED
:10C6D8005B6803B198472CB1A26802B1083A2346B7
:10C6E8001446F3E72246FAE77B660A00A86B0900BE
:10C6F80008020020706200202DE9F04F00F10C09BB
:10C7080089B00746484667F092FA06465D4869F0E0
:10C7180033F900F001035B48039369F02DF95A4D92
:10C72800C0F38003DFF874A102939EB1039B53B159
:10C738003B8A172B11D80121544A554809B0BDE846
:10C74800F04F66F0FEBD2B7A0BB1FFF793FC029B0E
:10C75800002BEDD109B0BDE8F08F1821484667F0ED
:10C768005EFA3A8AC37DB0F800B09342CBF3411821
:10C7780004460BF0100B0FD9454800920221454A98
:10C7880066F0F2FD384667F066F9BBF1000FE1D1BB
:10C7980002223D4B1A72DDE7BBF1000F0DD004A950
:10C7A800FFF7B2FC4A46E37D04A9A01CFFF79EFEF2
:10C7B8004846E17D67F02BFA29E095F808B0BBF10F
:10C7C800000F37D0C27AEB799A4205D1811C072233
:10C7D800284689F067FC48B3B8F1000F02D120461B
:10C7E80004A9DDE7BBF1010F27D102212A4A284815
:10C7F80066F0A7FDDCE72B7A022B3DD05046F9689E
:10C8080067F0C6F9B8F1010F04D1FFF7F1FD013E59
:10C81800F6B28AE7204604A9FFF776FC5246BAF832
:10C82800043004A9A01CFFF761FE28E0B8F1020F4C
:10C8380018D124E0B8F1000FD1D0B8F1020F1ED002
:10C84800BBF1020F01D1FFF715FCD4F80220E37AFF
:10C858002A60E288EB710123AA80227A2B72AA71DE
:10C86800FFF7C6FDE27DBAF80430BAF806101344A3
:10C878008B42C0DD02232B72B8F1010F98D0FFF76D
:10C88800F9FB95E72C6200209DCE0020A4660A00E3
:10C89800A86B0900BD660A00E7660A008C0800203C
:10C8A8002DE9F04F00F10C0785B00646384667F0D1
:10C8B800BEF905462A4869F05FF800F001092848E2
:10C8C80069F05AF84FF0010ADFF8A0B0C0F3800809
:10C8D80015B905B0BDE8F08FB9F1000F02D1B8F174
:10C8E800000FF6D0338A082B07D801211D4A1E48AD
:10C8F80005B0BDE8F04F66F024BD0921384667F061
:10C908008EF9037A328A01339A420446EDD37F23A3
:10C91800ADF80CA08DF80630037A694603445B7ABB
:10C9280001308DF80530FF238DF804300023ADF871
:10C938000A3010F8012C013D042A98BF1BF8023078
:10C948008DF80720ADF80830C3793A46FFF7CEFDD9
:10C95800217A3846013167F05AF9EDB2B8E700BFDD
:10C968002C620020A4660A00A86B090034CA0A00D9
:10C97800F8B50546224868F0FFFF43070F463CD547
:10C988002A78012A03D96FF015042046F8BD6B7880
:10C998000F2BF8D843F6FC746888031F9BB2A34298
:10C9A800F1D8A9880B1F9BB2A342ECD88842EAD3DE
:10C9B8007AB900220023134825F0DAFD044600283E
:10C9C800E3D1FFF7C9FB044640B10E4825F042FE0B
:10C9D800DBE768F0B1FE0028EBD1D4E72868696886
:10C9E800094E0A4B03C6A8681F6030602046FFF74F
:10C9F80041FD044606F12400E8E76FF00A04C4E7A5
:10CA0800080200205C62002030620020786200206A
:10CA180008B5FFF705FD00220A4B6FF040010A48F0
:10CA28001A6068F0ACFF430606D56FF480710648BB
:10CA380068F0A5FFFEF7DEFBBDE808400020FFF721
:10CA480041BD00BF78620020080200200A4A00F1B8
:10CA58000803116831B98160516839B9C2E90033F6
:10CA6800002070478B4204D00968F3E70B605360DD
:10CA7800F6E76FF0100070477062002008B50348B1
:10CA880068F07AFF00F0010008BD00BF2C620020AA
:10CA980070B59AB01422002104A889F0FBFA47F275
:10CAA8001213ADF80C304FF4807344F20102ADF864
:10CAB8000E30364B01A903A8CDE905235EF0FAFC38
:10CAC800034618B3324A0121324866F043FC1F2559
:10CAD800314BD3E8EF1F21F00101C3E8E21F002A20
:10CAE800F7D12E4E26F0BEFC346804B1043C002D6C
:10CAF8002B4D18BF0025002C41D023680BB12846C8
:10CB080098476468002C3AD0043CF6E702AB41220F
:10CB1800019809A988F054F9034608B1214AD2E7D7
:10CB2800214A0DF125030DF1650153F8040B8B42E1
:10CB380042F8040BF9D102AB20221C49019888F075
:10CB4800E7F8034608B11A4ABDE7019888F098F853
:10CB5800054610B1174A0346B5E71349104868F06F
:10CB680019FF1548203168F015FF144BD3E8EF1F63
:10CB780041F01001C3E8E21F002AA9D0F6E700231C
:10CB8800C6E9003326F082FC1AB070BD0000020925
:10CB98000C680A00686B09007C620020846200202F
:10CBA800EBCF00202A680A00ABCF00208BCF0020F3
:10CBB8004D680A0071680A000BD0002008020020A6
:10CBC80030B5A7B01422002108A889F063FA04231D
:10CBD8003D22002116A8159389F05CFA47F212133A
:10CBE800ADF81C304FF4807344F20102ADF81E30EA
:10CBF800284B2949CDE9092307A805AB202288F04D
:10CC080009F90346E0B1254A0121254866F0A2FB4F
:10CC18006FF0040426F026FC224B1D6865B1002045
:10CC28001860214BD3E8EF1F21F00201C3E8E21F8F
:10CC3800002AF7D144B3A84726F028FC27B030BD16
:10CC48001A4B0DF15502194603F1400053F8044BF5
:10CC5800834242F8044BF9D106AB029320230D48D6
:10CC6800CDE9001315AA4123059988F0A6FA0346D1
:10CC780008B10F4AC8E7059888F002F8044600286A
:10CC8800C8D00C4A0346BFE70DA8084968F082FEE1
:10CC98000DA8D0E7000002098BCF002091680A0098
:10CCA800686B0900806200207C620020ABCF002006
:10CCB800C7680A00E3680A00402208B5034989F0FA
:10CCC800F1F9B0FA80F0400908BD00BF39CA0A007E
:10CCD80010B598B004461422002102A889F0DAF9A8
:10CCE80044F21213ADF804304FF480734FF48042CD
:10CCF800ADF80630144B2146CDE9032304230DF18A
:10CD08001D008DF81C3068F045FE04F120010DF17E
:10CD18003D0068F03FFE6B46412207A901A888F054
:10CD280079F8044601A888F06EFB2CB9009887F0C2
:10CD3800A7FF012018B010BD044823460121044A6A
:10CD480066F008FB0020F5E700000209686B09009F
:10CD580000690A0010B5002834D01D4A136823B1B1
:10CD6800043B984231D05B68F9E71A4BD3E8AF1F10
:10CD7800890707D518480221184A66F0E2FA6FF0C9
:10CD88000F0010BD1468011D44605068116000B99F
:10CD98005160D3E8EF2F42F00101C3E8E01F0028FB
:10CDA800F7D1D30701D50020EBE70D4BD3E8EF1FF0
:10CDB80021F01001C3E8E21F002AF7D10948FCF767
:10CDC800F7F8F0E76FF01500DBE76FF07700D8E7CA
:10CDD800846200207C620020686B090024690A00D4
:10CDE80008020020A8080020044BD3E8AF3F13F046
:10CDF800100F034808BF0020704700BF080200203A
:10CE0800EBCF002070B50546194803688B4228D03F
:10CE1800184BD3E8AF3FDA0626D5036813B16FF095
:10CE28000F0070BD144AD2E8AF3FDB07F7D4D2E851
:10CE3800EF3F43F00204C2E8E64F002EF7D113F0AB
:10CE48000204ECD1016029460C4868F0A3FD0C48A7
:10CE580005F1200168F09EFD0A48FCF7A9F8204674
:10CE6800DFE76FF07700DCE76FF07C00D9E700BF01
:10CE780080620020080200207C620020ABCF0020E6
:10CE8800CBCF00209808002070B505460B4B1C68D6
:10CE980044B154F81C3C1C3C13B12846297B9847E4
:10CEA800E469F5E7064C074EB44200D370BD236829
:10CEB80013B12846297B98472034F5E70063002002
:10CEC800C06A0900006B090010B50446F8F7B8FFFE
:10CED800044901EB0011204668F04DF9BDE8104007
:10CEE800FDF7A0B98C620020002270B50446D1E994
:10CEF80001560748C1E901226DF072FC3DB1314687
:10CF080020462B46BDE870406FF06D02184770BD93
:10CF1800E41E002030B5051D04464FF48061284604
:10CF280085B068F061FD400533D4284668F057FDA8
:10CF3800810321D5E17871B3637B072B29D1224B7B
:10CF480093F890309B0624D568F0A5F908B30DF145
:10CF58000E0103A8FDF76AFAD8B92046BDF80E20DD
:10CF6800BDF80C1068F003FA034690B10121174A86
:10CF7800174868F037FD0CE0204668F0DDF90346F5
:10CF880020B10121134A124868F02CFD637B072B5E
:10CF9800D0D005B030BD0C4B93F89130DA0706D4E9
:10CFA800022319460C4A0A4868F01CFDC4E702230C
:10CFB80020461A46009168F0F9F903460028BBD0CC
:10CFC8000121064AEFE700BF80010020A3690A009B
:10CFD800286B090052690A0073690A008C690A0003
:10CFE80070B50546002200230E4825F0F5FBB8B9B8
:10CFF8000D4B1C6834B154F8143C1C3C03B19847E1
:10D00800E469F7E7094C0A4EB44204D32846BDE860
:10D01800704025F0D3BDA36803B198472034F3E7E7
:10D0280070BD00BFC01E002000630020C06A090058
:10D03800006B09002DE9F041044620270025EFF395
:10D04800118287F31288BFF36F8FE16929B1206AD3
:10D058000B688142E36108BF236282F31188BFF342
:10D068006F8F71B1D1E901680748C1E901556DF0C9
:10D07800B7FB1EB1002241462046B047FDF7D2F863
:10D08800DDE7BDE8F08100BFE41E00200348B0F8EA
:10D09800BC30C030002B08BF002070478001002042
:10D0A80030B50446F8F7B6FB0D460D4A0D498BB06E
:10D0B8000858D2F8E010884205D120460BB0BDE8E8
:10D0C8003040FFF7B7BF2434214610466DF096FC78
:10D0D8001DB1694620466DF0A1FC0BB030BD00BF04
:10D0E800104F00200800000038B5002204468A428C
:10D0F80002D10024204638BD012004F1C803D3E83A
:10D10800EF5F002D04D1C3E8EC0FBCF1000FF6D19E
:10D1180002D0D0340244EAE7002CEAD0C822002129
:10D12800204688F0B7FF04F1400004496DF098FCF0
:10D13800034904F124006DF036FCDBE7D5DF00007D
:10D14800135A0700F7B516460D4601210446FFF7A6
:10D15800A7FF012E23D0022E52D123693BB13548B7
:10D168000121354A66F0EDF8204668F06CFC25612F
:10D178002269138A012B5AD9D2681288043292B2D2
:10D18800934254D343D9012100922A482B4A66F08E
:10D19800EBF8204603B0BDE8F04068F054BC2069C5
:10D1A80040B9274A3146234866F0CBF8204668F054
:10D1B8004AFC01E02A8A2AB9284603B0BDE8F040B3
:10D1C800F8F7DEBE018A438A47695B1AC168C91B42
:10D1D8005B1A9A420CD91B4A3146164866F0B1F8D8
:10D1E80000222046216901F0E7F900232361E3E7E3
:10D1F800E9680C3066F0CCFC2846F8F7C1FEB7E7C2
:10D2080001213346104A0B4868F0ECFBCEE70022B8
:10D2180004F11003D3E8EF1FC3E8E02F0028F9D189
:10D228000122204603B0BDE8F04001F0C5B903B0C3
:10D23800F0BD00BF286B0900BF690A003F6A0A00F9
:10D24800DC690A00FA690A00216A0A0008B500F1D7
:10D25800C803D3E8EF2F013AC3E8E12F0029F8D13A
:10D26800AAB90B4B984212D303F5826290420ED2B0
:10D27800C01AD023B0FBF3F203FB120038B90548FB
:10D2880025F06EFABDE80840034825F097BC08BDB4
:10D29800F82F0020C01E0020C808002010B5044642
:10D2A80068F0E0FB26F0DEF80C4B04F1BC01D3F883
:10D2B800DC3043B90A4868F077FB26F0E7F8BDE8A8
:10D2C8001040FCF7AFBF994201D01B68F1E726F088
:10D2D800DDF82046FFF7BAFFF1E700BF8001002024
:10D2E8005C020020F8B5457B04468D420E4600AF2F
:10D2F8001CD1082D98BF694B6C4688B094BF53F871
:10D308002530674B6A466749CDE905134FF400732A
:10D31800ADF81C30644B42F8103F00234FF4E45141
:10D328006248F6F73DFFA546BD46F8BD4173DDB13D
:10D33800022D1CD0637B082B00F2AD8001A252F8AD
:10D3480023F000BFABD3000045D4000015D4000083
:10D3580031D3000031D3000031D3000031D30000B5
:10D3680085D3000031D3000068F07CFBE2E78378C6
:10D37800012BDFD140306DF081FBDBE70023C4E9EE
:10D388000D33E378012BCFD1A378494A012B04BF91
:10D39800032384F89830002304F1400025F07EFC34
:10D3A800C2E7082DC0D8DFE805F02A052117262690
:10D3B800212A2A0004F1400528466DF05FFB01216F
:10D3C8002046FFF76DFE204668F03DFB0022002353
:10D3D800284625F09BFCA7E70220FFF773F80346D1
:10D3E80020B10221334A314868F0FCFA237B13B19B
:10D3F8002046FFF749FD2046FFF728FF94E733460C
:10D408002D4A0221294868F0EDFA8DE7A378012B0F
:10D418008AD12A4B9D8A002D86D00A2340F2E73014
:10D42800002147F612265D434FF47A720023E5FB8C
:10D438000601F3F771FE02460B46ADE7237B3E2B50
:10D448000FD16D4688B06A461D4BCDE905340323DC
:10D4580042F8103F00234FF4C4511448F6F7A0FED9
:10D46800AD46164D05F1C006616911B9FCF7DAFE43
:10D478005AE7A2690B68914208BFA361204663611D
:10D48800FFF732FDB5F8BC30002B14BF3046002042
:10D4980025F066F9E8E70B4A3346B2E7D474090089
:10D4A8005A6A0A00646A0A0003000001286B09002E
:10D4B8005A620200756A0A00A66A0A008001002002
:10D4C800BD6A0A00E46A0A002DE9F04706460F46DD
:10D4D800904600254FF0D009DFF828A009FB05A0E9
:10D4E80068F0C0FA044620B183781E4206D1FFF7DF
:10D4F800ADFE0135052DF1D1BDE8F0874146B847AD
:10D508002046F4E7F82F0020002201200149FFF708
:10D51800DBBF00BF075A07002DE9F04105460E465C
:10D528000027DFF85880404668F09CFA044658B156
:10D53800437B012B02D0073B012B03D82388AB4246
:10D548000BD02046FFF782FE0137052F08F1D008DF
:10D55800E9D100242046BDE8F081A3781E42F9D124
:10D5680002212B46034A044868F03CFA2046FFF79C
:10D578006DFEEEE7006B0A00286B0900F82F00200B
:10D58800034BC01A034B00115843C0B2704700BF89
:10D59800F82F0020C54EECC470B51C461443054650
:10D5A8000E460DD0F8F736F90E49D1F8E0400E498D
:10D5B80009588C4206D102210C4A0D4865F0C1FE7B
:10D5C800002213460B49002D14BF2846084666F072
:10D5D80047FA044618B1711D0C3066F0C8FA2046A7
:10D5E80070BD00BF104F002008000000176B0A0034
:10D5F800286B0900FC1E002010B50446054825F0DC
:10D60800DDFA204600F0D2FE2046BDE81040FFF7C4
:10D618003BBC00BFB80800202DE9F04F002387B0BD
:10D6280000AFFB607B61B94B5A8B3AB1B84DD5F866
:10D63800DC403CB91C37BD46BDE8F08F1B68002BA9
:10D64800F4D1F7E754F8BC3903B1BC3B0026B14923
:10D6580001E01C461346B5F8BC20002A00F05481AE
:10D66800D5F8C8204AB904F1BC06002BE2D0D3F89B
:10D67800BC20002AEDD0BC3AEBE70A68002AF2D0B9
:10D68800D4F8A820002AEED0D4F8AC20002AEAD09A
:10D69800D4F8B020002AE6D0637B072B6AD1204655
:10D6A8009047002866D004F1C00068F098F9022875
:10D6B80060DC204668F0D6F904460028BAD0637BBF
:10D6C800072B40F01E812046D4F8A830B5F8BC10CE
:10D6D80007F1100298478146002800F00581B5F847
:10D6E800BC203B699A4208D30146D4F8AC60204676
:10D6F80007F1140307F10C02B0477B69D7F80C80D7
:10D708003B60B9F81030002B00F0F5804846D7F898
:10D7180010A067F046FD7860002840F0EF80B5F86B
:10D72800BC30DFF800B2002B14BF5846002000229E
:10D73800002325F051F878B900220023754824F019
:10D74800D9FF064600283BD1B5F8BC30002B18BFDE
:10D758005E46304625F004F86FF00B054846F8F7AA
:10D768000FFCB8F1000F00F0AA802A46204639685D
:10D77800C047A4E0D4F8BC3004F1BC02C6B9D5F85F
:10D78800E010C5F8DC308A4201D1C5F8E03000234A
:10D798002046C4F8BC30D4F8B030984700288ED062
:10D7A800637B072B40F0AD802046FFF777FD86E7C7
:10D7B8003360D5F8E0309A4208BFC5F8E060E6E784
:10D7C8003B68C0F804808360B5F8BCB00022DA4535
:10D7D8004FF000034FF000014C4898BF1FFA8AFB36
:10D7E800F8F750FB804650B1F8F72AFB4A4B5A46E7
:10D7F80003EB00134946404667F098FC8046B5F8AD
:10D80800BC3094F8C4909A4584BF01237B607B6840
:10D818009CBF09F102095FFA89F984F8C43004F160
:10D82800C00ADAE8EF3F0133CAE8E23F002AF8D13C
:10D8380004F1140B3146584668F0B6F8A378012B6A
:10D8480056D108F10C03042118467B6066F0CEF926
:10D85800228809F0FD0942EA09320280B8F810204E
:10D868007B68043A42800221184666F0C7F94046B0
:10D87800FCF75AFC8146002843D0DAE8EF3F013B29
:10D88800CAE8E23F002AF8D13146584668F0C0F8A5
:10D89800224A4B460121224868F0A4F84046F8F78E
:10D8A8006FFB20463146FFF71FFBB5F8BC301D481B
:10D8B800002B08BF002024F053FF6FF004056E46CC
:10D8C80088B0194A0423CDE905256A46079442F829
:10D8D800103F4FF4015112480023F6F761FC132161
:10D8E800B546204668F0D5F82046FFF7AFFCA1E61C
:10D8F8006FF01509C1E76FF079052FE76FF00405A0
:10D908002CE7FCF78FFCEFE79368FFDEAC1F0020E5
:10D9180080010020E41E00208C620020385F0A008D
:10D92800286B090040020020406B0A0040F2E243E5
:10D938002DE9F041D0F888600446B6FBF3F6031DE4
:10D94800184668F04CF88204B6B213D5B4F88C20A7
:10D95800B2420FD8B4F88E20B2420BD3D4E92412C5
:10D96800914207D1D3E8EF1F21F40051C3E8E21F29
:10D97800002AF7D1104B1D6865B155F80C7C1C3D89
:10D9880037B131462046B4F89230B4F89020B84701
:10D99800ED69F1E7094DDFF82880454501D3BDE879
:10D9A800F0812F6937B131462046B4F89230B4F887
:10D9B8009020B8472035F0E700630020C06A0900CE
:10D9C800006B09002DE9F041074608460D4667F04F
:10D9D80064FC064618B900263046BDE8F081144BB1
:10D9E8001C6884B154F8103C1C3C0BB9E469F8E796
:10D9F8002946384698470028EDD0284667F04DFC60
:10DA08000028F3D1E7E70B4CDFF82C804445E3D23C
:10DA1800E3680BB92034F9E72946384698470028C7
:10DA2800D9D0284667F039FC0028F3D1D3E700BFE6
:10DA380000630020C06A0900006B09002DE9F0416D
:10DA4800C37804468BB900F17E06114B1D687DB181
:10DA58001C3D04F170076B691BB13A4631462046FC
:10DA68009847ED6925B11C3DF5E700F17706ECE72D
:10DA7800084D094F04F17008BD4201D3BDE8F0819B
:10DA88006B691BB142463146204698472035F3E77B
:10DA980000630020C06A0900006B0900F8B5437AEA
:10DAA80004468372164668F0C6F9144B1D684DB1DA
:10DAB80055F8043C1C3D1BB132462046617A984714
:10DAC800ED69F4E70E4D0F4FBD420DD3A6B9637A49
:10DAD800012B11D9A378012B0ED1207A04F1700102
:10DAE800BDE8F84006F030BFAB691BB132462046AE
:10DAF800617A98472035E7E7F8BD00BF006300204A
:10DB0800C06A0900006B090038B505460C460F4885
:10DB18000521FFF7E9FAC0B1057223680367A388F6
:10DB2800A0F87430A37980F87630012343728372A9
:10DB38008370074BC0F8A830064BC0F8AC30064BD2
:10DB4800C0F8B030054BC0F88C3038BDF82F002035
:10DB5800B5E20000D1590700C55907001800280090
:10DB68002DE9F0410746884600250E4E304667F0FD
:10DB780079FF044620B18378012B0AD0FFF766FBB2
:10DB88000135052D06F1D006F0D100242046BDE868
:10DB9800F0814246394668F070F80028F6D12046F0
:10DBA800ECE700BFF82F0020F0B589B000AF0D46B4
:10DBB800FFF7D6FF044618B329463846FBF762F943
:10DBC800637B6D46082B98BF0F4A8AB094BF52F802
:10DBD80023300E4B6A46CDE907730D4B0D49099367
:10DBE8000D4BCDE9051442F8103F00234FF4425184
:10DBF8000A48F6F7D5FA2046AD46FFF727FB01207D
:10DC08002437BD46F0BD00BFD47409005A6A0A0023
:10DC180001030204636B0A0005000002286B090077
:10DC280038B50446134867F0DAFE420702D46FF0AD
:10DC38000A0038BD084667F030FB10B96FF01500D0
:10DC4800F7E7FEF71BFF0028F1D10A4867F0C7FE87
:10DC58000306C0F3C0150AD467F06EFD0028EDD0A6
:10DC680021462846FFF7A0FF0028E2D0E6E76FF03C
:10DC78007700DEE7080200202DE9F04706460F4648
:10DC8800904600254FF0D009DFF844A009FB05A015
:10DC980067F0E8FE044620B18378012B06D0FFF731
:10DCA800D5FA0135052DF1D100240DE037B13A46FA
:10DCB800314667F0E2FF08B92046F0E7637B434549
:10DCC800FAD1237AB342F7D12046BDE8F08700BFE6
:10DCD800F82F002070B58B780646012B0C4692B0C1
:10DCE80042D191F8703007AD032B37D8DFE803F045
:10DCF800023032341E492846F3F772FA059594F833
:10DD080071301E21049394F872301A4A039394F8E0
:10DD180073300AA8029394F87430019394F875301C
:10DD2800009394F876305FF091FE32460AAB10AD5E
:10DD38001C4603CCAC4210605160234602F1080235
:10DD4800F6D1206810603046A388938012B070BD69
:10DD58000949D0E70949CEE70949CCE70A2128460D
:10DD6800084A5FF073FEC9E700238DF82830DCE726
:10DD780084580A009F580A00AABA0A008B580A0059
:10DD880095580A003C7A0A00002210B583780446A8
:10DD98000B70C3784B70037A8B70437B81F8232018
:10DDA800023BDBB2062B8EBF13462848C35C2046D5
:10DDB80081F82030A378012B14BF0023637A81F8FF
:10DDC800213067F0ECFE81F82200A378012B3AD1CC
:10DDD80004F170038B60237A1D4AC3EBC303134419
:10DDE8004B60E27804F1770304F17E0012BB1A4617
:10DDF8000346C1E9032340F2E242D4F888304B617C
:10DE0800B3FBF2F30B83B4F890304B83B4F8923041
:10DE18008B83D4F8A4302BB15B7CDA0644BF012392
:10DE280081F82330D4F8A43013B15B7C9B0603D46B
:10DE3800002010BD0246DCE791F8233043F00203CE
:10DE480081F82330F4E76FF01500F2E779CA0A0089
:10DE5800800100202DE9F04104460F4615469846FA
:10DE6800002B6ED01B6823B10221394A394865F06E
:10DE780068FA29462046FFF7D3FE064600283FD118
:10DE88002046294667F0CFFE044600285CD097E874
:10DE98000F00314D05F1080C8CE80F00AB8A002B00
:10DEA80008BF4FF49673AB822B8A03B9AB892B82D8
:10DEB8006B8A03B9EB8929486B8267F090FD4305AB
:10DEC80001D5FDF797F995F8DB2095F8DA309A42F5
:10DED80019D903212046FFF705FA0220FEF7CAFAEE
:10DEE800054658B10220FEF7EDFA20460021FFF75B
:10DEF800F9F92046FFF7AAF92E4601E0C8F80040D4
:10DF08003046BDE8F08102212046FFF7EBF92046B4
:10DF180067F0ECF905460028F0D00021204621736F
:10DF2800FFF7E0F92046FFF791F90320FEF7A2FA80
:10DF380003460028E0D00221094A064867F052FD4E
:10DF4800DAE76FF01506DBE76FF00B06D8E700BFDE
:10DF58009C6B0A00286B0900800100200802002041
:10DF6800D25A0A0038B5044608460D4667F095F9B6
:10DF780038B3154B93F89030990707D4E37873B109
:10DF880029462046BDE8384000F042BB94F8993055
:10DF98009A07F3D5201D67F022FD4304EED42946E5
:10DFA800204667F090FE58B92B88A4F88C306B880F
:10DFB800A4F88E30AB88A4F89430EB88A4F8963097
:10DFC80038BD6FF01500FBE780010020F7B510F8A9
:10DFD800333C0446A0F140060BBB304667F0CEFE4A
:10DFE8003C4B1D684DB155F8183C1C3D1BB13046E3
:10DFF80014F8341C9847ED69F4E7374D374FBD42A4
:10E0080005D3304603B0BDE8F040FFF71FB96B6891
:10E018001BB1304614F8341C98472035EFE710F848
:10E028003E3C012B53D110F83D3C8BB9FCF726FB45
:10E0380069304CD102212A4A2A4865F082F940F217
:10E0480039120023204603B0BDE8F04024F05EBE3C
:10E05800A0F13C05D5E8EF3F23F40052C5E8E12FD5
:10E068000029F7D199041FD5E36C69460093636DC5
:10E0780030460193FFF776FF034678B9D5E8EF3FBE
:10E0880023F48053C5E8E23F002AF7D14FF400613A
:10E09800284603B0BDE8F04067F0A6BC124A02214A
:10E0A800104867F09FFCF1E74FF428130F4A6946C0
:10E0B8003046CDE90023FFF755FF034628B94FF452
:10E0C8008051284667F090FCE0E7094AE7E703B08B
:10E0D800F0BD00BF00630020C06A0900006B0900A2
:10E0E800D16B0A00286B0900046C0A00180028008C
:10E0F800296C0A0008B568B1094B00F10C011A68CF
:10E1080022B9074867F050FC104605E0914204D058
:10E118001268F5E76FF0150008BD6FF07700FBE7B0
:10E12800086300202DE9F0411C486CF01BFB1C49DA
:10E138001A486CF055FB1B4918486CF051FB1A49FA
:10E1480016486CF04DFB68F082FA04F0B3FA044606
:10E1580000BB06F097F80446E0B967F0CEFE264605
:10E16800A046124F384667F07DFC054668B104307A
:10E1780067F035FCC30705D50321284685F80880D4
:10E18800FFF7B0F82846FFF761F80136052E07F1CA
:10E19800D007E7D12046BDE8F08100BFE41E00208B
:10E1A800DC620020E8620020F4620020F82F0020E2
:10E1B80003460121014A024865F0CCB8DC6C0A002C
:10E1C800986B090080B500AF88B06A46074BCDE967
:10E1D8000530032342F8103F00234FF4C25104488E
:10E1E800F5F7DEFF6FF00B00BD4680BD046D0A0039
:10E1F800986B090070B500225026094D06FB02F302
:10E208005C19EB583BB10132052AF7D1FFF7DAFF69
:10E218006FF00B0003E01846024A62600C6070BDA4
:10E22800146300202075090070B5044652EA030003
:10E2380008D0F7F7EFFA074D074ED5F8E0503058F9
:10E24800854201D1002213462046BDE870400431C2
:10E25800FFF7A2B9104F00200800000038B50546A6
:10E2680018462B68DBB15B7B072B18D10B7A012B87
:10E2780007D001210B4A0C4865F06CF86FF01500C7
:10E2880038BDCB7A072BF9D9C8618A6105F130000E
:10E298006CF0A6FA284667F048FD0020F0E76FF01A
:10E2A8007F00EDE72B6D0A00986B09002DE9F84F08
:10E2B80088469146D0F8B44000AF44B1483C236B3F
:10E2C80063B92068B43067F04FFDA46CF5E7FBF73D
:10E2D800A9FF00263046BD46BDE8F88F04F1300A94
:10E2E80050466CF0A2FA05460028F0D066F059FFB7
:10E2F80080B16C4688B06A46294BCDE905350323C1
:10E3080042F8103F00234FF4C2512648F5F748FF62
:10E31800A546DEE7284665F0E5FBE56C06469DB9AF
:10E32800A38C058A403B9BB23F2B03D8238D9D428B
:10E3380028BF1D46042106F10C0065F057FC058036
:10E34800A38C04354380E56445451FD8B6F810B062
:10E35800AB4506D100220023504624F0CBF9F7F74D
:10E368000FFEA38CA3F140023F2A06D8AB451ABF83
:10E37800002213460C4AF361B2612068B43067F09A
:10E38800F3FC236B13B1204667F0CFFCE36C984590
:10E398002CBF0021A3EB0801C9F80030E16499E71C
:10E3A800436D0A00986B0900B55E0700F7B504468F
:10E3B8000026234D234FBD4201D303B0F0BD298869
:10E3C800204667F06AFD6B68019001A920469847CE
:10E3D800002830DB019B2A889A829A8403F1100274
:10E3E800D2E8EF1FC2E8E06F0028F9D19E64DE642E
:10E3F8009E60A16B03F10802F9B9C4E90D221C6003
:10E40800DE6003F130006CF0ADF9019843681B68D9
:10E4180003B19847019B1033D3E8EF1F41F0010186
:10E42800C3E8E21F002AF7D101984368DB6913B1FA
:10E4380000F1100198470835BDE70A60A263DEE7DE
:10E44800A86A0900C06A09007FB50D46064604217E
:10E4580005F10C0065F0E3FB2A8A438804469342E1
:10E4680008D000931346444A0121444864F07CFFD5
:10E4780004B070BD417839B90121414A3F4804B020
:10E48800BDE8704064F05DBF0278122A22D0132ADA
:10E498001AD0012AECD0022113463848394A64F0D0
:10E4A80059FF617802220120356867F0DCFC0446D8
:10E4B8000028DDD002210C3065F064FB00232146E2
:10E4C80003704370284624E0022BD1D00222009228
:10E4D8002D4AC9E7082B03D0082200922B4AC3E72C
:10E4E8003468637B072B02D00221294AC6E7E37808
:10E4F800A3B10222012067F0B6FC05460028B7D078
:10E5080002210C3065F03EFB00232946037043705E
:10E51800204604B0BDE8704067F0D5BCEB68132016
:10E528001A88ADF808205A88ADF80A209A88ADF8FC
:10E538000C20DB880222ADF80E3067F094FC05460B
:10E54800002895D002A92046FFF73CFA064602218A
:10E5580005F10C0065F016FB86F00103DBB20380C1
:10E568002946204667F0AFFC002E81D0204602A93C
:10E5780067F0A9FB7CE700BF5B6D0A00986B090098
:10E588007C6D0A00086E0A009D6D0A00C86D0A00BD
:10E59800FA6D0A0008B50B8A032B06D80121044A34
:10E5A800044864F0CEFE002008BDFFF74DFFFAE7EF
:10E5B800306E0A00986B090038B50B8A0546032BA4
:10E5C8000C4609D801210F4A0F4864F0BAFE2046CC
:10E5D800BDE83840F7F7D4BC042104F10C0065F01D
:10E5E8001EFB4188284667F07FFC30B9074A0B4676
:10E5F8000548022164F0AEFEE9E7436821465B69FD
:10E608009847E4E74E6E0A00986B09006B6E0A00A3
:10E6180070B5134A0C4613780646013313F0FF0110
:10E628000ABF01230B46194613701220082267F00F
:10E638001AFC054688B108210C3065F0A3FA228837
:10E648002946028062884280A2888280E288C2804D
:10E658003046BDE8704067F036BC6FF00B0070BD07
:10E668002BD0002023281FD81A2804D8431E182B83
:10E678000ED906207047A0F11B03082B1ED8DFE82F
:10E6880003F0051D1B231D19251D050003207047D8
:10E6980001230F4A83401A40C2B90E4A1A40002A81
:10E6A8000CBF06200120704700F07F03522B05D1D4
:10E6B80000207047012070470520704710F0400F78
:10E6C80014BF0020062070470420704702207047BE
:10E6D800AAAA8A02545545012DE9F74F064608466D
:10E6E8000C46F7F7ADFB182343432D4F0546FA18A0
:10E6F80091680191E16806F15400D0E8AF0FC007B6
:10E708000AD40121274A284867F01AFC6FF0150936
:10E71800484603B0BDE8F08FE06800781071002229
:10E72800FA500B78D22B0FD133682146186869F05C
:10E73800FAF8814640B101211C4A1B4867F000FCE9
:10E748002046F7F71DFCE3E7182303FB0573D4F80D
:10E758000C80D4F814B0B4F810A09E6000232146B1
:10E768001A46301DFFF77AFD81460028D0D010F1F7
:10E77800690F04D101210E4A0B4867F0E1FB626979
:10E78800A8EB0B0812FA88F2E26018225543019BA5
:10E798007A19A4F810A0936047F80590B8E700BF6D
:10E7A800AC640020A76E0A00186B0900C16E0A004D
:10E7B800D46E0A0008B5EFF31181202383F3128881
:10E7C800BFF36F8F002303600F4B5A68C2B9C3E9C8
:10E7D800000081F31188BFF36F8F0C4824F0EEF925
:10E7E800031E0CDA01210A4A0A4864F0B3FD00232B
:10E7F80083F31188BFF36F8F0323184602DF08BD28
:10E8080010605860E5E700BFA464002000090020FC
:10E81800F76E0A00186B0900094B011F9A6809482E
:10E82800914204BF00229A601A6A914204BF0022F2
:10E838001A629A6B914204BF00229A636BF070BE11
:10E84800AC640020A01D00200121024A024867F0A4
:10E8580077BB00BF206F0A00186B090010B504468B
:10E8680000F15003D3E8EF1F41F00101C3E8E21FB4
:10E87800002AF7D1201F67F08CFB04F174000449CB
:10E888006CF0EEF82068BDE8104003F06BBD00BFE7
:10E89800A1F8000073B50E46438D418B01328B42BF
:10E8A80028BF0B469A42054609D9022100921D4805
:10E8B8001D4A64F059FD0024204602B070BD304660
:10E8C800FFF7D0FE6FF01403034113F0010310D0DB
:10E8D800F6F7A0FF154B1958154BD3F8E0309942BD
:10E8E8001DD0144B1B685A1A18BF4FF0FF3213463D
:10E8F80000E0114A00211148FFF796FC0446002861
:10E90800DAD0F7F79DFA18220D4B012102FB0033EC
:10E9180004F10C009D6065F035F90670CCE7002223
:10E92800E5E700BF186B09003D6F0A00080000000A
:10E93800104F0020F46400201C4E0E00281F0020F9
:10E94800AC64002070B5044601F10C000D4665F07A
:10E9580076F9266801462B8AEA68306868F07CFDFB
:10E968001E2100222046FFF795FF014630B90121FC
:10E97800044A054867F0E4FA002070BD204667F0B5
:10E98800FAFAF9E7626F0A00186B0900F0B51D463C
:10E9980003680E460039044618BF012187B018687D
:10E9A800174668F06AFD40B904F1540067F022FC8C
:10E9B800002846D0002007B0F0BD002D43D0182213
:10E9C8000021684687F066FB6FB1002213212046BC
:10E9D800FFF760FF019030B91C4801211C4A67F01D
:10E9E800AFFA1120E7E7236829461B6828460093F9
:10E9F8000023ADF812300C9B164A0393BDF834304F
:10EA08008DF80860ADF8103001238DF814306B468E
:10EA180067F098FB9DF8143063B1002FCAD00198B5
:10EA2800F7F7AEFA2A46314620469DF8143067F0CB
:10EA3800ECFBBFE701990029BCD0204667F09BFAA0
:10EA4800B8E71220B7E70120B5E700BF186B090047
:10EA58007F6F0A00036007002DE9F3410B8A044623
:10EA68000D4643B90121294A294867F069FA00206F
:10EA780002B0BDE8F0810768012105F10C0065F0DE
:10EA8800CEF87B7B0646072BF1D154F8043C002BCB
:10EA9800EDD0002203781F4F043C17F832004FEAEC
:10EAA800C208984207EBC20114D12A8A48789042DA
:10EAB80026D90121009316481346174A64F054FCDE
:10EAC80004234744BA78012AD1D1002BCFD00022A1
:10EAD800317811E001321C2ADFD1104A02210C489A
:10EAE80064F038FC31780846FFF7BCFD2122C240AB
:10EAF80012F00102BBD10623204667F086FBB6E779
:10EB08004B682046294698470346DAE7986F0A007B
:10EB1800186B090048750900CD6F0A00B36F0A0029
:10EB2800F8B5124A0746002311480D4664F098FFCD
:10EB3800044638B901212B460E4A0F4864F00AFCF6
:10EB48002046F8BD00F10C060921304665F00FF8A3
:10EB58002046F7F775F91822084B012102FB00330C
:10EB680030469F6065F00EF80570E9E71C4E0E0010
:10EB7800281F0020DC6C0A00186B0900AC64002018
:10EB88002DE9F0410E8A0446043EF6B2022E0846EC
:10EB98008CB001D0102E64D104210C3065F03FF800
:10EBA8000DF1080805884788011D3246404666F081
:10EBB80068FA002857D0A5B300268FB3AF4230D3E8
:10EBC8004FF42053404601A98DF80460ADF8063093
:10EBD80066F02AFA48BB1422002107A887F05AFADF
:10EBE80011212046FFF79CFF0990002837D001210A
:10EBF8000C30CDE9074864F0C5FF00230A90394678
:10EC080003701A4A0B93284607AB67F09BFADDE9B5
:10EC180009131B78FBB90846F7F7B2F90A2301E094
:10EC28003D4601232A4610210EE042F601034046E4
:10EC380007A98DF81C60ADF81E3066F0F5F90028BC
:10EC4800C9D010232A461946204667F0DEFA00206C
:10EC58000CB0BDE8F081204667F08DF9F7E7112088
:10EC6800F6E70420F4E70E20F2E700BFCDF100003C
:10EC78002DE9FF41036804460D461868012168F034
:10EC8800FCFB40B904F1540067F0B4FAA0BB1220B1
:10EC980004B0BDE8F08110220021684687F0FAF937
:10ECA80021212046FFF73CFF029038B34FF00108BE
:10ECB800009405F10C072B8A012B04D820460299F1
:10ECC80067F059F918E0384664F0B9FF6B46014619
:10ECD8000B4A06468DF80C8067F034FA9DF80C3024
:10ECE800002BE8D00298F7F74BF93246202120464E
:10ECF8009DF80C3067F089FA0020C9E71120C7E7B2
:10ED0800756407002DE9FF41036804460D4618683D
:10ED1800012168F0B2FB40B904F1540067F06AFAC7
:10ED2800A0BB122004B0BDE8F08110220021684683
:10ED380087F0B0F90F212046FFF7F2FE029038B3B2
:10ED48004FF00108009405F10C072B8A012B04D819
:10ED58002046029967F00FF918E0384664F06FFF13
:10ED68006B4601460B4A06468DF80C8067F0EAF9B7
:10ED78009DF80C30002BE8D00298F7F701F93246DD
:10ED88000E2120469DF80C3067F03FFA0020C9E7B5
:10ED98001120C7E7F9640700F0B51D46036804466B
:10EDA8000E4685B001211868174668F066FB38B929
:10EDB80004F1540067F01EFA50BB122005B0F0BDF4
:10EDC80065B310220021684687F064F93946204669
:10EDD800FFF7A6FE029018B3BDF828302946ADF813
:10EDE8000430012328468DF80C300E4A6B460094F7
:10EDF80067F0A8F99DF80C3002995BB10846F7F75F
:10EE0800BFF82A46314620469DF80C3067F0FDF9D8
:10EE18000020D3E7204667F0AEF8F9E70120CDE7F8
:10EE28001120CBE7F96407002DE9F0410E8A04466A
:10EE3800043EF6B2022E08468CB001D0102E76D1D0
:10EE480004210C3064F0EBFE0DF1040805884788B6
:10EE5800011D3246404666F014F9002869D085B392
:10EE680077B3BD422DD80121606868F006FB0646DD
:10EE780078BB42F602038DF8000069464046ADF8BB
:10EE8800023066F0D1F820B342F60303404606A9E3
:10EE98008DF81860ADF81A3066F0C6F8C8B1012DC3
:10EEA80003D14FF6FF739F4213D004F1540067F06B
:10EEB800A1F9002814BF002012200CB0BDE8F08191
:10EEC8003D4601232A460821204667F09EF9002086
:10EED800F3E7182200210DEB020087F0DBF8092187
:10EEE8002046FFF71DFE0890F8B101210C30CDE94E
:10EEF800064864F047FE0023099003700A23394648
:10EF08008DF82C30284606AB0B4A67F01BF99DF8A4
:10EF18002C3008992BB10846F7F732F89DF82C30B9
:10EF2800D0E7204667F027F8D1E71120C5E704208D
:10EF3800C3E70E20C1E700BF85F200002DE9F043CA
:10EF48000F460446062187B007F10C0064F067FEFF
:10EF58000588EDB1B0F80280B8F1000F17D045452B
:10EF680016D8002382888DF800308DF804304FF4CD
:10EF78002053684601A9D7F80C90ADF80220ADF8E7
:10EF8800063066F051F8064660B10A2301E04546AE
:10EF980001232A460621204667F037F9002007B0EA
:10EFA800BDE8F0830146142201A83F7C87F072F87F
:10EFB80007212046FFF7B4FD0290D8B10A23414645
:10EFC8008DF81530284601AB0B4ACDE90369019449
:10EFD8008DF8147067F0B6F89DF8153002992BB1CA
:10EFE8000846F6F7CDFF9DF81530D2E7204666F0C3
:10EFF800C2FFD3E71120D2E771F000007FB5CB68DC
:10F0080004461D888DB15E8876B1B5420DD81022B0
:10F018000021684687F03EF805212046FFF780FD6D
:10F02800019058B9112007E0354601232A460421EA
:10F03800204667F0EAF8002004B070BD6B46314600
:10F048002846084A009467F07DF8DDE9011323B9E2
:10F058000846F6F795FF0A23E8E7204666F08BFF97
:10F06800E9E700BF756007002DE9F04342F60103A8
:10F07800002591B0D2F8008006460F4600680BA91B
:10F08800D8F8049014468DF82C50ADF82E3065F061
:10F09800CBFF00286DD04FF4205330680BA98DF8B2
:10F0A8002C50ADF82E3065F0BFFF38B1A3681BB106
:10F0B8005A88BA4200D25F80012010E06168084691
:10F0C80066F026FFB8F82A20B8F81A309A4294BF9A
:10F0D800C0EB0200C0EB0300032803D8002011B0E6
:10F0E800BDE8F083084664F004FD054661680846FB
:10F0F80066F00EFF6B8A2A8AA3EB020C6B69EA683A
:10F10800D21AACEB0203B8F82AC0B8F81A20944512
:10F1180094BFC0EB0C00C0EB0200834228BF03463B
:10F128006BB9887AF6F784FE0022002364F098FC15
:10F1380005460028D2D00146606864F0EBFC002345
:10F1480000933146D6F804801023484602AAC047E7
:10F15800061E0EDB227CE068964227D001460BA8EB
:10F1680065F08FFF40B9237C134A0221134864F0ED
:10F17800F1F80023A3609FE7F2B202A906A865F0A0
:10F1880080FF10B90E4A3346EFE706A90BA865F0D1
:10F198004BFF0028EDD100230421637405F10C0016
:10F1A80064F0F0FCA0600780A36884E7324602A9F7
:10F1B80086F078FFEDE700BFEC6F0A00186B0900D6
:10F1C8000B700A002DE9FF414FF000084FF420535F
:10F1D80005460E46006802A9144617688DF808808F
:10F1E800ADF80A3065F020FFA0B142F601032868A7
:10F1F80003A98DF80C80ADF80E3065F015FF48B105
:10F2080023691BB15A88B24200D25E80012004B043
:10F21800BDE8F0816168286865F006FF10B1002339
:10F228002361F3E7E368A0681A786AB1B7F81AC0EF
:10F23800798D038A8C4594BFC3EB0C03C3EB0103A0
:10F24800934201DA0020E2E704210C3064F09AFCD2
:10F2580020610680236929465E80074B019400934C
:10F2680038460023A26867F078F80028EADB2069AE
:10F27800003818BF0120CAE72D6107002DE9F347C0
:10F28800176805468946006851681446D7F804A0EF
:10F2980065F0CAFE804600284BD195222946504683
:10F2A80067F04CFF0646207540B1E3681B780BB148
:10F2B80084F81480002002B0BDE8F0872946504643
:10F2C80068F014F910B908232375F3E7A0682675C8
:10F2D80064F00FFC02210C3064F054FC164B2061E2
:10F2E800A0F8009000930194334629463846A26856
:10F2F80067F033F8002807DA10F1FF0F32BF0E204D
:10F308004042C0B22075D5E72369002BD2D0A0684F
:10F3180066F0FEFD7B8D7A8B9A4294BFC0EB0200AB
:10F32800C0EB0300E3681B78984294BF00200120DB
:10F33800C1E70120BFE700BF295F07002DE9F041C1
:10F3480082B000AF044688460022002339463B4875
:10F3580023F010F80546B0B16D4688B06A46384BC0
:10F36800CDE90534032342F8103F00234FF4C2517E
:10F378003448F4F715FFAD466FF00B0630460837F2
:10F38800BD46BDE8F081F6F745FA2F4B29461A58D5
:10F398002E4B38681A602C2286F07CFE3B680022CF
:10F3A8001C603C680023C4E90155C4E90955284894
:10F3B800391D7D6022F0DEFF064688B123686C4661
:10F3C80088B06A462349CDE90513032342F8103F64
:10F3D8004FF4C4512B461B48F4F7E2FEA546CBE791
:10F3E8000146B022786886F055FE78681A4B83602B
:10F3F8005C306BF0B7F97B685433D3E8EF2FC3E880
:10F40800E16F0029F9D17B681C60636A7D681BB9CC
:10F4180004F10C006BF0A6F9626A05F1A803C5F8BF
:10F42800A820A26A636202B9A36217227B685A8580
:10F438005A830433C8F80030A0E700BF841D0020B9
:10F448002A700A00186B090008000000F464002004
:10F45800A01D00204F700A00D808002008B5437B83
:10F46800072B06D002210C4A0C4866F069FD0020E3
:10F4780008BD042166F038FD10B9094A0121F3E7F7
:10F4880000F15003D3E8AF3FDB0701D4054AF5E7A5
:10F4980050F8040CECE700BFFA6D0A00186B09007D
:10F4A80074700A00A76E0A002DE9F04F85B000AF0E
:10F4B800B860EFF31188202383F31288BFF36F8FAE
:10F4C800584C204666F01AFD2668054688F31188D0
:10F4D800BFF36F8F00285FD0F6F7B2FC182202FB4B
:10F4E80000F35149C81851F803A003690021D0E975
:10F4F8000248FB6090F80490B0F806B086F0CAFDA8
:10F50800A87AF6F795FC6969034659B16A7AD00773
:10F5180006D45A6A284612687B60926890477B68CE
:10F5280000226A61294618466BF06DF9B9F1000F9F
:10F538000DD064B1236853B11B6843B1BAF1000F11
:10F548002ED001215346394A394863F003FF1EB3D0
:10F558000020B9686BF052FA00281DDA6C468AB0B0
:10F568006A46344B0593344BCDE906304FF40073AB
:10F57800ADF82030314B42F8103F00234FF41151C1
:10F588002B48F4F70DFE0023A54683F31188BFF33B
:10F598006F8F0323184602DF1437BD46BDE8F08F8E
:10F5A800201D66F0D5FF4846FFF75CF80528CED841
:10F5B80001A353F820F000BF05F60000D9F50000BC
:10F5C80057F5000005F6000057F50000D9F50000D2
:10F5D80004F15403D3E8AF3FDA0705D40121184AF0
:10F5E800134866F0ADFCB2E7A36D002BAFD0002343
:10F5F800144A04F1780023F089FBA8E754F8543B37
:10F608001D68D4E8AF3FDB07E8D5B8F1000F9ED0FE
:10F61800002403E02846F968C0470134A3B29B459B
:10F62800F8D894E7A4640020AC6400208F700A0026
:10F63800186B0900AE700A0084CA0A0004000001B1
:10F64800A76E0A001C4E0E00F8B50F461646FFF7C7
:10F6580005FFB0B1446A20461CB150F8A84904B16E
:10F66800A83C731C194638B1428B458DAA4228BF65
:10F678002A469A4207D264B902210A4A0A4863F024
:10F6880069FE0020F8BD32463946BDE8F840FFF76C
:10F6980001B9D4F8A85005B1A83D20460B462C4620
:10F6A800E2E700BFC9700A00186B090007B50B46EE
:10F6B80000210246F6F7AEF801910E4909580E48A6
:10F6C8000068884204D00D48D0F8E000884201D193
:10F6D8000022134601A90A4822F04CFE014638B917
:10F6E8001C22019886F0D6FC019803B05DF804FB53
:10F6F8000020FAE708000000F4640020104F002002
:10F70800BC1D002010B50022044600F10803D3E810
:10F71800EF0FC3E8E12F0029F9D108B1F6F730FC63
:10F728002146BDE8104001486AF0FABEBC1D002021
:10F738002DE9F743044678300F4690461E466BF095
:10F748009DF9A06D50B90221144A154866F0F8FBDE
:10F75800204603B0BDE8F04300F086B8114B98424C
:10F768004FF0000317D045684360A06DD0F818909B
:10F77800FFF7C8FF00232068A36566F01AFF3DB1B4
:10F788002068CDF8009043463A4631460068A847BD
:10F7980003B0BDE8F0831D46ECE700BFE4700A0043
:10F7A800186B0900F8640020F7B550F8044C0546BA
:10F7B800002C55D000F1A40104F1240066F001FDED
:10F7C8002E1F05F1580700220023384622F092FF29
:10F7D800024658BB6B6D2BB101466FF0670330468C
:10F7E800FFF7A6FF002345F8043C05F15003D3E8D2
:10F7F800EF1F21F00101C3E8E21F002AF7D1636A75
:10F8080073BB04F10C0600220023304622F072FF7D
:10F8180078B9666886B92146124826606AF080FE83
:10F82800286803B0BDE8F04002F0BABEF6F7A8FBBE
:10F83800C9E7F6F7A5FBE6E7A26833689642636076
:10F8480008BFA36077683FB1B3696FF067010093A1
:10F85800002320681A46B8473046FFF753FFD8E719
:10F8680003B0F0BD841D002010B504460430FFF736
:10F878009BFF1321606866F00CF9034630B1BDE8C0
:10F8880010400121024A034863F064BD10BD00BF67
:10F89800FB700A00186B0900F0B589B0044654F8EB
:10F8A800783D00AF38461968FEF714FA6E4688B0FE
:10F8B8006A460B4BCDE905374FF40073ADF81C30A1
:10F8C800084B42F8103F00234FF4E2510648F4F782
:10F8D80067FC2046B546FFF7C7FF2437BD46F0BD95
:10F8E80019710A0003000001186B090070B550F87F
:10F8F800043C0446061F002B3BD039B1436D002B56
:10F9080037D01B7CDA0734D505231CE00568284668
:10F9180002F090FD6B7A012B2BD0646D4CB3237CE5
:10F92800DB0726D5E368002BEED030466269617CA0
:10F93800FEF7B0FF054668B9637C01210D4A0E4801
:10F9480063F008FD0E2300223046BDE870401146E2
:10F95800FFF7EEBEE368D4E90512984718B12846C8
:10F96800F6F70EFBEEE729463046FEF7B5FE00280F
:10F97800F5D170BD45710A00186B090038B5836D63
:10F98800044623B3164A934221D0CB68DD78F5B1FB
:10F99800052D406815D00F2D1AD1437A012B17D8A1
:10F9A800022166F009F908B1103011D104F178008C
:10F9B8006BF064F8A26D137C43F00103137400200C
:10F9C80038BD437A032B03D8064AD15CE9E70E25F4
:10F9D80000222B4611462046FFF7AAFEEFE700BF9C
:10F9E800F864002080CA0A0010B50C4608B301B3B9
:10F9F800FFF734FDE8B1436A3BB153F8A82902B1D7
:10FA0800A83A996D8C4206D062B90430214666F056
:10FA1800D8FB204602E02046064A9A65BDE8104019
:10FA2800FFF770BED2F8A81001B1A83913460A46EC
:10FA3800E7E710BDF8640020F8B51D460F461646E6
:10FA4800F6F7FEF91823044C03FB00400123C0E934
:10FA58000376C3800575F8BDAC64002008B585F051
:10FA68004AFB38B101210346034A044866F002FF05
:10FA78006FF0040008BD00BF6C710A00706B0900CC
:10FA880010B51846144607491022A047041E07DA85
:10FA980001212346044A054866F0ECFE204610BDC5
:10FAA8000024FBE7A834002082710A00706B09006B
:10FAB800F8B506460F460024094D15F8013CB34237
:10FAC80007D12946384666F02BFF10B10548204477
:10FAD800F8BD1034802C05F11005EED10020F7E7B1
:10FAE8008D6500208C650020F8B506460F46002479
:10FAF800094D15F8013CB34204D12946384666F051
:10FB08000FFF30B90C34602C05F10C05F1D1002041
:10FB1800F8BD02482044FBE70934002008340020DF
:10FB2800F8B506460F460024094D15F8013CB342C6
:10FB380007D13946284666F0F3FE10B1054820443F
:10FB4800F8BD0C34602C05F10C05EED10020F7E768
:10FB5800A3CB0020A2CB002038B50C4619466BB1C8
:10FB680003F114055B698AB9E268A360954200D184
:10FB7800E36000230D681A464B61A847A3685BB988
:10FB8800601C0649BDE8384066F002BF1360E368B0
:10FB98009D4208BFE260ECE738BD00BFA7C90A0074
:10FBA80070B5204B144682689A420FD1A568C66882
:10FBB80075B922793046216866F0BAFE024628B146
:10FBC8001949013066F0E4FE15701581012070BDF9
:10FBD800E0680028FBD02B888B420AD0F6D2E06878
:10FBE800A36801380433E060003818BF0120A3601F
:10FBF800EDE7256822792946304666F099FE0246E7
:10FC080060B93046084966F093FE02460028E6D0FF
:10FC18002946013066F0BCFE23791370A3685B881F
:10FC28001381DCE7B9000100A7C90A00102110B54B
:10FC38000648F9F757FB034630B1BDE810400121EB
:10FC4800034A044866F016BE10BD00BF9834002071
:10FC5800A3710A00706B0900F8B5054600260B4C25
:10FC68002746621C65B91046094966F059FE28B94D
:10FC78000136082E04F11004F2D100273846F8BDE9
:10FC88002846217865F0F9FFF1E700BF8C65002070
:10FC9800A7C90A00F8B506464C1C01F13305671ED2
:10FCA80066B12246304614F8011C65F0E6FF18B923
:10FCB8000A34AC42F3D100273846F8BD2046024941
:10FCC80066F02EFEF3E700BFA7C90A00F8B505469F
:10FCD80000260B4C2746621C65B91046094966F098
:10FCE8001FFE28B90136082E04F11004F2D10027AE
:10FCF8003846F8BD2846217865F0BFFFF1E700BF18
:10FD080020660020A7C90A002DE9F04106460F46E3
:10FD1800904665F0E2FA50B339463046FFF7E4FE04
:10FD2800054678B90446134A104666F0A0FDC0B9E6
:10FD38000C225443104A601C3946104466F028FED1
:10FD4800A5181655012105F1080001FA08F166F019
:10FD580009FEBDE8F04147F612220023074822F0C9
:10FD6800D5BF0134082C02F10C02DDD1EAE7BDE869
:10FD7800F08100BF103400200834002068340020CF
:10FD88000246014610B5042311F8010B0832F9F7B1
:10FD980067FA034630B1BDE810400121024A034822
:10FDA80066F068BD10BD00BFC9710A00706B09001C
:10FDB800022110B5094866F0D5FD084007D1084969
:10FDC800084A0B88084CA24202D300B10B8010BD30
:10FDD8005068083203449BB20120F4E70C66002007
:10FDE80002CC0020006B0900106B090008B5012146
:10FDF800024A034866F01FFE002008BDE5710A00AC
:10FE0800706B090038B514460E4B82680D469A424D
:10FE180015D122792168C06866F08AFD78B1D4F8D6
:10FE2800C8302F2B03D9FFF7E1FF002038BD04EBC2
:10FE380083021581018901335181C4F8C83001203A
:10FE4800F4E700BFB900010008B50121034A0448DE
:10FE580066F0F1FD6FF0150008BD00BF39720A00A9
:10FE6800706B090070B50B4B164682689A420ED12A
:10FE7800C5686C1C33352046316866F051FD18B1F1
:10FE88002046716866F084FD0A34AC42F3D1012043
:10FE980070BD00BFB900010008B513468168074A64
:10FEA800914209D11A791968C06866F041FD18B104
:10FEB8000023036043600381012008BDB9000100ED
:10FEC80040F239120023014822F020BF30350020CB
:10FED80008B50421084866F045FD6FF002010648A0
:10FEE80066F04BFD044866F0C2FCC30701D5FFF776
:10FEF800E7FF002008BD00BF60350020024608B5B6
:10FF08000749013066F044FD00230C3202F8043C36
:10FF1800D2E8EF1FC2E8E03F0028F9D108BD00BFD2
:10FF2800A7C90A002DE9F04385B00E4690469946C8
:10FF3800044600AF58B90121344A354866F07BFDC4
:10FF48006FF0150528461437BD46BDE8F08307F164
:10FF5800080165F043F80546A0B16D4688B06A46C9
:10FF68002C4BCDE905344FF40073ADF81C302A4B07
:10FF780042F8103F00234FF4E2512548F4F710F9F6
:10FF8800AD46DDE72046391D63F0FFFB786858B1C0
:10FF98000A2229465DF0F8FD034628B101211F4ACF
:10FFA8001B4866F067FCCBE7002007F10801FFF764
:10FFB800B7FD044620BB002EC4D01949FFF7B0FD99
:10FFC800044638B90121174A114866F034FD6FF02C
:10FFD8000B05B7E7002307F1080100F8013B66F0BD
:10FFE800D7FC04F1080104224846C047041EA9DAD8
:08FFF800012123460C4A0648D2
:020000021000EC
:1000000066F03CFC2546A1E7002EEED10660466076
:1000100086609BE7D2580A00706B090045720A009F
:100020000300000161720A00A7C90A007C720A007D
:1000300082710A002DE9F04706460D461D48002151
:1000400090461F469DF820A0DDF82490FFF732FB74
:10005000044688B1456080F811A0C0F81490C760CC
:10006000C0F818804A4651463046FFF7F1FA054677
:1000700038B92046FFF74AFB6FF00B052846BDE86C
:10008000F087002201231146FFF7DAFC2846A5601D
:1000900042464946B847054618B12046FFF736FBA9
:1000A000ECE72146304666F05EFB05460028E5D0C9
:1000B000F3E700BF1C4E0E002DE9F0471F46BDF8C8
:1000C000203006468846D1F80C90002B4ED17B1E7E
:1000D000012B4ED8012F49460CBF15781588FFF724
:1000E000DDFD0446B8B915B93846BDE8F087494684
:1000F000FFF7D4FD044638B91F4802211F4A66F0B5
:100100009EFC6FF01000F0E706F17001013066F020
:1001100043FC337A2370D9F83830DBB9B4F808A03F
:100120002581B9F83230AB4203D04946404666F0EB
:1001300088FCAA4505D00022307A06F17001FFF74D
:10014000E7FD002DD0D10E49601C66F025FC25701E
:100150002581C9E72A464146304698470028C4DB36
:1001600001380128DAD96FF00D00BEE76FF0060004
:10017000BBE76FF00C00B8E7706B09009E720A00D5
:10018000A7C90A002DE9F04180460F4616461D46D4
:10019000FFF7CAFC044680B91749FFF7C5FC0446BF
:1001A00030B9BDE8F0410121144A154866F047BC5A
:1001B000394600F8018B66F0EFFB238973B9628939
:1001C00072B926816581214611F8010B65F089F825
:1001D00080B12046BDE8F041FFF7D6BD9E4204D372
:1001E0006289AA4206D29E42ECD263892681AB4242
:1001F000E9D2E7E7BDE8F081A7C90A00B8720A00B2
:10020000706B090010B5FFF78FFC044678B101460A
:1002100011F8010BF9F736F8034620B10121044A21
:10022000044866F02BFB002323606360A36010BDCD
:10023000D7720A00706B09002DE9F047284B16466B
:10024000826807469A422DD1C5686B8E53B34FF032
:1002500000086C1C05F1330A06F17009B4F8073088
:100260009BB12246304614F8011C65F00AFDE0B946
:10027000214614F8010CFDF777FC30B1437B072BC6
:1002800008BF48F00108FCF7E5FF0A345445E5D102
:10029000B8F1000F06D16B6BA5F8328013B141465F
:1002A000384698470120BDE8F0874946307A65F026
:1002B00018F878B90B4B9D4202D1304666F0DEFD4E
:1002C0002046094966F068FB002304F8013CA4F8C5
:1002D0000730DAE74946204666F05EFBD5E700BF07
:1002E000B900010038090020A7C90A0073B50C46FF
:1002F0000546082104F11000164666F037FB12236C
:1003000004223146CDE9003228462246024BFFF74F
:1003100091FE02B070BD00BFC96E070038B505463A
:100320000C460F48012166F021FB10F0010F0D4B28
:100330000AD11D835C830A4866F09DFA830709D4BD
:10034000BDE83840FFF7C0BD198B5A8BA94202D8CF
:100350009442EFD838BD94421D83ECD9EAE700BF40
:1003600060350020103500202DE9F0419846BDF899
:1003700018300646012B174636D84344012B454614
:1003800035DCFFF76DFC044668B9FFF769FC0446ED
:1003900048B90221194A1A4866F051FB6FF010055E
:1003A0002846BDE8F081B8F1000F11D00023217A72
:1003B00021FA03F2D00703D53A78DA40D20719D5EB
:1003C0000133032BF4D13B7803F007031943217267
:1003D00006F17001601C66F0DFFA337A01212046D5
:1003E000237066F096FDDBE76FF00605D8E76FF047
:1003F0000C05D5E76FF01205D2E700BFF4720A00D2
:10040000706B090010B56FF0020104460E4866F0EB
:10041000B8FA0D4866F02FFAC20704D5002200236F
:100420000A4822F077FC204666F0D3F958B12046FE
:10043000FFF716FC38B1037ADB0704D5BDE810409E
:10044000012166F066BD10BD60350020303500200A
:1004500070B56FF00801174866F093FA40F2391250
:1004600000231548F8F7A2FD0026144C651C284609
:10047000134966F059FAB0B9237ADB0713D5294638
:10048000FDF772FB054620B166F0A5F92846FCF79A
:10049000E1FE6FF0020104F10C0066F072FA002137
:1004A000204666F036FD0136082E04F11004DDD139
:1004B00070BD00BF60350020B83400208C6500207E
:1004C000A7C90A002DE9F04385B08946164698462B
:1004D000044600AF58B90121414A424866F0AFFADC
:1004E0006FF0150528461437BD46BDE8F08307F1C7
:1004F000080164F077FD0546A0B16D4688B06A46F4
:10050000394BCDE905344FF40073ADF81C30374B4F
:1005100042F8103F00234FF4E2513248F3F744FE13
:10052000AD46DDE72046391D63F033F9786858B1F0
:100530000A2229465DF02CFB034628B101212C4AF2
:10054000284866F09BF9CBE7002007F10801FFF788
:10055000B3FA044690B9FFF783FB044638B901218A
:10056000244A204866F06BFA6FF00B05BAE70023C7
:1005700007F1080100F8013B66F00EFAB9F1000F2F
:100580002AD0022239464046B047061E07DA01212A
:100590003346194A134866F071F93546A2E73B78AD
:1005A000022E237209D00221144A0E4866F047FA3F
:1005B0000021204666F0ADFC94E77B78012B05D93D
:1005C0000F4A3146074866F059F9F1E7204603F033
:1005D000010166F08EFC85E72046FFF793FC81E77A
:1005E000D2580A00706B090045720A00030000012E
:1005F00061720A0020730A0082710A0042730A00C5
:1006000096730A0037B504460D46FFF755FA0246C1
:10061000D0B1037A0C308DF8043066F02CF910F06C
:10062000010318BF01238DF80530022301AA2946D2
:100630002046F8F72FFE034620B10121034A044863
:1006400066F01CF903B030BD0346F0E7E7730A001B
:10065000706B090070B500250A4C661C0A493046CB
:1006600066F062F9014630B9204666F042FC314638
:100670002078FFF7C7FF0135082D04F11004ECD1F5
:1006800070BD00BF8C650020A7C90A0008B5012114
:10069000114866F06BF9C3071CD4FFF78DFB0F49B7
:1006A0000F486AF0E1F9002340F239120C48F8F7DC
:1006B00077FC0C490C486AF0D7F902210B4866F028
:1006C00055F90B480B496AF0CFF9BDE808400A48D4
:1006D000FDF714BD08BD00BF0C6600204570070083
:1006E000B8340020C11201003035002060350020F0
:1006F00068340020D57007001009002003462DE95A
:10070000F04148B1008A38B901244FF0140C114966
:10071000DFF844E0714501D3BDE8F081D1E900760E
:10072000BB4204D30CFB0672143A93420ED93444F4
:10073000A2B214460831EDE70CFB0578434507D01B
:1007400001356219AE4292B2F6D1F2E70025F8E720
:100750001046E1E7006B0900106B09002DE9F74F27
:1007600099464FF6FF73BDF830400746002C08BF8E
:100770001C46444B90461B880091834252D2424B08
:100780001D68002D43D04FF0140B083DAE682EB10C
:1007900056F8083C1B8ABB4203D900266B689E4270
:1007A00043D3AD68002D32D0083DEFE773682B448A
:1007B000BB4234D29DB20836344B9E42F6D3DEE7BC
:1007C0004046D15864F034FCA0B101350AF1010A69
:1007D000ADB273685345EED9009B9D4217D8BD4218
:1007E000F3D3142303FB0AF3326802EB030BB8F1D3
:1007F000000FE5D1B9F1000F0CD1013CA4B229469C
:1008000058460E9A0D9B98470CB10028DDD103B0D5
:10081000BDE8F08FDBF80C309945D6D1EDE74FF00D
:10082000000AD6E701251A4EC6E70BFB06F2296837
:10083000009801EB020ABAF810309842E7D39F42C1
:1008400018D8B8F1000F0DD1B9F1000F14D1013C47
:100850001946A4B250460E9A0D9B9847002CD6D04C
:1008600040B9D4E740468958019364F0E1FB019B0D
:100870000028E9D0013691E7DAF80C209145F9D14A
:10088000E5E700BF02CC002010660020106B0900D5
:10089000006B090010B59EB010220021684685F05B
:1008A000FDFB142200210DEB020085F0F7FB4FF455
:1008B0001053ADF8103080231022ADF812304FF4F1
:1008C0008063284C6946CDE906340DEB02001CAB71
:1008D00084F0A4FA034630B1234A0121234865F08D
:1008E000CDFF1EB010BD014648220AA885F0D6FBF8
:1008F00022461C990AA884F0FFFB034660B101213F
:100900001B4A1A4865F0BAFF1C9884F0BDF90346EB
:100910000028E6D0174AE0E74FF6FF710120164A9B
:100920000AAB66F084FB1022144904AB0AA884F0D9
:1009300001FC04461C9884F0A7F914B1104A234620
:10094000CBE708220D4B03F11001187811F8014D87
:10095000013A03F8014B0870F7D10821094866F005
:1009600005F8BEE70002C00310740A00706B0900AE
:1009700039740A0057740A0081680700983400200F
:100980006D740A00603500202DE9F04118490446D5
:10099000A1F1300015461E46BDF818706AF089F8BE
:1009A000144865F068FF010705D4FFF773FFFFF7F0
:1009B00051FEFFF73FF92046FFF752F968B1037A7D
:1009C000DA070AD500F10C04204665F054FFC3078E
:1009D00003D40221204665F0C9FF10233A4606934E
:1009E00031462846BDE8F041034B66F084B900BFAC
:1009F000E8340020603500209834002010B51B48F2
:100A000065F039FFC0F3C00080F0010408B9FFF7BA
:100A100041FF164865F02FFF0346144865F02BFF91
:100A2000DA0622D5830606D5FCB1FFF713FEBDE832
:100A30001040FFF7FFB820210C4865F097FF102207
:100A40000B49881885F032FB48B90A486AF01AF851
:100A5000BDE810406FF00101044865F092BF4FF609
:100A6000FF710120FFF75AFCDFE710BD6035002061
:100A7000983400203035002008B51021034865F077
:100A800075FFFFF7BBFF002008BD00BF60350020E9
:100A90002DE9F3470446624865F0EDFEC10713D423
:100AA000FFF78AF92368002518684FF4C053694698
:100AB0008DF80050ADF8023064F0BAFA60B96FF00A
:100AC000770002B0BDE8F087564865F0D4FE4207D3
:100AD000E6D46FF01500F4E7236801A9186841F621
:100AE00001038DF80450ADF8063064F0A1FA002837
:100AF000E5D04D4D22F0BAFC2B6826689BB9002E3C
:100B000065D1002204F10803A2606A68002A68D156
:100B1000C5E90033424865F0AEFEC30771D422F048
:100B2000B9FC0020CDE76B68002B77D053E9023287
:100B3000142101FB023333F8047C002E4FD1002F27
:100B4000DFD023681E8ABE42DBD829680029E1D0A5
:100B50000022A1F108031868008AB0424AD904F1C2
:100B60000803002A40D09168A1600029CDD093608D
:100B7000D0E7F37C318A23F08003F37489B9791CC0
:100B8000DBB289B243F080033182F3740F4609F17E
:100B9000FF3914361FFA89F9B9F1000FE9D1474638
:100BA000CDE78F42F2D301AB0846204ACDF804A02E
:100BB00066F03DFA019B43B1338A01211C4A1D486E
:100BC00065F05CFE22F066FC83E73946DEE7984676
:100BD000194A17884FF0000AB4F80490DCE7B846C9
:100BE000F8E713606B6095E76A68A1602B60002AE4
:100BF00090D1F7E7986800288CD01A46A0F1080336
:100C0000A9E71421D4E9002301FB0323108A33F858
:100C1000041CFFF783FBFFF71BFC80E71B68FFDE6C
:100C20000C66002060350020106600201768070061
:100C300083740A00706B090002CC00202DE9F04F8C
:100C4000B9B000AF0C46904638493A46D7F808018B
:100C5000994662F07AFD40B9FFF7FAF86FF0150592
:100C60002846E437BD46BDE8F08F3E68391D304662
:100C700062F08FFD3EB901212D4A2E4865F0DFFE5E
:100C80006FF015043FE0786800BB4FF0000B07F1F0
:100C9000080A5146304687F814B064F0A3F90546B7
:100CA00008B36C4688B06A46234BCDE905364FF44D
:100CB0000073ADF81C30214B42F8103F4FF4E25165
:100CC0005B461C48F3F770FAA546D9E70A220021D3
:100CD0005CF05EFF03460028D7D00121184A154872
:100CE00065F0CCFDCCE7C7F810A0E4B1C0224846BF
:100CF00007F12001C047041E07DA01212346114AEB
:100D00000C4865F0BBFD2546AAE7A40807F12003BF
:100D1000C7E906344FF6FF7101200B4A07F11003B3
:100D200066F085F99CE72346F2E700BFA4740A0049
:100D3000D2580A00706B090045720A0003000001D6
:100D400061720A0082710A00A9FB0000002330B51D
:100D5000B5B001918DF808003393044601AB0D4600
:100D600001204FF6FF710B4A66F061F9339B73B1B6
:100D70009B0003AA29462046F8F7A2FA034620B1B1
:100D80000121054A054865F079FD35B030BD1A46A8
:100D9000F0E700BF0DFE0000AB740A00706B0900A5
:100DA0002DE9F34100F17008CDE9001204460F4629
:100DB000007A4146154664F094FA06466B464FF6B3
:100DC000FF710120214A66F032F91EB14146207AB6
:100DD000FFF7BCFF3946207AFEF76EFE40B1294688
:100DE000013065F0D9FD1EB14146207AFFF70AFCBB
:100DF00094F8088039464046FEF796FE0446C8B18E
:100E000029464046FEF790FEC8B1844217D0228999
:100E1000638952EA030106D00589418995420CD8BD
:100E2000994200D24381002323606360A3600EB126
:100E3000FEF7AAFF02B0BDE8F0810281F0E7601C76
:100E4000294665F0A9FD2046F1E700BF6DFE0000D0
:100E500014212DE9F04F0646036885B01A8A0192E5
:100E6000426801FB023333F8043C029322F0FEFA9D
:100E70003C4806F1080165F0E6FF8046002866D18F
:100E800022F008FB6FF0010005B0BDE8F08F1422DE
:100E9000336802FB0535344AAB6893423BD14FF0CF
:100EA000000AEB68A3F832A05C1C03F1330B204668
:100EB0002E4965F039FD074650BB214614F8010C58
:100EC000FCF752FE034658B9214614F8010C64F0B1
:100ED00008FAA8B1214614F8010CFFF737FF0FE01C
:100EE000427B072A31D100F170013A46007A039320
:100EF000FEF70EFF039B1846FCF7ACF9002FE3D179
:100F000020461A4965F048FD04F801ACA4F807A092
:100F10000A345C45CBD195F91330002B05DA2B69E7
:100F200023F000431B0C1B042B6109F101097368BA
:100F30001FFA89F5AB42AAD80D4865F09CFCC3079F
:100F400008D422F0A7FA00209EE74746D3E74FF0E7
:100F50000009ECE7DDE90101FFF7E0F9FFF778FAB6
:100F6000EFE700BF10660020B9000100A7C90A0022
:100F70000C660020002307B50193FFF7BFFB411C5F
:100F800089B20846034A01AB66F051F8019803B0F4
:100F90005DF804FB0B6E07002DE9F04387B0437B3F
:100FA0008046072B0C46154602AF40F0A680002372
:100FB0003B7342F60303206807F10C01FB8164F0E8
:100FC00037F80646002834D1D4F80490B9F1000F60
:100FD00005D101214B4A4C4865F031FD8DE00123DC
:100FE0002146009007F10802C847031E11DA6D463A
:100FF00088B002AAD36104234449C2E9051442F827
:10100000103F4FF4015133463F48F3F7CDF8AD465A
:1010100073E0012B05D001213D4A3B4865F02EFCD1
:101020006BE03B7A13F0300F67D02046FFF7A2FF4A
:101030000446002320683B7342F6021307F10C01BB
:10104000FB8163F0F5FF18B12046FFF793FF0446DC
:10105000002642F60219206839463E70A7F8029031
:1010600063F0E6FF18BB002320683B7342F60213CF
:1010700007F10C01FB8163F0DBFF064600283CD141
:10108000D4F80490B9F1000FA3D0022300902146B8
:10109000404607F10C02C847031EA8DB022BBAD159
:1010A000BB8905EA0300003818BF012026E042F69C
:1010B00003032068391D3E71FB8063F0B9FF0028EF
:1010C000D1D04FF42053206807F108013E727B8194
:1010D00063F0AEFF0028C6D042F60103206807F196
:1010E0000C013E73FB8163F0A3FF0028BBD02046B8
:1010F000FFF740FF04460028ADD100201437BD465D
:10110000BDE8F083C9740A00706B0900DD740A0041
:1011100003750A002DE9F84315468946942269684B
:10112000064666F00FF88046002841D1022230467C
:101130006968FFF731FF00283DD000211F48AF8AC2
:10114000FEF7B8FA0237044680B11D211C4B4761F7
:101150003A464174C0F80C80436085613046FEF722
:1011600077FA074638B92046FEF7D0FA6FF00B053C
:101170002846BDE8F883012342464146FEF760FC5D
:10118000A98A07F10C00023162F000FD20F8029BF1
:10119000AA8A296984F05CFF21463046A76065F081
:1011A000E2FA05460028E3D02046FEF7AFFADFE773
:1011B0004FF0FF35DCE76FF01505D9E71C4E0E0048
:1011C0001D68070070B505468AB03A4865F053FBC4
:1011D00042070C4667D515B16B7B072B66D1666855
:1011E00030460596FFF78AFA2268ADF81800002A03
:1011F0002FD005A9029130490023019101210091CE
:101200004FF6FF710593FFF7A9FA059E1EB96FF01F
:1012100001000AB070BD6660002330688DF81030A0
:1012200042F6030304A9ADF8123063F001FF40B9A0
:101230000598C3689B799B0608D565F0B1FEADF8AB
:101240001800059865F053FF606028B96FF015002D
:10125000DFE70028E0D1DAE7BDF818003DB101234F
:10126000014622462846A375FFF754FFD1E76FF0E9
:101270007F0307930223ADF8203042F60213ADF846
:10128000123005ABA57502930C4B4FF6FF7101931D
:10129000012304AA00932B4609948DF81050FFF700
:1012A0005DFA0798B5E76FF00A00B2E76FF07F00CC
:1012B000AFE700BF080200204B68070031150100AE
:1012C00073B5044650F8083C00F130056FF0010199
:1012D000A0F120062846019365F053FB0D4B00203A
:1012E00044F81C3C0C4B314644F8183C01AB44F824
:1012F000103C042324F8080C24F8060C24F80C3CB9
:10130000FFF760FF18B90221284665F02FFB02B0F5
:1013100070BD00BF64760900050401002DE9F84F97
:1013200090463D4B826805469A4200AF70D1D0F896
:101330000C90D8F8004009F1010609F1330AB6F81B
:101340000730F3B13246204616F8011C64F099FCD0
:10135000B8B14FF495722946204665F0F3FE30B3DC
:10136000032812D1EB4688B06A462C4BCDE90535EF
:1013700042F8100F00234FF4C4512948F2F714FF2C
:10138000DD460A365645DAD142E0052820460CBF34
:101390004FF0030B4FF0020B64F043FC834506D97A
:1013A00098F804305B45ECD288F804B0E9E7494688
:1013B000284665F046FB1B4B994529D1207A04F15C
:1013C0007001FEF7B1FB054610B303890BB94389E1
:1013D000F3B12046FCF7D8F82A89134B134923F8B8
:1013E00020206A8903EB80035A80182202FB001137
:1013F0000B6104230E4A20464A600E4A8B828A60A3
:10140000FFF7E0FE20B101210B4A054865F017FB0C
:101410000120BD46BDE8F88FB90001001C750A0027
:10142000706B0900380900208ECB00201465002065
:10143000647609002F6F070030750A0070B5044606
:101440008AB0384865F017FA42070D4663D514B1E3
:10145000637B072B62D16E6830460596FFF74EF925
:101460002A68ADF81800002A2FD005A902912E494C
:1014700000230191012100914FF6FF710593FFF7C1
:101480006DF9059E1EB96FF001000AB070BD6E6067
:10149000002330688DF8103042F6030304A9ADF83C
:1014A000123063F0C5FD40B90598C3689B79DB062F
:1014B00008D565F075FDADF81800059865F017FEC4
:1014C000686028B96FF01500DFE70028E0D1DAE79F
:1014D000BDF818002CB101462A46204665F06DFE85
:1014E000D3E76FF07F0342F6021207930123ADF8B2
:1014F000122005AA02920D4AADF82030CDE9003243
:101500004FF6FF71234604AA09958DF81040FFF7A6
:1015100025F90798B9E76FF00A00B6E76FF07F008A
:10152000B3E700BF080200204B6807003115010037
:101530002DE9F84F14463F4B826880469A4238D1D5
:10154000D0F80C903C4B99451BD100263B4D2846CA
:101550003B4965F0E9F978B90722294615F8010CED
:10156000FCF78EFB40BB236929461A6915F8010C6C
:1015700053881288FEF706FE0136082E05F10C0589
:10158000E5D109F1010709F1330AB7F80720A3896A
:101590009A420BD1394617F8010CFCF7E5FA0646DA
:1015A00020B1437B072B0AD0FBF754FE0A3757457F
:1015B000EBD14FF0010B2AE0FBF74CFEDCE7D9F84A
:1015C0003C3023B14146984708B93046ECE79422B5
:1015D0004146304665F0B6FD83460028F5D1A38923
:1015E000022B17D1B7F807309A0720D53046226969
:1015F000A188FFF78FFD054618B92269937D013355
:1016000093753046FBF726FE002DA560CEDA5846CE
:10161000BDE8F88F012B0AD1B7F80730DB0706D5F4
:1016200030462269A18865F0C8FD0546E9E75D46B8
:10163000E7E700BFB900010038090020A3CB002074
:10164000A7C90A0073B5437B0446072B0D461AD180
:10165000061D4FF48031304665F088F9C30315D478
:1016600002232046CDE900332A460A4B0A49FEF7F9
:10167000E1FC044620B16FF48031304665F081F919
:10168000204602B070BD6FF07F04F9E76FF0770479
:10169000F6E700BF8D6A07005368070070B5437B0B
:1016A0000546072B0C4686B040F0A1800B7C062B2C
:1016B00010D8DFE803F004045A5A629528000B683A
:1016C000CBB11B784BB1022B13D00121494A4A48B8
:1016D00065F0D4F86FF0150009E0082301930623A4
:1016E000224600934549464B2846FEF7A3FC06B028
:1016F00070BD1623F2E7102304212246CDE9003104
:10170000404B4149F0E708680028E3D00678002EF6
:10171000E0D14FF4245302A98DF80860ADF80A30E7
:1017200063F086FC08B342F60213206803A98DF823
:101730000C60ADF80E3063F07BFCB0B142F60313E1
:10174000206804A98DF81060ADF8123063F070FCC9
:1017500058B142F60413206805A98DF81460ADF85D
:10176000163063F065FC0028B4D108230422274911
:10177000CDE900322246264BB6E7086880B3002642
:101780004FF4205302A98DF80860ADF80A3063F0D9
:101790004FFC00289ED042F60103206803A98DF873
:1017A0000C60ADF80E3063F043FC002892D042F696
:1017B0000203206804A98DF81060ADF8123063F0C0
:1017C00037FC002886D042F60303206805A98DF86F
:1017D0001460ADF8163063F02BFC00283FF47AAFAC
:1017E00004232246CDE900330A490B4B7CE76FF016
:1017F0007F007CE74D750A00706B09006572070079
:10180000BF6D0700216B07001D1801004119010081
:10181000516B0700B91C0100B96A07002DE9F047B8
:101820008EB0064617461C46169D31B12A46002149
:101830006B680EB0BDE8F047184763B902213D4A16
:101840003D4865F0FCF82A46002130466B68984711
:101850000EB0BDE8F0871378062B08D0142B05D006
:101860000121364A344865F009F8ECE702214FF0CF
:101870000008C146013C8DF81010A4B207F1010A1E
:101880009C420CD2002CDED1B8F1000FDBD02A46EE
:10189000414630460EB0BDE8F04765F0C5BC1422A5
:1018A000002109A884F0FAFBBAF8002093B2002BBB
:1018B000C9D0BAF802101FFA81F8B8F1000FC2D0EF
:1018C0004345C0D89DF8103013B3022B25D02B7C94
:1018D000ADF80C10002B42F6010308BF4FF4205363
:1018E000ADF8063004AB029301AB099302ABADF83F
:1018F00034200C932A4630466B688DF8049009A971
:1019000098470028A4D03B78E41AA4B29A44B7E7D9
:10191000BAF80430ADF81230D9E70AF104030DF13A
:1019200011000AF1140C53F804EB634540F804EB82
:10193000F9D1CCE762750A00706B09006C750A007A
:101940002DE9F04F93B0174680461C460A461C9D71
:1019500031B12A4600216B6813B0BDE8F04F18473B
:10196000297C022940F083804BB99B4A9B4865F053
:1019700066F82A46002140466B6898475BE03B7852
:10198000062B08D0082B05D00121954A934864F016
:1019900075FFEEE71146002642F6020A013C8DF87B
:1019A0002010A4B207F1010B9C420BD2002CE0D115
:1019B000002EDED02A463146404613B0BDE8F04F37
:1019C00065F032BCBBF800901FFA89F6002ED0D02B
:1019D000BBF802009DF82020ADF81C00BBF80410F5
:1019E000ADF81E1062B1022A15D0296831B308A8DB
:1019F00063F01EFB10B33B78E41AA4B29B44D3E718
:101A000008AA06929BF806209BF8071042EA0122DA
:101A1000ADF82220E9E70A236881A981A5F808909A
:101A20004046019200932A466E4B6F49FEF702FB37
:101A300086B2002EBED113B0BDE8F08F4FF0000388
:101A4000102200210EA88DF81430ADF816A084F0F5
:101A500025FB05AA0D9206AA109240462A466B68FD
:101A6000ADF844900DA998470028C4D1E3E70329B5
:101A700066D113B90221584A78E73B78072B02D088
:101A8000152B81D102220026013C8DF82020A4B222
:101A900007F101090DF1200A9C4287D3B9F800B083
:101AA0001FFA8BF6002E3FF464AF9DF8203063B12F
:101AB000022B13D02968F1B1504663F0B9FAD0B1C6
:101AC0003B78E41AA4B29944E6E799F8053099F80E
:101AD000062043EA0223ADF82230EBE709F10503C3
:101AE0000DF1210209F1150153F8040B8B4242F864
:101AF000040BF9D1DEE799F80230B9F803208DF82C
:101B00001E304FF000038DF8143042F6030300211D
:101B1000ADF81C200EA81022ADF81630CDF818A094
:101B200084F0BCFA05AB0D9306AB10932A464046F1
:101B30006B68ADF844B00DA998470028C0D17AE78A
:101B40002A68167876B92BB9234A0221234864F013
:101B500076FF07E03B78012B09D80221204A1F4875
:101B600064F08CFE2A46002140466B68F4E6B2F829
:101B700002A0013CA4B207F10109AAF5245A9C4233
:101B800004D2002CEED1002EECD013E7012C01D8AA
:101B9000164ADAE7B9F800B01FFA8BF6002EE1D04A
:101BA000BAF1040FDED801A353F82AF0C11B0100DB
:101BB000651B0100C91B0100D11B0100391C01007C
:101BC000032C1BD80A4AC0E7032C17D8094ABCE7E4
:101BD000032C13D8084AB8E762750A00706B090035
:101BE0006C750A00A56A0700811C010080750A0057
:101BF0008E750A009C750A00AA750A00B9F80230B1
:101C0000ADF820302B68102200210EA8039384F039
:101C100045FA039B2A460D9308AB109340466B6828
:101C2000ADF844B00DA9984700283FF404AF3B78C5
:101C3000E41AA4B29944A2E7082C01D80F4A84E719
:101C400099F802308DF8203099F803308DF8213062
:101C500099F8052099F8043043EA0223ADF82230C0
:101C600099F806308DF8243099F8073099F8082053
:101C700043EA0223ADF82630C4E700BFB8750A0076
:101C800070B5102B05461146049C0BD00121084A63
:101C9000084864F0F3FD2246284663680021BDE849
:101CA000704018472246BDE8704065F027BB00BF72
:101CB0006C750A00706B09002DE9F04F8FB0074674
:101CC000189D184629B953B90221544A544864F062
:101CD000B6FE2A46002138466B6898479BE0137889
:101CE000012B07D0022B20D001214E4A4C4864F032
:101CF000C5FDEEE70B464FF00409013880B24845B8
:101D00008DF81030E5D34FF00008B0FBF9FBC24668
:101D1000541CCDF8008004AEBBF1000F08D12A4658
:101D20003846009965F080FA75E04FF01209E4E753
:101D300023880193BDF804300093B8F1000F53D10C
:101D40009DF81030002B37D0022B3CD02968002999
:101D500045D12B7C042B4DD14FF42053304602A9A2
:101D60008DF808A0ADF80A3063F062F900283BD086
:101D700042F60103304603A98DF80CA0ADF80E30F1
:101D800063F056F980B342F60203304609A98DF894
:101D900024A0ADF8263063F04BF928B342F60303D4
:101DA000304609A98DF824A0ADF8263063F040F93B
:101DB00000BB4FF0010819E0A378E27843EA022360
:101DC000ADF81230C2E7A31C0DF1110204F11201AB
:101DD00053F8040B8B4242F8040BF9D1B6E73046B6
:101DE00063F026F90028B4D04FF000080BF1FF3B58
:101DF0004C4491E7102200210AA884F04FF9BDF865
:101E000004302A46ADF8343038466B68099609A983
:101E100098470028EAD10FB0BDE8F08F62750A003C
:101E2000706B0900C6750A0007B5437B0A46072B8D
:101E30002CD14B683BB908234FF0040ECDE9003E8E
:101E4000144B154909E0012B11D0097B5B0001936C
:101E500041B1202311490093114BFEF7EBF803B079
:101E60005DF804FB0E230F4900930F4BF5E74B89F8
:101E700033B10C234FF0040CCDE9003C0B4BE0E7F1
:101E80000A230221CDE90031094BDAE76FF07F0028
:101E9000E5E700BF116E0700B51E0100756C070075
:101EA000B56B0700356C07008D6B0700E56A07000E
:101EB000D16A07002DE9F04F85B002AF8046914608
:101EC0009A460E463C6B41B96BB925680023224601
:101ED0000093F1B24046A84730E0B1F5807F28BFBB
:101EE0000E262568F2E76368002B71D123890AF179
:101EF000FF35B4F80AB07B60ADB202F1010A002DE3
:101F00004DD099F80030AB4228BF2B46012B0AD8A0
:101F100002213E4A3E4864F0B1FC00230093224671
:101F200004212568D6E7BAF80020023B91B29BB2A3
:101F300041B90121374A364864F081FD0C37BD466E
:101F4000BDE8F08F7868884201D88B4518D26D467D
:101F50008AB002AA304BC2E905317B68C2E9073B6F
:101F6000052342F8103F00234FF422512848F2F78E
:101F70001BF9AD4600230093256822460E21A9E7F0
:101F80002281009322460021404626680AF102037E
:101F9000B0470028D2D099F80030AB4206D921468C
:101FA0004046FFF741FF0028C8DAE3E7238962894A
:101FB0009A4205D10023009325682246194689E7F5
:101FC0000133238199F80030ED1AADB29A4496E7B7
:101FD000CDF800A0134625682246A8470028ADD0BA
:101FE000238A013B9A4503DA009633462568E4E7E5
:101FF000638921460AEB030540466581FFF714FF1C
